:100000000C941D1D0C944E1D0C944E1D0C944E1DF5
:100010000C944E1D0C944E1D0C944E1D0C944E1DB4
:100020000C944E1D0C944E1D0C944E1D0C944E1DA4
:100030000C944E1D0C944E1D0C944E1D0C944E1D94
:100040000C944E1D0C9474880C944E1D0C944E1DF3
:100050000C944E1D0C944E1D0C941BDD0D94510EF2
:100060000C944E1D0C94CB5A0C94C15A0C944E1DFA
:100070000C944E1D0C944E1D0C944E1D0C944E1D54
:100080000C947C520C944E1D0C944E1D0C944E1DE1
:100090000C944E1D0C944E1D0C944E1D0C944E1D34
:1000A0000C944E1D0C944E1D0C944E520C944E1DEF
:1000B0000C944E1D0C944E1D0C944E1D0C9420520D
:1000C0000C944E1D0C944E1D0C944E1D0C94705DA2
:1000D0000C94465D0C944E1D0C944E1D0C944E1DBC
:1000E0000C944E1DFD1E431F491F701F7D1F861F50
:1000F000911F5527752851298429E134E1349F2A1D
:10010000422B5128E134E134DF2C782EB02EE1343B
:10011000AE30E134E134FF31E134E1348932BC32D4
:10012000E1343833F433BF2EC72EEB2E0F2F432F7D
:10013000E62FFA2F133020302D304130FE5A045B69
:10014000165B265B2E5B5B5B325B5B5B365B3A5B15
:100150005B5B3E5B425B465B4E5B5B5B585B77C6C3
:1001600099C6B9C6DEC603C7BAC828C74BC76EC78B
:1001700093C7B8C7DDC702C827C8BAC84CC871C87A
:1001800096C848CA4BCA4FCA52CA55CA7FCA59CA2A
:100190005CCA60CA63CA66CA6ACA6DCA70CA7FCAC4
:1001A00074CA77CA7ACAFBFAFEFAEDFAF1FAF7FADC
:1001B00035FB02FB06FB0CFB10FB14FB1AFB1EFBC2
:1001C00022FB35FB28FB2CFB30FBFB0113026901F2
:1001D0004D01EF01D90195017901B1019701E701C5
:1001E0000D02C901D101D90133019B015701084A10
:1001F000D73B3BCE016E84BCBFFDC12F3D6C74313B
:100200009ABD56833DDA3D00C77F11BED9E4BB4C91
:100210003E916BAAAABE000000803F05A84CCDB25B
:10022000D44EB93836A9020C50B9918688083CA63C
:10023000AAAA2ABE000000803F000C94B02E0C94A5
:10024000701F0C9455CA0C94AE300C94BC320C94B4
:10025000FE5A0C946ACA0C94DDC70C94365B0C945D
:1002600020300C94585C0D9486000C940CFB0C947C
:1002700028FB0C94B9C60C9428C70C94DEC60C94C9
:10028000BF2E0C94C15B0C942D300C942CFB0C9461
:10029000EDFA0C9403C70C94205C0D9421000C948F
:1002A000861F0C9484290C944FCA0C9474CA0D9424
:1002B0009A000C94422B0C94782E0C9471C80C94D8
:1002C00006FB0C9413300C94265B0C94FD1E0C94CE
:1002D0000F2F0D9417000C94911F0C94BAC80C9416
:1002E00070CA0C94EF5B0C94C72E0C94F4330C94EE
:1002F000EB2E0D943D000C94B8C70C9427C80C94B9
:1003000055270C9438330C94165B0C94491F0C94AD
:1003100093C70C94432F0C94A55C0C9475280C94F3
:1003200052CA0D94FC170C9463CA0D9435000D94B9
:100330004F000C94E1340D9490000C949F2A0C947F
:1003400066CA0C9402FB0C9430FB0C942E5B0C944C
:1003500051290C945B5B0C94465B0C94FA2F0C9423
:10036000FE5B0D9445000C94425B0C941AFB0D94BB
:1003700057170C9460CA0C943A5B0C94FF310C94A0
:10038000F1FA0C944CC80C941EFB0C9496C80C9477
:1003900022FB0D9472000C944E5B0C947D1F0C9408
:1003A00035FB0D947C000C946DCA0C9477CA0C94A8
:1003B000FEFA0D94A4000C943E5B0C946EC70C9452
:1003C000585B0C9402C80C94431F0C94325B0D9440
:1003D00059000C9451280C94045B0C9448CA0D9459
:1003E0002B000C9477C60C94125C0C94E62F0C94A2
:1003F00041300C94DF2C0D940D000C945CCA0C94CD
:100400004BC70C9459CA0C947FCA0C944BCA0C94D9
:1004100089320C9499C60C9414FB0D9463000C94CF
:1004200010FB0C94FBFA0D9412000C94F7FA0C9448
:100430007ACA4E414E494E495459494E46CDCCCCCC
:100440003D0AD7233C17B7D13877CC2B329595E6A8
:10045000241FB14F0A000020410000C84200401C88
:100460004620BCBE4CCA1B0E5AAEC59D7400407AD5
:1004700010F35A00A0724E18090010A5D4E800002D
:10048000E87648170000E40B54020000CA9A3B00CB
:100490000000E1F505000080969800000040420F42
:1004A000000000A08601000000102700000000E806
:1004B00003000000006400000000000A00000000CB
:1004C000000100000000002C76D888DC674F08236C
:1004D000DFC1DFAE59E1B1B796E5E3E453C63AE6D2
:1004E00051997696E8E6C28426EB898C9B62ED40B2
:1004F0007C6FFCEFBC9C9F40F2BAA56FA5F4900501
:100500005A2AF75C936B6CF9676DC11BFCE0E40D34
:1005100047FEF520E6B500D0ED902E030094357728
:10052000050080841E080000204E0A000000C80C50
:10053000333333330F986E12831141EF8D211489B9
:100540003BE65516CFFEE6DB18D1844B381BF77C13
:100550001D901DA4BBE424203284725E228100C958
:10056000F124ECA1E53D274D323520500A4D3234BF
:10057000005072696E742050617573656400526535
:1005800073756D65005549205061757365004E6F38
:10059000204D61746368203A004D333033452D316E
:1005A000533635433455004D393939004D353032E5
:1005B0000A4D353030004D3330334530533231350C
:1005C000433855000A202A2A2A7265636461742E12
:1005D000646174615B305D203D004732380A473109
:1005E000204631303030205A313000556E737570EE
:1005F000706F72746564204F7074696F6E205365FC
:100600006C6563746564004D3139305335350A4784
:1006100032380A4732390A4D3430300A4D313034DD
:10062000533231350A4732380A4D3130395332317D
:10063000350A4D34323053310A4731583130305950
:1006400031303046353030300A47315A300A4D3576
:1006500030300A4D31313720536574205A204F66AF
:1006600066736574004731204631303030205A308F
:100670002E30004732380A473120463130303020A2
:100680005A302E30004D353030005A204F66667398
:100690006574203A202573004D353030005A204FC4
:1006A0006666736574203A202573004732385A0A0B
:1006B000473146313530305A302E30004732380A13
:1006C000473146313530305A302E30004D38340005
:1006D000473146313030305A302E30004732380AF8
:1006E000473146313030305A302E30005A204F6674
:1006F00066736574203A202573004D353030004D07
:10070000383400426567696E5377697463680072B4
:1007100065636461742E61646472203D3D0072659E
:10072000636461742E646174615B305D203D3D00E3
:1007300077616974776179203D3D000A202A2A2A71
:100740004E6F7A7A6C6554656D705374617475730D
:100750005B325D203D00434F4D4D554E4943415462
:10076000494F4E0044525952554E004552524F5235
:100770005300494E464F004543484F0047322F47EC
:10078000332062616420706172616D65746572739B
:100790000A00536C6565702E2E2E005A2050726F21
:1007A00062652050617374204265640A005A2050CB
:1007B000726F626520506173742042656400486FF7
:1007C0006D652058592046697273740A00486F6D30
:1007D00065205859204669727374004D31313720B5
:1007E00050726F6265206661696C65642E0A4732DB
:1007F000380A0070726F62655F72657769706500B4
:10080000473239205265747279696E670050726F91
:1008100062696E67204661696C6564004D313137ED
:1008200020426564206C6576656C696E6720666140
:10083000696C65642E0A4730205A31300A4D3330D6
:10084000302050323520533838300A4D3330302084
:100850005035302053300A4D33303020503235205F
:10086000533838300A4D3330302050353020533033
:100870000A4D3330302050323520533838300A4D4D
:10088000333030205035302053300A473420533134
:100890000070726F62655F6661696C6564004D31FE
:1008A000313720426564206C6576656C696E67201F
:1008B000646F6E652E00205A3A200020593A2000BD
:1008C00042656420583A20004D65736820706F6956
:1008D0006E742063616E6E6F742062652072657342
:1008E0006F6C7665640A004E6F204D6F76652E0042
:1008F000456E642066696C65206C6973740A0042F9
:100900006567696E2066696C65206C6973740A009E
:10091000526573756D6520534400286E6F206669BB
:100920006C65290043757272656E742066696C652A
:100930003A20002E0A0044656C6574696F6E20666B
:1009400061696C65642C2046696C653A20004669D3
:100950006C652064656C657465643A005072696EFC
:10096000742074696D653A20000A53746174733A97
:100970002046696C616D656E7420757365643A20FC
:10098000002C204C6F6E67657374206A6F623A208A
:1009900000546F74616C2074696D653A2000537463
:1009A0006174733A20002C204661696C65643A20BA
:1009B000002C2046696E69736865643A20005072A5
:1009C000696E74733A200053746174733A20004561
:1009D00020436F6F6C696E672E2E2E004520486590
:1009E0006174696E672E2E2E006F6666007707723F
:1009F000076B076407560744454255473A004D3197
:100A0000313320530042656420436F6F6C696E6719
:100A10002E2E2E004265642048656174696E672E33
:100A20002E2E006F6B004348414D4245525F5445A6
:100A30004D5045524154555245004D4F54494F4E2B
:100A40005F4D4F44455300544845524D414C5F5013
:100A5000524F54454354494F4E004155544F52450F
:100A6000504F52545F53445F5354415455530050B8
:100A7000524F4D50545F535550504F525400454DB6
:100A8000455247454E43595F5041525345520043EA
:100A90004153455F4C494748545F42524947485487
:100AA0004E45535300544F47474C455F4C494748C8
:100AB000545300534F4654574152455F504F57458A
:100AC00052004255494C445F50455243454E5400F4
:100AD0004C4556454C494E475F44415441005A5F8E
:100AE00050524F4245004155544F4C4556454C00DD
:100AF0005052494E545F4A4F420050524F47524560
:100B00005353004155544F5245504F52545F544532
:100B10004D5000564F4C554D4554524943004545A4
:100B200050524F4D0042494E4152595F46494C4543
:100B30005F5452414E534645520053455249414C31
:100B40005F584F4E5F584F4646004649524D5741F9
:100B500052455F4E414D453A4D61726C696E20328F
:100B60002E305F44573320544D33442035534D4489
:100B7000424220534F555243455F434F44455F55D2
:100B8000524C3A68747470733A2F2F6769746875A1
:100B9000622E636F6D2F496E73616E697479417552
:100BA000746F6D6174696F6E2F4D61726C696E2F19
:100BB000747265652F437265616C6974795F4D610C
:100BC000726C696E322E302E782050524F544F4343
:100BD0004F4C5F56455253494F4E3A312E30204DBF
:100BE000414348494E455F545950453A544D33446A
:100BF000204D61782045585452554445525F434F2B
:100C0000554E543A3120555549443A63656465322E
:100C10006132662D343161322D343734382D3962EA
:100C200031322D6335356336326633363766660AC0
:100C3000002F2F20003F4A206F7574206F662072AE
:100C4000616E67652028302E303120746F20302E81
:100C500033290A0020466C6F773A200050726F7477
:100C600065637465642050696E0A00206F75742096
:100C70006F662072616E67650A00536572766F2039
:100C8000003A200020536572766F200050726F6228
:100C900065205A204F66667365743A2000496E7667
:100CA000616C69642065787472756465720A0020ED
:100CB000643A0020693A0020703A0020643A00202B
:100CC000693A0020703A0064697300656E00432938
:100CD0000A0061626C656420286D696E2074656D20
:100CE000702000436F6C642065787472756465735E
:100CF0002061726520004F4646004F4E0046696CE9
:100D0000616D656E742072756E6F757420646973A1
:100D100074616E636520286D6D293A200046696C08
:100D2000616D656E742072756E6F757420004D650F
:100D3000736820706F696E742063616E6E6F7420CB
:100D40006265207265736F6C7665640A004D34329B
:100D50003120696E636F72726563742070617261B5
:100D60006D657465722075736167650A004F66660C
:100D700073657473204170706C69656400457272AC
:100D80003A20546F6F206661722100546F6F2066A5
:100D900061722066726F6D207265666572656E6342
:100DA0006520706F696E740A00454550524F4D20A2
:100DB0004F4B0A004572726F722077726974696EC8
:100DC0006720746F20454550524F4D210A00363739
:100DD00026033C3D380E2E303E131A1C1808440AD8
:100DE000FF430809070001627573793A2070617545
:100DF00073656420666F7220696E7075740A006294
:100E00007573793A2070617573656420666F72201E
:100E1000757365720A00627573793A2070726F6338
:100E2000657373696E670A007061757365004D368E
:100E30003030200A204D313137200A002066696C9D
:100E4000616D656E745F72756E6F75742000666992
:100E50006C616D656E745F72756E6F757420540091
:100E600046696C616D656E7452756E6F7574205451
:100E70000053544F505045442E20005072696E74F8
:100E800065722073746F707065642064756520747A
:100E90006F206572726F72732E20466978207468B5
:100EA00065206572726F7220616E642075736520B3
:100EB0004D39393920746F20726573746172742EE4
:100EC000202854656D706572617475726520697350
:100ED0002072657365742E205365742069742061D7
:100EE000667465722072657374617274696E6729C5
:100EF0000A004E6F20436865636B73756D207769D8
:100F00007468206C696E65206E756D6265722C2048
:100F10004C617374204C696E653A20004E6F20431B
:100F20006865636B73756D2077697468206C696E92
:100F300065206E756D6265722C204C617374204C57
:100F4000696E653A2000636865636B73756D206D2B
:100F500069736D617463682C204C617374204C69F3
:100F60006E653A20004C696E65204E756D62657243
:100F7000206973206E6F74204C617374204C696E0D
:100F800065204E756D6265722B312C204C61737437
:100F9000204C696E653A20004D313130007761692F
:100FA000740A004D313137004D3331005344207203
:100FB000656164206572726F720A00446F6E65200D
:100FC0007072696E74696E672066696C650A004BA1
:100FD000494C4C2063617573656420627920746F9D
:100FE0006F206D75636820696E6163746976652032
:100FF00074696D65202D2063757272656E7420634F
:101000006F6D6D616E643A20002020506C616E6ED1
:10101000657242756666657242797465733A20003E
:101020002046726565204D656D6F72793A200043E8
:101030006F6D70696C65643A2053657020203820AC
:10104000323031390A00207C20417574686F723A61
:101050002054696E794D616368696E657333440A23
:1010600000323031392D30372D333000204C617350
:101070007420557064617465643A2000322E305FCC
:101080004457330A004D61726C696E0020536F66DD
:1010900074776172652052657365740A0020576128
:1010A000746368646F672052657365740A00204238
:1010B000726F776E206F75742052657365740A00C5
:1010C0002045787465726E616C2052657365740A90
:1010D00000506F77657255700A0073746172740AFC
:1010E000006175746F25632E67006572726F7220E0
:1010F00077726974696E6720746F2066696C650A1F
:1011000000446F6E6520736176696E672066696C56
:10111000652E0A004D323900205A3A0020593A0013
:1011200020583A00656E6473746F70732068697438
:101130003A200047323858590043616E6E6F742070
:101140006F70656E2073756264697220005344206D
:1011500063617264206F6B0A006F70656E526F6F0F
:1011600074206661696C65640A00766F6C756D65E4
:101170002E696E6974206661696C65640A00534467
:1011800020696E6974206661696C0A004D32340012
:101190004D32332025730057726974696E6720746D
:1011A0006F2066696C653A20002E0A006F70656ECC
:1011B000206661696C65642C2046696C653A200084
:1011C0002E0A006F70656E206661696C65642C2064
:1011D00046696C653A200046696C652073656C65EC
:1011E000637465640A002053697A653A2000466991
:1011F0006C65206F70656E65643A20006672657379
:101200006800646F696E67002066696C653A20004B
:101210004E6F772000454E4420535542524F55544F
:10122000494E450A002220706F73002220706172BF
:10123000656E743A2200535542524F5554494E45FB
:101240002043414C4C207461726765743A220074EB
:101250007279696E6720746F2063616C6C2073759E
:10126000622D67636F64652066696C6573207769BA
:10127000746820746F6F206D616E79206C6576657F
:101280006C732E204D4158206C6576656C20697317
:101290003A310A005344207072696E74696E672097
:1012A0006279746520004E6F742053442070726917
:1012B0006E74696E670A00496E76616C69642065B8
:1012C000787472756465720A007C3C3E5E2B3D3F0B
:1012D0002F5B5D3B2C2A225C00486F6D65202573D7
:1012E00025732573204669727374002046697273F2
:1012F000740A00486F6D652000220A00556E6B6EFF
:101300006F776E20636F6D6D616E643A20220020EE
:10131000746F6F206C6F6E67206578747275736977
:101320006F6E2070726576656E7465640A00206366
:101330006F6C6420657874727573696F6E2070725B
:101340006576656E7465640A004D32383020503021
:10135000205339300050726F62696E6720506F6998
:101360006E742025692F2569002E0A002F00507207
:101370006F62696E67206D65736820706F696E7447
:101380002000202844525952554E29004732392016
:101390004175746F20426564204C6576656C696E9A
:1013A00067003F20284C2C522C462C4229206F7578
:1013B00074206F6620626F756E64732E0A003F287A
:1013C00056296572626F7365206C6576656C20695D
:1013D0007320696D706C61757369626C652028306B
:1013E0002D34292E0A00426164205A2076616C75E2
:1013F000650A004E6F2062696C696E6561722067D4
:101400007269640A0046696E6973686564210A003E
:10141000206F662000205A00205900476F696E67D0
:1014200020746F3A20580043570A00206469723ACA
:101430000020616E676C653A0053746172742072AB
:1014400061646975733A00506F736974696F6E698E
:101450006E67207468652070726F62652E2E2E0A8A
:10146000003F4E756D626572206F66206C65677314
:1014700020696E206D6F76656D656E74206E6F7479
:1014800020706C61757369626C652028302D313570
:10149000292E0A003F2028582C5929206F757420C6
:1014A0006F6620626F756E64732E0A003F53616D24
:1014B000706C652073697A65206E6F7420706C6142
:1014C000757369626C652028342D3530292E0A0029
:1014D0004D3438205A2D50726F6265205265706508
:1014E00061746162696C69747920546573740A006F
:1014F0003F2856296572626F7365206C6576656C4E
:1015000020697320696D706C61757369626C652008
:1015100028302D34292E0A0053544F502063616C1B
:101520006C65642062656361757365206F66204237
:101530004C546F756368206572726F72202D207233
:101540006573746172742077697468204D39393914
:101550000A0053544F502063616C6C6564206265CF
:101560006361757365206F6620424C546F756368C4
:10157000206572726F72202D2072657374617274AF
:101580002077697468204D3939390A002F2F61633B
:1015900074696F6E3A00627574746F6E00656E6484
:1015A0000070726F6D70745F0073686F77004D38F4
:1015B000373620526573706F6E64696E67205052C3
:1015C0004F4D50545F00554E4B4E4F574E20535485
:1015D0004154450047434F44455F494E464F004CF8
:1015E00043445F50415553455F524553554D450067
:1015F00046494C414D454E545F52554E4F55545FF0
:10160000434F4E54494E55450046494C414D454E79
:10161000545F52554E4F5554004D323400436F6E57
:1016200074696E75650044697361626C6552756EAC
:101630006F7574005075726765204D6F726500504C
:1016400061757365640070617573656400486F74DB
:10165000656E6420746F6F20636F6C640A00506164
:1016600075736500507265737320627574746F6E64
:1016700020286F72204D3130382920746F20726518
:1016800073756D650A00496E736572742066696CC6
:10169000616D656E7420616E642070726573732075
:1016A000627574746F6E20286F72204D3130382946
:1016B0000A00436F6E74696E7565005265686561F6
:1016C0007420446F6E6500526568656174696E6769
:1016D0002E2E2E00526568656174696E670048653C
:1016E0006174657254696D656F75740052656865E3
:1016F00061740048656174657254696D656F7574D5
:1017000000507265737320627574746F6E20286F59
:1017100072204D3130382920746F20686561742043
:101720006E6F7A7A6C650A004E6F7A7A6C6520501B
:1017300061726B656400436F6E74696E7565004E0F
:101740006F7A7A6C65205061726B656400486F74C3
:10175000656E6420746F6F20636F6C640A0072653D
:1017600073756D656400626567696E00436F6E74C2
:10177000696E75650044697361626C6552756E6F60
:1017800075740050757267654D6F726500506175B4
:10179000736564004C6F61642046696C616D656EB1
:1017A0007400436F6E74696E7565004C6F616420E0
:1017B00046696C616D656E74205400496E73657284
:1017C000742066696C616D656E7420616E64207052
:1017D0007265737320627574746F6E20286F722047
:1017E0004D313038290A00526573756D650024F457
:1017F000D43050C38E20C2A24017828B7011127A4F
:10180000910D816CD90AA861E108C758660761513A
:1018100043061E4B5D05C145A7041A411104093D4D
:101820009803713931034036DB0265339102D430BD
:101830005402802E1D02632CEE01752AC501B028CA
:10184000A001102781018F2564012B244B01E02288
:101850003401AC211F018D200D01801FFC00841E6E
:10186000ED00971DDF00B81CD200E61BC600201B50
:10187000BC00641AB200B219A8000A19A0006A18C4
:101880009900D117910040178B00B51684003116CE
:101890007E00B31579003A157300C7146F00581411
:1018A0006A00EE1366008813630025135E00C712FA
:1018B0005B006C12570015125400C11151007011D9
:1018C0004F0021114B00D61049008D1047004610E3
:1018D000440002104200C00F4000800F3E00420F43
:1018E0003C00060F3B00CB0E3800930E37005C0E19
:1018F0003500270E3400F30D3200C10D3100900D7C
:101900003000600D2E00320D2D00050D2C00D90C7D
:101910002B00AE0C2900850C29005C0C2700350C2F
:1019200027000E0C2600E80B2400C40B2400A00B9B
:1019300023007D0B23005A0B2100390B2100180BCB
:101940002000F80A1F00D90A1E00BB0A1E009D0ACB
:101950001D00800A1D00630A1C00470A1B002C0A98
:101960001B00110A1A00F7091A00DD091900C40941
:101970001900AB091900920917007B0918006309C7
:1019800017004C09160036091600200916000A092E
:101990001500F5081500E0081400CC081400B8087C
:1019A0001400A4081400900813007D0812006B08AE
:1019B00013005808120046081200340811002308CA
:1019C00011001208110001081100F0071000E007D3
:1019D0001000D0071000C0071000B0070F00A107CB
:1019E000100091070E0083070F0074070F006507B2
:1019F0000E0057070E0049070E003B070D002E078B
:101A00000E0020070D0013070D0006070D00F90654
:101A10000C00ED060D00E0060C00D4060C00C80614
:101A20000C00BC060C00B0060C00A4060B009906C6
:101A30000C008D060B0082060B0077060B006C066F
:101A40000B0061060A0057060B004C060A0042060E
:101A50000A0038060A002E060A0024060A001A06A2
:101A60000A001006090007060A00FD050900F40532
:101A70000900EB050900E2050900D9050900D005B8
:101A80000900C7050900BE050900B5050800AD0538
:101A90000800A50509009C050800940508008C05B0
:101AA0000800840508007C050800740508006C0522
:101AB0000700650508005D050700560508004E058E
:101AC00007004705070040050800380507003105F5
:101AD00007002A050700230507001C050600160558
:101AE00007000F0507000805060002050700FB04B4
:101AF0000600F5040700EE040600E8040600E20410
:101B00000700DB040600D5040600CF040600C90464
:101B10000600C3040600BD040600B7040600B104B5
:101B20000500AC040600A6040600A00405009B0402
:101B3000060095040500900406008A04050085044B
:101B40000500800406007A04050075040500700491
:101B500005006B04050066040500610405005C04D3
:101B6000050057040500520405004D040500480413
:101B70000500430405003E0404003A040500350452
:101B80000500300404002C0405002704040023048D
:101B900005001E0404001A040400160405001104C4
:101BA00004000D04040009040500040404000004FA
:101BB0000400FC030400F8030400F4030400F00331
:101BC0000400EC030400E8030400E4030400E00361
:101BD0000400DC030400D8030400D4030400D00391
:101BE0000400CC030400C8030300C503030024F46D
:101BF00004D9201BC40C5C0E9804C4095F0265075D
:101C00007101F405F900FB04B30048048700C10327
:101C100069005803550003034500BE023A008402E0
:101C2000310053022A002902250004022000E401A9
:101C30001C00C8011900AF011700980114008401AD
:101C40001300710110006101100051010E004301E9
:101C50000D0036010B002B010B0020010B001501BC
:101C600009000C01090003010800FB000800F30053
:101C70000800EB000700E4000600DE000600D800C4
:101C80000600D2000600CC000500C7000500C20017
:101C90000500BD000400B9000400B5000400B10057
:101CA0000400AD000400A9000400A5000300A20088
:101CB00003009F0004009B000300980003009500B0
:101CC000020093000300900003008D0002008B00CF
:101CD00003008800020086000200840003008100E7
:101CE00002007F0002007D0002007B0002007900FC
:101CF000020077000100760002007400020072000A
:101D00000100710002006F0002006D0001006C0014
:101D100002006A000100690002006700010066001D
:101D20000100650001006400020062000100610022
:101D30000100600001005F0002005D0001005C0026
:101D400001005B0001005A00010059000100580029
:101D50000100570001005600010055000100540029
:101D60000100530000005300010052000100510027
:101D70000100500001004F0001004E0000004E0025
:101D800001004D0001004C0001004B0000004B0021
:101D900001004A000100490001004800000048001D
:101DA0000100470001004600000046000100450018
:101DB0000000450001004400010043000000430012
:101DC000010042000000420001004100000041000B
:101DD0000100400001003F0000003F0001003E0004
:101DE00000003E0001003D0000003D0001003C00FD
:101DF00000003C0000003C0001003B0000003B00F4
:101E000001003A0000003A000100390000003900EA
:101E100001003800000038000000380001003700E1
:101E200000003700010036000000360000003600D8
:101E300001003500000035000000350001003400CD
:101E400000003400000034000100330000003300C3
:101E500000003300010032000000320000003200B8
:101E600001003100000031000000310001003000AD
:101E7000000030000000300001002F0000002F00A3
:101E800000002F0000002F0001002E0000002E0097
:101E900000002E0001002D0000002D0000002D008C
:101EA00000002D0001002C0000002C0000002C0080
:101EB00000002C0001002B0000002B0000002B0074
:101EC00000002B0001002A0000002A0000002A0068
:101ED00000002A000100290000002900000029005C
:101EE000000029000000290001002800000028004F
:101EF0000000280000002800000028000100270042
:101F00000000270000002700000027000000270035
:101F10000100260000002600000026000000260028
:101F2000000026000100250000002500000025001B
:101F3000000025000000250000002500010024000D
:101F40000000240000002400000024000000240001
:101F500001002300000023000000230000002300F4
:101F600000002300000023000000230001002200E5
:101F700000002200000022000000220000002200D9
:101F800000002200010021000000210000002100CB
:101F900000002100000021000000210000002100BD
:101FA00001002000000020000000200000002000B0
:101FB00000002000000020000000200000002000A1
:101FC00001001F0000001F0000001F0000001F0094
:101FD00000001F0000001F0000001F0001001E0085
:101FE00000001E0000001E0000001E00000004375C
:101FF00000001E290000511B0000581000001009AD
:102000000000CC040000780200004101000062657D
:1020100064002C2073797374656D2073746F707015
:10202000656421204865617465725F49443A200007
:102030004265642048656174696E67204661696C19
:1020400065640048656174696E67206661696C65E6
:10205000640042454420544845524D414C2052555D
:102060004E4157415900546865726D616C2052753C
:102070006E617761790045312048656174696E67EA
:10208000204661696C65640048656174696E67200B
:102090006661696C656400453120544845524D4184
:1020A0004C2052554E4157415900546865726D613C
:1020B0006C2052756E617761790057616974696E41
:1020C0006720666F72206865617475702E0A004C17
:1020D000656176696E6720473236003F53706563ED
:1020E000696669656420582C5920636F6F72646952
:1020F0006E617465206F7574206F6620626F756EF7
:1021000064732E0A003F2852296570656174207639
:10211000616C7565206E6F7420706C617573696297
:102120006C653B206D757374206265206174206C52
:102130006561737420312E0A003F2852296570654D
:102140006174206D757374206265207370656369B6
:1021500066696564207768656E206E6F742075739C
:10216000696E6720616E204C43442E0A003F537015
:1021700065636966696564206E6F7A7A6C65207440
:10218000656D7065726174757265206E6F74207014
:102190006C61757369626C652E0A003F53706563EC
:1021A00069666965642066696C616D656E7420732B
:1021B000697A65206E6F7420706C61757369626CEA
:1021C000652E0A003F537065636966696564207017
:1021D00072696D65206C656E677468206E6F74201F
:1021E000706C61757369626C652E0A003F5072698C
:1021F0006D65206C656E677468206D757374206200
:102200006520737065636966696564207768656ECB
:10221000206E6F74207573696E6720616E204C4369
:10222000442E0A003F537065636966696564206ED9
:102230006F7A7A6C652073697A65206E6F7420708E
:102240006C61757369626C652E0A003F5265747229
:10225000616374696F6E204D756C7469706C69652B
:1022600072206D7573742062652073706563696692
:102270006965642E0A003F53706563696669656429
:102280002052657472616374696F6E204D756C7451
:1022900069706C696572206E6F7420706C61757303
:1022A00069626C652E0A003F5370656369666965F3
:1022B00064206C6179657220686569676874206E56
:1022C0006F7420706C61757369626C652E0A0043CF
:1022D000292E0A003F537065636966696564206250
:1022E00065642074656D7065726174757265206EC9
:1022F0006F7420706C61757369626C65202834306E
:102300002D00473236207374617274696E672E2E09
:102310002E0A004F46460A004661646520486569FA
:102320006768742000426564204C6576656C696E50
:102330006720004661696C656420746F20656E617A
:10234000626C6520426564204C6576656C696E67D9
:102350000A00496E76616C6964206D6573682E0AA7
:10236000004469666665723A200046726F6D537468
:10237000703A00537465707065723A00556E4C6522
:1023800076656C3A004C6576656C65643A0052611E
:10239000773A20202020000A4C6F676963616C3A0D
:1023A000004361703A004D302F3120427265616BFD
:1023B0002043616C6C656400436F6E74696E756573
:1023C000004D302F3120427265616B2043616C6C8F
:1023D00065640050726F6265205A204F66667365AF
:1023E000743A200050726F62652059204F66667300
:1023F00065743A200050726F62652058204F6666FF
:102400007365743A20003F59206F7574206F662001
:1024100072616E67652028302D34353020746F204E
:10242000343530290A003F58206F7574206F6620BC
:1024300072616E67652028302D34373520746F2027
:10244000343735290A003F5A206F7574206F662093
:1024500072616E676520282D323020746F20323013
:10246000290A00220A00656E7175657565696E67D7
:102470002022002042002050006F6B006F70656EBC
:1024800000545249474745524544003A2000666986
:102490006C616D656E74007A5F6D696E00795F6D59
:1024A000696E00785F6D696E005265706F72746955
:1024B0006E6720656E6473746F70207374617475D9
:1024C000730A00205A3A0020593A0020436F756E73
:1024D0007420583A0020453A00205A3A0020593AD0
:1024E00000583A0020746F6F206C6F6E672065781B
:1024F00074727573696F6E2070726576656E74653F
:10250000640A0020636F6C64206578747275736967
:102510006F6E2070726576656E7465640A000000E7
:102520000000000000000000000000004842000021
:102530004842000080405761726E696E673A2048D9
:102540006F6D696E672042756D702044697669739E
:102550006F72203C20310A000202040000A04000FB
:1025600000A040000000400080ED430000E1430077
:1025700000EB43FFFFFF5A5F53544F505F50494EEB
:10258000005A5F535445505F50494E005A5F4D49C1
:102590004E5F50494E005A5F454E41424C455F5098
:1025A000494E005A5F4449525F50494E005A5F43BA
:1025B000535F50494E00595F53544F505F50494E3E
:1025C00000595F535445505F50494E00595F4D4983
:1025D0004E5F50494E00595F454E41424C455F5059
:1025E000494E00595F4449525F50494E00595F437C
:1025F000535F50494E00585F53544F505F50494EFF
:1026000000585F535445505F50494E00585F4D4944
:102610004E5F50494E00585F454E41424C455F5019
:10262000494E00585F4449525F50494E00585F433D
:10263000535F50494E0053535F50494E005345522B
:10264000564F335F50494E00534552564F325F50FC
:10265000494E00534552564F315F50494E00534545
:1026600052564F305F50494E005344535300534429
:102670005F4445544543545F50494E0053434B5FBC
:1026800050494E0052414D50535F44395F50494EBE
:102690000052414D50535F44385F50494E00524103
:1026A0004D50535F4431305F50494E004D4F5349B8
:1026B0005F50494E004D4F534645545F445F50496B
:1026C0004E004D49534F5F50494E004D41583636EC
:1026D00037355F53535F50494E004C45445F504976
:1026E0004E004845415445525F4245445F50494E73
:1026F000004845415445525F305F50494E004649BD
:102700004C5F52554E4F55545F50494E0046414E16
:10271000315F50494E0046414E5F50494E004531B1
:102720005F535445505F50494E0045315F454E411F
:10273000424C455F50494E0045315F4449525F501D
:10274000494E0045315F43535F50494E0045305F6D
:10275000535445505F50494E0045305F454E41420D
:102760004C455F50494E0045305F4449525F5049E7
:102770004E0045305F43535F50494E00455F4D5515
:1027800058325F50494E00455F4D5558315F5049B2
:102790004E00455F4D5558305F50494E00415652EE
:1027A0005F53535F50494E004156525F53434B5F56
:1027B00050494E004156525F4D4F53495F50494E6C
:1027C000004156525F4D49534F5F50494E005445AA
:1027D0004D505F4245445F50494E0054454D505F57
:1027E000315F50494E0054454D505F305F50494E67
:1027F0000046494C57494454485F50494E0054588C
:102800004400525844002054002052004163636544
:102810006C65726174696F6E3A20500050574D3A82
:1028200020202534640050574D3A20202534640080
:1028300050574D3A20202534640050574D3A2020FF
:102840002534640050574D3A2020253464005057F9
:102850004D3A20202534640050574D3A202025342D
:10286000640050574D3A20202534640050574D3AAB
:1028700020202534640050574D3A20202534640030
:1028800050574D3A20202534640050574D3A2020AF
:102890002534640050574D3A2020253464005057A9
:1028A0004D3A20202534640050574D3A20202534DD
:1028B000640050574D3A202025346400433A2000EC
:1028C000423A2000413A200020202020434F4D0072
:1028D0002020206E6F6E2D7374616E6461726420AF
:1028E00050574D206D6F646500202020636F6D7020
:1028F00061726520696E7465727275707420656EA0
:1029000061626C6564002020206F766572666C6F72
:102910007720696E7465727275707420656E61627D
:102920006C6564003A20002020202054494D534B10
:1029300000423A2000202020205443435200413AD4
:1029400020002020202054434352002020202043F8
:10295000533A20002020202057474D3A200050575E
:102960004D3A20202534640050574D3A202025341C
:10297000640047004800000088008A008C00B30013
:10298000B400000098009A009C00A800AA00AC00C7
:1029900028012A012C012020202054494D455200B5
:1029A000440045006E00800081006F00B000B1005F
:1029B0007000900091007100A000A1007200200141
:1029C0002101730020697320616C736F2074696545
:1029D0006420746F20746869732070696E005449B4
:1029E0004D45523143000A202E0020200020205067
:1029F0006F72743A200020202000202020416E6158
:102A00006C6F6720696E203D2025356C64003C7535
:102A10006E757365642F756E6B6E6F776E3E0020FA
:102A200028412532642920200025336420002573A5
:102A300050494E3A20004F7574707574203D200047
:102A4000496E70757420203D2000416E616C6F6787
:102A500020696E203D2025356C640070726F7465AE
:102A600063746564200020284125326429202000F9
:102A70002533642000257350494E3A200002280077
:102A800001FE270101F1273B00E6274300DB274534
:102A900000CE274400C1273201B4273301A82734D0
:102AA000019D2735019227280187272A017C272CA1
:102AB0000172272A0167271C01592718014D271A7F
:102AC0000143272C01382722012A271E011E272413
:102AD00001162709010D270701FE260201F1260A2A
:102AE00001E2260801DA260D01CB264201C2263278
:102AF00001B5260701AC2633019E260A019126085E
:102B000001842609017C2634016E263101692635AF
:102B1000015E260B0153260601482605013D2604C9
:102B200001362635012D26350123263701162626A6
:102B3000010C26030101263601F6250301ED25319E
:102B400001E3253D01D6253801CC250E01C1253CE8
:102B500001B6250E01AD252801A325300196253E9D
:102B6000018C25130181252E0176251301526573F1
:102B7000656E643A200043616E6E6F74206F7065FD
:102B80006E2073756264697220002569730025697F
:102B90006D20256973002569682025696D202569E8
:102BA0007300256964202569682025696D202569E1
:102BB00073002569792025696420256968202569C5
:102BC0006D202569730023646566696E6520444540
:102BD0004641554C545F0000626564004B64200020
:102BE0004B6920004B702000504944204175746FA0
:102BF00074756E652066696E69736865642120501E
:102C0000757420746865206C617374204B702C207F
:102C10004B6920616E64204B6420636F6E73746136
:102C20006E74732066726F6D2062656C6F772069B9
:102C30006E746F20436F6E66696775726174696F39
:102C40006E2E680A00504944204175746F74756E89
:102C500065206661696C6564212074696D656F75B6
:102C6000740A00453120544845524D414C2052557C
:102C70004E415741590042454420544845524D4128
:102C80004C2052554E4157415900546865726D6150
:102C90006C2052756E61776179004531204865611D
:102CA00074696E67204661696C65640042656420E2
:102CB00048656174696E67204661696C65640048A7
:102CC000656174696E67206661696C65640050496E
:102CD00044204175746F74756E65206661696C651A
:102CE00064212054656D706572617475726520741D
:102CF0006F6F20686967680A00204B643A200020E3
:102D00004B693A2000204B703A20000A20436C6146
:102D10007373696320504944200A00204B643A20B1
:102D200000204B693A2000204B703A20000A204EC8
:102D30006F206F76657273686F6F740A0020547528
:102D40003A2000204B753A2000206D61783A20002F
:102D5000206D696E3A200020643A2000206269618B
:102D6000733A2000504944204175746F74756E6544
:102D70002073746172740A00504944204175746F65
:102D800074756E65206661696C6564212054656D9B
:102D9000706572617475726520746F6F2068696701
:102DA000680A00504944204175746F74756E65203F
:102DB0006661696C65642120426164206578747283
:102DC00075646572206E756D6265720A0070012C03
:102DD0000190012701B0012201C0011D01F001187D
:102DE000011002130130020E016002090190020479
:102DF00001C002FF000003FA004003F5008003F069
:102E000000D003EB002004E6007004E100E004DCE5
:102E1000004005D700C005D2004006CD00D006C84E
:102E2000008007C3003008BE00F008B900C009B434
:102E300000B00AAF00B00BAA00D00CA500000EA095
:102E400000500F9B00C01096005012910000148C8F
:102E500000C0158700B0178200B0197D00D01B7824
:102E600000001E730040206E0090226900F0246470
:102E70000040275F0090295A00E02B5500102E508B
:102E80000020304B0010324600E033410090353CCA
:102E9000001037370070383200A0392D00B03A28C2
:102EA00000A03B2300603C1E00103D1900903D1423
:102EB00000103E0F00703E0A00C03E0500003F00BB
:102EC00000403FFBFF803FF6FFC03FF1FF202D2079
:102ED000496E76616C696420657874727564657298
:102EE000206E756D62657220210A001000C9021003
:102EF000012C014001220170011801B0010E01F006
:102F00000104015002FA00B002F0003003E600D0E4
:102F100003DC009004D2007005C800A006BE0000CB
:102F200008B400B009AA00D00BA000600E960060A3
:102F3000118C000015820020197800C01D6E00A0C1
:102F4000226400B0275A00902C500000314600E067
:102F5000343C0010383200903A2800603C1E00A03B
:102F60003D1400803E0A00203F00004531205448B7
:102F700045524D414C2052554E4157415900424512
:102F80004420544845524D414C2052554E415741E2
:102F90005900546865726D616C2052756E6177617D
:102FA00079004531204572723A204D415854454DC3
:102FB00050004572723A204D415854454D502042C0
:102FC0004544004D415854454D502074726967671F
:102FD00065726564004531204572723A204D494E54
:102FE00054454D50004572723A204D494E54454D5E
:102FF0005020424544004D494E54454D5020747276
:1030000069676765726564000A0A0020205A5F4D8F
:10301000494E3A002020595F4D494E3A0020205831
:103020005F4D494E3A004D383420582059205A20DF
:103030004500202F002042403A0020403A0020570F
:103040003A0020573A00446F6E652E0A0066616CA4
:103050007365004641494C3A204E6F20747269678F
:103060006765722064657465637465640A0046412F
:10307000494C3A204E6F69736520646574656374CA
:103080006564202D20706C656173652072652D72FA
:10309000756E20746573740A0020646574656374CA
:1030A00065642E0A003D20424C546F7563682070A1
:1030B00072652056332E3120286F7220636F6D7039
:1030C000617469626C6529003D205A2053657276EF
:1030D0006F2050726F6265003D20424C546F7563E3
:1030E000682056332E310020282B2F2D20346D736D
:1030F000293A20003A2033306D73206F72206D6FB3
:1031000072650A002E2050756C73652077696474AF
:1031100068002A2A20506C656173652074726967A3
:103120006765722070726F62652077697468696E76
:1031300020333020736563202A2A0A004641494C17
:103140003A20424C544F55434820656E61626C658D
:1031500064202D2053657420757020746869732075
:1031600064657669636520617320612053657276BA
:103170006F2050726F6265207769746820494E56DF
:10318000455254494E472073657420746F2027744C
:10319000727565272E0A0020204445504C4F594532
:1031A000442073746174653A204C4F5720286C6F2B
:1031B0006769632030290020204445504C4F594511
:1031C000442073746174653A204849474820286C4C
:1031D0006F676963203129003D204D656368616E2A
:1031E0006963616C205377697463682064657465F2
:1031F000637465640A005741524E494E473A20496C
:103200004E56455254494E472073657474696E6733
:103210002070726F6261626C79206261636B7761AA
:103220007264732E0A002E204465706C6F7920261C
:103230002073746F7720342074696D65730A003DC4
:1032400020424C546F75636820436C6173736963EB
:1032500020312E322C20312E332C20536D6172748C
:1032600020312E302C20322E302C20322E322C20A9
:10327000332E302C20332E312064657465637465E1
:10328000642E0A002E20436865636B20666F7220EF
:10329000424C544F5543480A002E205A5F4D494E28
:1032A0005F454E4453544F505F494E564552544922
:1032B0004E473A20002E2050726F6265205A5F4DB3
:1032C000494E5F50494E3A20002C2073746F77208E
:1032D000616E676C653A202020002C206465706C5C
:1032E0006F7920616E676C653A2000536572766F66
:1032F0002070726F626520746573740A2E20757376
:10330000696E6720696E6465783A2020004D343319
:1033100020576169742043616C6C656400436F6E73
:1033200074696E7565004D343320576169742043AC
:10333000616C6C6564005761746368696E672070C6
:10334000696E730A0064697300656E0061626C6582
:10335000640A00656E6473746F70206D6F6E6974BB
:103360006F722000204500205A00205900204D395E
:1033700032205800205A00205900580020204D616A
:10338000783A2000205A00205900580020204D692A
:103390006E3A2000536F667420656E6473746F70AC
:1033A000733A20004732380020496E76616C6964B8
:1033B0002065787472756465722000544D33442022
:1033C0004D61782052656164792E005072696E7487
:1033D000696E672E2E2E005072696E7420506175D2
:1033E0007365640063616E63656C005072696E742E
:1033F0002041626F727465640055492041626F72AA
:103400007400726573756D65004D3234000080ED97
:10341000430000E1430000EB430000000000000017
:103420000000000000290A002062797465733B20C7
:10343000637263200053657474696E6773205374FC
:103440006F726564202800454550524F4D206461DD
:10345000746173697A65206572726F722E0A002931
:103460000A002062797465733B2063726320002038
:1034700073746F7265642073657474696E6773200A
:10348000726574726965766564202800202863611E
:103490006C63756C6174656429210A0020213D20EC
:1034A00000454550524F4D20435243206D69736D86
:1034B00061746368202D202873746F7265642920FD
:1034C000002053697A653A2000496E6465783A2095
:1034D00000204D61726C696E3D563730290A0045F7
:1034E0004550524F4D2076657273696F6E206D693D
:1034F000736D617463682028454550524F4D3D00FF
:103500000A20696E6974207A70726F62655F7A6FE3
:103510006666736574203D2000454550524F4D202E
:10352000496E697469616C697A65640A0048617200
:1035300064636F6465642044656661756C742053D0
:10354000657474696E6773204C6F616465640A000A
:10355000E8030000BC020000640000004B00000013
:103560000000FA430000C84300007041000096428A
:103570000000A0420000A0420000C84300000C432D
:103580003A0A0020204D363033200020440020200D
:103590004D34313220530046696C616D656E742084
:1035A00072756E6F75742073656E736F723A0A0070
:1035B0002055004C0046696C616D656E74206C6F1F
:1035C00061642F756E6C6F6164206C656E677468E2
:1035D000733A0A0020204D383531205A0020204D02
:1035E00038353120590020204D3835312058005AC7
:1035F0002D50726F6265204F6666736574002044BB
:103600000020490020204D33303420500020440059
:1036100020490020204D33303120500050494420B3
:1036200073657474696E67733A0A00204A0020203B
:103630004732392057204900205A0020204D34328B
:10364000302053004175746F20426564204C6576CC
:10365000656C696E673A0A00205A002059002020E4
:103660004D323036205800486F6D65206F666673A6
:1036700065743A0A00204A0020540020530020209C
:103680004D323035204200204A3C6A756E635F64DB
:1036900065763E00416476616E6365643A20423C23
:1036A0006D696E5F7365676D656E745F74696D6576
:1036B0005F75733E20533C6D696E5F66656564722D
:1036C0006174653E20543C6D696E5F74726176650D
:1036D0006C5F66656564726174653E00205400200D
:1036E000520020204D323034205000416363656C1D
:1036F00065726174696F6E2028756E6974732F73BB
:1037000032293A20503C7072696E745F6163636560
:103710006C3E20523C726574726163745F616363D6
:10372000656C3E20543C74726176656C5F616363C6
:10373000656C3E0A00204500205A002059002020D8
:103740004D3230312058004D6178696D756D2041E2
:103750006363656C65726174696F6E2028756E694C
:1037600074732F7332293A0A00204500205A002032
:10377000590020204D3230332058004D6178696D5A
:10378000756D206665656472617465732028756E59
:103790006974732F73293A0A00537465707320702B
:1037A000657220756E69743A0A0020204D323030FF
:1037B0002044300A0020204D323030204400204484
:1037C000697361626C65640A0046696C616D656E5F
:1037D000742073657474696E67733A0020286D6D88
:1037E00029002020473231202020203B20556E69BF
:1037F000747320696E206D6D00486F6D696E67206F
:103800004661696C65640000002100240027002ADD
:10381000002D003000330001010000040107010AFF
:103820000100002200250028002B002E003100346A
:103830000002010000050108010B01000020002327
:1038400000260029002C002F003200000100000398
:103850000106010901050505050705080808080214
:103860000202020A0A080804040404010101010119
:103870000101010303030303030303040707070C08
:103880000C0C0C0C0C0C0C020202020606060606BE
:103890000606060B0B0B0B0B0B0B0B01021020206B
:1038A0000808102040102040800201020108040294
:1038B000010102040810204080804020100804020A
:1038C0000180040201804020100804020108040263
:1038D0000101020408102040800102040810204069
:1038E0008000000A0B02090C0D0E080703040100FA
:1038F00000000000000000000000000000000000C8
:103900000000000000000000000000000012111084
:1039100000000000000000000000000000000000A7
:103920000000000000000050726F62696E67204660
:1039300061696C65640A0050726F62696E67204647
:1039400061696C6564002E0A006F70656E206661A7
:10395000696C65642C2046696C653A2000706F774D
:1039600065726F6666004B494C4C45442E200050F2
:1039700072696E7465722068616C7465642E206B68
:10398000696C6C28292063616C6C6564210A0053A2
:10399000544F505045442E20005072696E74657229
:1039A0002073746F707065642064756520746F2077
:1039B0006572726F72732E20466978207468652074
:1039C0006572726F7220616E6420757365204D3967
:1039D000393920746F20726573746172742E2028D7
:1039E00054656D70657261747572652069732072BB
:1039F000657365742E205365742069742061667444
:103A000065722072657374617274696E67290A0049
:103A10006563686F3A004572726F723A0042696C72
:103A2000696E656172204C6576656C696E672047CA
:103A30007269643A0A009101B70111241FBECFEFE9
:103A4000D1E2DEBFCDBF00E00CBF18E0A0E0B2E0E5
:103A5000EAE8F1E502E00BBF02C007900D92AA3937
:103A6000B107D9F72DE1AAE9B8E001C01D92AE3A3D
:103A7000B207E1F71DE1CCE1DDE100E006C02197EE
:103A80000109802FFE010F94EE24CB31D10780E095
:103A90000807A9F70F949B0E0D94B3280C9400000F
:103AA0002F923F924F925F926F927F928F929F924E
:103AB000AF92BF92CF92DF92EF92FF920F931F933C
:103AC000CF93DF93CDB7DEB7E3970FB6F894DEBFA1
:103AD0000FBECDBF80910901817091E098272091A0
:103AE000B908921781F19093B908811116C00E940C
:103AF000485E8091981783FF09C083EA93E00E9493
:103B0000B55361E080E00F945C0A1DC060E081E085
:103B10000F945C0A8CEB93E014C00091981703FBA0
:103B2000002700F90E94D75D80919817877F8093C6
:103B30009817002341F060E081E00F945C0A85ED66
:103B400093E00E94B5538091151481FF11C18091BB
:103B50009A1590919B15891B8F70843008F008C1CD
:103B60008CE0E3EEF3E1DE01119601900D928A956F
:103B7000E1F780910D1890910E18A0910F18B09157
:103B8000101888A799A7AAA7BBA79C01AD016091AF
:103B9000E3137091E4138091E5139091E6130F9471
:103BA000F6246B017C016093E3137093E41380931C
:103BB000E5139093E6138091111890911218A0913B
:103BC0001318B09114188CA79DA7AEA7BFA79C018E
:103BD000AD016091E7137091E8138091E913909122
:103BE000EA130F94F62468A379A38AA39BA3609396
:103BF000E7137093E8138093E9139093EA1380918D
:103C0000151890911618A0911718B091181888AB34
:103C100099ABAAABBBAB9C01AD016091EB1370916A
:103C2000EC138091ED139091EE130F94F6244B0159
:103C30005C016093EB137093EC138093ED139093FE
:103C4000EE13A7019601C701B6010F94671E2B0161
:103C50003C0128A139A14AA15BA1CA01B9010F9475
:103C6000671E9B01AC01C301B2010F94F7242B0125
:103C70003C01A5019401C501B4010F94671E9B018D
:103C8000AC01C301B2010F94F7240F94A5279B0147
:103C9000AC0160E070E080E89FE30F94F125209193
:103CA00063023091640240916502509166020F9464
:103CB000671E2DEC3CEC4CEC5DE30F94671E20E09E
:103CC00030E040E85EE30F94671E2B013C0120E0EA
:103CD00030E040E85FE30F94011E87FFF1C3A301CA
:103CE0009201C701B6010F94671E28A539A54AA500
:103CF0005BA50F94F7246093E3137093E413809310
:103D0000E5139093E613A301920168A179A18AA11A
:103D10009BA10F94671E2CA53DA54EA55FA50F94F2
:103D2000F7246093E7137093E8138093E91390935B
:103D3000EA13A3019201C501B4010F94671E28A9DB
:103D400039A94AA95BA90F94F7246093EB137093E8
:103D5000EC138093ED139093EE130E94B9BE8CE0A8
:103D6000FE013196A3EEB3E101900D928A95E1F741
:103D70008091B80881110C9433398091B6089091E4
:103D8000B7089C012F5F3F4F3093B7082093B608C8
:103D9000883E934010F40C94333981E08093B80846
:103DA0001092B7081092B60880911311882309F475
:103DB00098C30E94ABCD811194C38091B5088F5FE9
:103DC0008093B5088091B508853620F01092B5082B
:103DD00010921311E09113118E2FEE0F990BAA0B75
:103DE000BB0BFC013197E730F10508F0A0C0882734
:103DF000EE58FF4F8F4F0D94EE240E94A3CD8823E1
:103E000009F495C081E08093290288EE93E00E9436
:103E1000B55380E190E090931D1680931C1685E0C9
:103E20008093101602E80093131684E190E1A0E05D
:103E3000B0E08093141690931516A0931616B093C5
:103E400017160F94800181E09AE590931D168093D8
:103E50001C1686E390E090931F1680931E1687E051
:103E6000809310160093131684E890E0A0E0B0E071
:103E70008093141690931516A0931616B0931716E8
:103E80000F94800152C00E94A3CD882309F44FC033
:103E900048C086EF93E00E94B55381E09AE5909385
:103EA0001D1680931C1680E490E090931F1680935B
:103EB0001E1607E00093101682E88093131684E81C
:103EC00090E0A0E0B0E08093141690931516A093B4
:103ED0001616B09317160F9480010093131127C084
:103EE0008091B408882319F10E94A3CD8823F9F0AA
:103EF0000E94ABCD81111BC0F7C20E94A3CD8823C5
:103F0000B1F00E94ABCD811112C01CC30E94ABCD99
:103F100081110DC042E060E070E0CB010E94C1CD94
:103F200004C00E94ABCD811102C010921311809188
:103F30002902882309F4ACC280910F1190911011CD
:103F4000892B09F08FC18091B1089091B208892B1B
:103F500009F01EC184E096E090931D1680931C1614
:103F600080EA90E890931F1680931E1617E0109336
:103F7000101602E80093131680EA90E0A0E0B0E08B
:103F80008093141690931516A0931616B0931716D7
:103F90000F9480018091060290910702A09108027F
:103FA000B09109020097A105B10511F510921D16F7
:103FB00010921C1615E010931016009313168AE841
:103FC00090E1A0E0B0E08093141690931516A093B2
:103FD0001616B09317160F94800189E090E0909325
:103FE0001D1680931C16109310160093131640C0D4
:103FF0000196A11DB11DF5E0B695A79597958795FA
:10400000FA95D1F70197A109B109009731E0A3070B
:10401000B10558F0B0931D16A0931C1690931F166F
:1040200080931E161093101607C090931D16809350
:104030001C1685E08093101612E8109313168AE878
:1040400090E1A0E0B0E08093141690931516A09331
:104050001616B09317160F94800188E090E09093A5
:104060001D1680931C1685E080931016109313166E
:104070008CE890E1A0E0B0E08093141690931516C0
:10408000A0931616B09317160F9480018091060224
:1040900090910702A0910802B09109020097E1E017
:1040A000AE07B10550F0B0931D16A0931C16909367
:1040B0001F1680931E1687E005C090931D168093EF
:1040C0001C1685E08093101682E88093131688E80A
:1040D00090E1A0E0B0E08093141690931516A093A1
:1040E0001616B09317160F948001809106029091D6
:1040F0000702A0910802B0910902BA2FA92F982FA8
:1041000088270097F1E0AF07B10550F0B0931D1676
:10411000A0931C1690931F1680931E1687E005C06F
:1041200090931D1680931C1685E08093101612E85C
:104130001093131681EA90E0A0E0B0E0809314168B
:1041400090931516A0931616B09317160F9480012E
:1041500080912518882319F082E090E002C083E066
:1041600090E090931D1680931C1685E080931016A6
:104170001093131685E490E1A0E0B0E0809314164C
:1041800090931516A0931616B09317160F948001EE
:104190000091B1081091B208053611057CF4109316
:1041A0001D1600931C1685E08093101682E88093FC
:1041B000131680E090E1A0E0B0E011C0C801845681
:1041C000910990931D1680931C1685E0809310161C
:1041D00082E88093131681E090E1A0E0B0E0809344
:1041E000141690931516A0931616B09317160F94E5
:1041F00080010F5F1F4F1093B2080093B108093C74
:10420000110564F184E094E00E94B55381E090E0F0
:104210009093101180930F118093290281E09AE509
:1042200090931D1680931C168DE290E090931F16BC
:1042300080931E1687E08093101682E880931316F1
:1042400084E890E0A0E0B0E08093141690931516F7
:10425000A0931616B09317160F9480011092B80809
:104260000C94333980919A1590919B15891B8F700E
:1042700009F092C10E9448D781118EC18091981790
:1042800082FD8AC112C384E690E090931D1680934C
:104290001C1610931016009313168EE090E1A0E008
:1042A000B0E08093141690931516A0931616B09351
:1042B00017160F948001C60182539048880F991FEA
:1042C00090931D1680931C161093101600931316CE
:1042D0008FE090E1A0E0B0E0809314169093151663
:1042E000A0931616B09317160F9480010E94C4ED88
:1042F00090E090931D1680931C1685E08093101615
:1043000082E88093131686E190E1A0E0B0E080930C
:10431000141690931516A0931616B09317160F94B3
:10432000800120E030E048EC52E460910714709185
:1043300008148091091490910A140F94671E0F9429
:10434000632670931D1660931C1615E010931016CB
:1043500002E80093131686E290E1A0E0B0E08093BB
:10436000141690931516A0931616B09317160F9463
:10437000800160910E0C70910F0C8091100C909147
:10438000110C0F94632670931D1660931C161093E6
:1043900010160093131686E390E1A0E0B0E080933E
:1043A000141690931516A0931616B09317160F9423
:1043B000800160916509709166098091670990910B
:1043C00068090F94632670931D1660931C16109352
:1043D0001016009313168CE390E1A0E0B0E08093F8
:1043E000141690931516A0931616B09317160F94E3
:1043F00080018091120C9091130C90931D16809364
:104400001C16109310160093131684E390E1A0E09D
:10441000B0E08093141690931516A0931616B093DF
:1044200017160F9480018091690990916A09909301
:104430001D1680931C1610931016009313168AE312
:1044400090E1A0E0B0E08093141690931516A0932D
:104450001616B09317160F9480010091AD08011144
:104460003CC18091AF08811138C18091B40881119D
:104470008BC18091C4159091C515A091C615B091BE
:10448000C7158C3420E19207A105B10509F0A1C13F
:1044900030E6C32E36E1D32E0AE186E194E10E9494
:1044A000205CE090A208F090A308181619060CF002
:1044B00085C38AE1E816F10414F40C94F4347EC345
:1044C0008CE0FE013196A3EEB3E101900D928A9546
:1044D000E1F70E94B9BE809115148D7F8093151469
:1044E00047CC1092B5086ECC86EB95E00E94B55390
:1044F0008091B30890E0A0E0B0E0895B9F4FAE4FA1
:10450000B54A21E03AE530931D1620931C1690938E
:104510001F1680931E1687E08093101682E8809302
:10452000131684E890E0A0E0B0E080931416909316
:104530001516A0931616B09317160F9480011092BB
:10454000B408F3CC81E0809329021092131184EC1B
:1045500095E00E94B55381E09AE590931D168093F3
:104560001C168EE490E090931F1680931E1687E031
:104570008093101682E88093131684E890E0A0E000
:10458000B0E08093141690931516A0931616B0936E
:1045900017160F948001CBCC8CE090E090931D1601
:1045A00080931C1605E00093101682E88093131682
:1045B00084E190E1A0E0B0E080931416909315168A
:1045C000A0931616B09317160F9480010E94A6ECC4
:1045D00020E13EE040E050E00F94572421153105E2
:1045E00091E04907510560F050931D1640931C1649
:1045F00030931F1620931E1687E08093101606C076
:1046000030931D1620931C160093101602E8009399
:10461000131680E190E1A0E0B0E08093141690932F
:104620001516A0931616B09317160F9480010E94CA
:10463000A6EC20E13EE040E050E00F9457242CE34C
:1046400030E040E050E00F94572430931D16209343
:104650001C1615E0109310160093131682E190E1DA
:10466000A0E0B0E08093141690931516A093161650
:10467000B09317160F9480010E94C4ED882391F027
:104680000E94C4ED8F5F8093B008C82ED12C833375
:1046900008F0F9CDC601880F991F90931D168093DD
:1046A0001C1604C010921D1610921C1610931016A2
:1046B000009313168EE090E1A0E0B0E08093141612
:1046C00090931516A0931616B09317160F948001A9
:1046D00010921D1610921C16F7CD20E030E048EC29
:1046E00052E460910E0C70910F0C8091100C90911F
:1046F000110C0F94671E6B017C016091120C70917C
:10470000130C072E000C880B990B0F94081E9B01AD
:10471000AC01C701B6010F94F1250F946A266436E7
:10472000710510F064E670E070931D1660931C161E
:1047300045E0A42EA092101652E8B52EB0921316A2
:1047400084E290E1A0E0B0E08093141690931516F7
:10475000A0931616B09317160F948001C0900E0CFC
:10476000D0900F0CE090100CF090110C20E030E095
:1047700040E253E4C701B6010F94572718160CF016
:104780003AC1011188C137C18091A40801E0080F26
:104790000093A40890E090931D1680931C1685E06A
:1047A0008093101682E88093131682E490E1A0E0D3
:1047B000B0E08093141690931516A0931616B0933C
:1047C00017160F9480010A3008F453CE1092A408F3
:1047D00050CE8A349041A105B10509F459CE80E04C
:1047E0000E949FCE20E030E040E251E40F94671E2B
:1047F0000F94632670931D1660931C1615E010939A
:10480000101602E80093131688E490E1A0E0B0E0EF
:104810008093141690931516A0931616B09317163E
:104820000F94800181E00E949FCE20E030E040E2C2
:1048300051E40F94671E0F94632670931D166093C6
:104840001C1610931016009313168AE490E1A0E052
:10485000B0E08093141690931516A0931616B0939B
:1048600017160F94800182E00E949FCE20E030E076
:1048700040E251E40F94671E0F94632670931D1657
:1048800060931C1610931016009313168CE490E19D
:10489000A0E0B0E08093141690931516A09316161E
:1048A000B09317160F948001F3CD80916509909114
:1048B0006609A0916709B091680988A399A3AAA382
:1048C000BBA36091690970916A09072E000C880BDF
:1048D000990B0F94081E6B017C0120E030E040E052
:1048E00050E40F94F62428A139A14AA15BA10F94AA
:1048F0005727181604F140900E0C50900F0C609042
:10490000100C7090110C6091120C7091130C072E0A
:10491000000C880B990B0F94081E4B015C0120E0E2
:1049200030E040E251E40F94F624A30192010F9489
:104930005727181604F58DE090E090931D1680938C
:104940001C1685E08093101682E88093131684E18C
:1049500090E1A0E0B0E08093141690931516A09318
:104960001616B09317160F948001809112118111C1
:104970003FC081E03DC020E030E040E050E4C701AE
:10498000B6010F94F72428A139A14AA15BA10F9485
:10499000011E87FD0EC020E030E040E251E4C50179
:1049A000B4010F94F724A30192010F94011E87FF15
:1049B000B8CC84E190E090931D1680931C1685E09E
:1049C0008093101682E88093131684E190E1A0E0B2
:1049D000B0E08093141690931516A0931616B0931A
:1049E00017160F94800180911211811101C082E08D
:1049F0008093121196CC6091120C7091130C072EBB
:104A0000000C880B990B0F94081E9B01AC01C70189
:104A1000B6010F9457276091AF0887FDAEC066239B
:104A200009F423CD062E000C770B8BE397E00F944F
:104A3000110A1092AF081092B2081092B10884E0E7
:104A400090E090931D1680931C1685E080931016BD
:104A500002E8009313168EE890E1A0E0B0E08093A6
:104A6000141690931516A0931616B09317160F945C
:104A7000800181E09AE590931D1680931C1683E5D2
:104A800090E090931F1680931E1687E08093101677
:104A90000093131663C01092AD0820E030E040E2AE
:104AA00051E46091A5087091A6088091A7089091A3
:104AB000A8080F94671E0F94632670931D166093C9
:104AC0001C16A0921016B092131684E590E1A0E097
:104AD000B0E08093141690931516A0931616B09319
:104AE00017160F94800120E030E040E251E460911D
:104AF000A9087091AA088091AB089091AC080F9416
:104B0000671E0F94632670931D1660931C16A09267
:104B10001016B092131688E590E1A0E0B0E0809303
:104B2000141690931516A0931616B09317160F949B
:104B3000800182ED95E00E94B55381E09AE5909363
:104B40001D1680931C1681E490E090931F168093AD
:104B50001E1687E080931016B092131684E890E03A
:104B6000A0E0B0E08093141690931516A09316164B
:104B7000B09317160F94800178CC662309F475CC96
:104B80008091B1089091B2089C012F5F3F4F309304
:104B9000B2082093B10865E070E00F94DA24909396
:104BA0001D1680931C1685E08093101682E8809372
:104BB00013168EE890E1A0E0B0E0D4CF1E141F04DD
:104BC0000CF04CCB9091C11580916016981322C0C7
:104BD0009091C2158091611698131CC023E0E216D3
:104BE000F104C4F0909162169093C0158091631601
:104BF0008093C3159330D1F4982F9D7F9038B1F4F2
:104C0000909164169F3409F059C0909165169B34B9
:104C100009F054C08AE1E0E6F6E1DF011D928A95D1
:104C2000E9F71092A3081092A20818CB833809F074
:104C300045C080916416909165169827892798271A
:104C4000A0E0B0E08093C4159093C515A093C6155D
:104C5000B093C715C0906616D12CE12CF12CC092F0
:104C6000C815D092C915E092CA15F092CB15A7E6E7
:104C7000B6E140E050E0BA014C155D056E057F05D8
:104C800008F04AC04A015B01B694A79497948794B0
:104C9000F4013696EE0FFF1FE054FA4E8C9190E02F
:104CA000982F882711962C911197822B91838083BE
:104CB0004E5F5F4F6F4F7F4F1296DECF813861F5A9
:104CC0008091641690E0A0E0B0E08093C4159093CA
:104CD000C515A093C615B093C71580916516482FCA
:104CE00050E060E070E04093C8155093C9156093A0
:104CF000CA157093CB15A6E6B6E1ECECF5E190E0B1
:104D000020E030E02817390739F04D9150E0419309
:104D100051932F5F3F4FF6CF8AE1E0E6F6E1DF01E6
:104D20001D928A95E9F71092A3081092A20885E1D6
:104D300094E00E94B55360911311161664F4062E88
:104D4000000C770B80E397E00F94110A8AE00E9431
:104D5000AA520C94E5346091CC157091CD158EE17A
:104D600097E00F94F3098AE00E94AA524091C4157B
:104D70005091C5156091C6157091C7158FE097E0E9
:104D80000F94E2098AE00E94AA528091C415909182
:104D9000C515A091C615B091C715E5E7F2E000E092
:104DA00010E0419151916191719141155105610559
:104DB0007105D1F1481759076A077B0791F5AC01D6
:104DC000BD014850504161097109453051056105E7
:104DD000710568F1AC01BD01477F42335041610567
:104DE000710541F18433F0E19F07A105B10511F18F
:104DF000AC01BD014654504161097109473051056C
:104E000061057105D0F0AC01BD0144555041610907
:104E10007109453051056105710588F402E110E022
:104E20000EC00F5F1F4FBDCF0FEF1FEF08C003E095
:104E300010E005C008E010E002C00FE010E08A506A
:104E40009042A109B109833D9105A105B10530F05A
:104E50000F3F2FEF120721F40C94E53409E110E025
:104E6000F6E3CF2EF4E0DF2EF60181916F01882367
:104E700019F00E94AA52F8CFB801012E000C880B3D
:104E8000990B0E941E530E94AF5383E097E00E944B
:104E9000B5530A31110510F00C94E134F80188275C
:104EA000E758FF4F8F4F0D94EE248091CC159091D1
:104EB000CD1581309105E1F4109229028FEF809396
:104EC000841A60E080E00F945C0A04E414E0D801E6
:104ED0008D918D01882319F00E94AA52F8CF81E0AC
:104EE0009AE590931D1680931C168EE290E0AFC059
:104EF0008230910509F0C5C081E0809329020E94AB
:104F000035EE8FEF96E090939E0980939D098BE09C
:104F100090E090931D1680931C1605E000931016E8
:104F200012E81093131680E092E1A0E0B0E08093C5
:104F3000141690931516A0931616B09317160F9487
:104F4000800110921D1610921C16009310161093DB
:104F500013168EE090E1A0E0B0E0809314169093D9
:104F60001516A0931616B09317160F948001109281
:104F70001D1610921C1600931016109313168FE036
:104F800090E1A0E0B0E08093141690931516A093E2
:104F90001616B09317160F94800110921D161092DA
:104FA0001C16009310161093131686E190E1A0E0F2
:104FB000B0E08093141690931516A0931616B09334
:104FC00017160F94800162E070E080E090E00E948C
:104FD000B3CE10921D1610921C160093101610934B
:104FE000131680E190E1A0E0B0E080931416909356
:104FF0001516A0931616B09317160F9480011092F1
:105000001D1610921C16009310161093131682E1B1
:1050100090E1A0E0B0E08093141690931516A09351
:105020001616B09317160F9480010EE614E0F801DF
:1050300081918F01882319F00E94AA52F8CF81E054
:105040009AE590931D1680931C168DE290E0909344
:105050001F1680931E1687E08093101682E88093B7
:10506000131684E890E0A0E0B0E0809314169093CB
:105070001516A0931616B09317160F9480010C9472
:10508000E5348330910549F581E08093290208E9F0
:1050900014E0D8018D918D018823C9F00E94AA5295
:1050A000F8CF8091C4159091C515A091C615B09107
:1050B000C7158233F0E19F07A105B10509F05BC474
:1050C0008091CC159091CD15009709F023C4809163
:1050D0000502882309F40DC31DC3049711F00C9435
:1050E000E534109229020C94E5348091CC1590910E
:1050F000CD1581309105D1F41092290280910502DD
:10510000882319F082E090E002C083E090E0909361
:105110001D1680931C1685E08093101682E88093FC
:1051200013168EE190E1A0E0B0E09FCF82309105B0
:1051300019F502EC14E0F80181918F01882319F030
:105140000E94AA52F8CF81E0809329028091121127
:10515000843049F081E09AE590931D1680931C16E7
:1051600085E390E074CF81E09AE590931D168093DB
:105170001C1686E390E06BCF8330910509F04CC09C
:1051800020910502222319F190931D1680931C167D
:1051900085E08093101682E8809313168EE190E1EB
:1051A000A0E0B0E08093141690931516A093161605
:1051B000B09317160F94800140E060E070E088EC37
:1051C00092E40E949CEE109205020C94E53482E079
:1051D00090E090931D1680931C1685E08093101626
:1051E00082E8809313168EE190E1A0E0B0E0809316
:1051F000141690931516A0931616B09317160F94C5
:10520000800140E060E070E0CB010E949CEE81E014
:10521000809305020C94E534049711F00C94E53466
:10522000809178098823F1F082E090E090931D1638
:1052300080931C1685E08093101682E880931316E5
:105240008FE190E1A0E0B0E08093141690931516E2
:10525000A0931616B09317160F9480011092780938
:105260000C94E53483E090E090931D1680931C1617
:1052700085E08093101682E8809313168FE190E109
:10528000A0E0B0E08093141690931516A093161624
:10529000B09317160F94800181E0809378090C94E5
:1052A000E5346091CC157091CD1580E090E00F94BD
:1052B000061E6B017C0120E030E04AEF53E40F94BE
:1052C000011E87FF11C020E030E040E251E4C70139
:1052D000B6010F94572718166CF0C12CD12C70E230
:1052E000E72E71E4F72E06C0C12CD12CEAEFEE2E8A
:1052F000E3E4FE2EC701B6010F94632670934F02BC
:1053000060934E020C94E5348091C4159091C515BC
:10531000A091C615B091C7158830F0E19F07A1058F
:10532000B10509F050C081E09AE590931D16809375
:105330001C168DE290E090931F1680931E1687E056
:105340008093101612E81093131684E890E0A0E002
:10535000B0E08093141690931516A0931616B09390
:1053600017160F94800110921D1610921C1605E05E
:10537000009310161093131680E190E1A0E0B0E0C6
:105380008093141690931516A0931616B0931716C3
:105390000F94800110921D1610921C160093101687
:1053A0001093131682E190E1A0E0B0E08093141610
:1053B00090931516A0931616B09317160F948001AC
:1053C0000E9435EE8FC08A3020E19207A105B10519
:1053D000E1F58091CC159091CD15813F910511F0AB
:1053E0000C94E53481E09AE590931D1680931C1689
:1053F00086E390E090931F1680931E1687E08093BB
:10540000101682E88093131684E890E0A0E0B0E0E4
:105410008093141690931516A0931616B093171632
:105420000F9480014EE755E065E875E084E00E9446
:105430007F9560E081E795E00E94F6ED87E695E0D4
:1054400090939E0980939D094DC08C309041A10599
:10545000B10509F047C08091CC159091CD15019709
:1054600009F040C00F94E0171092121181E0809370
:1054700029028CE090E090931D1680931C1685E025
:105480008093101612E81093131684E190E1A0E0C7
:10549000B0E08093141690931516A0931616B0934F
:1054A00017160F94800181E09AE590931D16809362
:1054B0001C1685E390E090931F1680931E1687E0DC
:1054C000809310161093131684E890E0A0E0B0E0EB
:1054D0008093141690931516A0931616B093171672
:1054E0000F9480018091C4159091C515A091C615A7
:1054F000B091C7158C309041A105B10511F00C9405
:10550000E5348091CC159091CD15029711F00C9453
:10551000E5340F94E01781E08093AF0810921211E8
:10552000809329021092B2081092B10881E09AE5A6
:1055300090931D1680931C1682E590E088CD2091F3
:10554000CC153091CD15B90180E090E037FF09C04E
:105550000F94061E20E030E040E857E40F94F62454
:1055600002C00F94061E20E030E048EC52E40F9495
:10557000F1256B017C0120E030E040EA51EC0F9412
:10558000572787FD31C020E030E040EA51E4C701F1
:10559000B6010F94011E18163CF1A7019601609107
:1055A0000714709108148091091490910A140F94B3
:1055B000F62420E030E048EC53E40F94671E905846
:1055C0000F946326CB010F947504C0920714D092F8
:1055D0000814E0920914F0920A148AEF96E090936E
:1055E0009E0980939D0928C020E030E048EC52E4F9
:1055F00060910714709108148091091490910A1415
:105600000F94671E0F94632670931D1660931C16EB
:1056100085E08093101682E88093131686E290E16D
:10562000A0E0B0E08093141690931516A093161680
:10563000B09317160F9480016091071470910814AD
:105640008091091490910A148E010B5E1F4F23E084
:1056500041E00F94D9189F938F938CEE96E09F931F
:105660008F93045111091F930F930F94991DC80133
:105670000E948DCF0F900F900F900F900F900F9072
:105680000C94E5348091CC159091CD15009729F4B8
:1056900081E0809329020C94E53481309105B1F4C6
:1056A00080910502882349F081E09AE590931D16C8
:1056B00080931C168CE390E0CACC81E09AE590932D
:1056C0001D1680931C168BE390E0C1CC82309105AF
:1056D000F9F28330910539F58091050240E0882385
:1056E00089F060E070E088EC92E40E949CEE1092F9
:1056F000050281E09AE590931D1680931C1689E3BC
:1057000090E0A5CC60E070E0CB010E949CEE81E0CF
:105710008093050281E09AE590931D1680931C16F4
:105720008AE390E094CC8530910559F540E060E043
:1057300070E084E393E40E9436CD46E060E070E0E0
:105740008CE892E40E9436CD84EB90E090931D1695
:1057500080931C1605E00093101612E810931316A0
:1057600084E390E1A0E0B0E08093141690931516C6
:10577000A0931616B09317160F94800186E490E05C
:105780002DC08630910599F540E060E070E080E73B
:1057900093E40E9436CD46E060E070E08CED92E448
:1057A0000E9436CD80EF90E090931D1680931C16DA
:1057B00005E00093101612E81093131684E390E1AD
:1057C000A0E0B0E08093141690931516A0931616DF
:1057D000B09317160F9480018EE690E090931D16FB
:1057E00080931C160093101610931316BFC0813FB0
:1057F000910511F00C94E53440E060E070E0CB01DD
:105800000E949CEE41E060E070E0CB010E949CEEC3
:105810001092050240E060E070E0CB010E9436CDBE
:1058200046E060E070E0CB010E9436CD10921D167C
:1058300010921C1605E00093101612E81093131630
:1058400084E390E1A0E0B0E08093141690931516E5
:10585000A0931616B09317160F94800161E070E0C4
:1058600080E090E00E94B3CE10921D1610921C169C
:1058700000931016109313168AE390E1A0E0B0E0B5
:105880008093141690931516A0931616B0931716BE
:105890000F94800161E070E080E090E00E94B3CE60
:1058A00084E190E090931D1680931C1600931016CF
:1058B0001093131684E190E1A0E0B0E080931416F9
:1058C00090931516A0931616B09317160F94800197
:1058D00081E09AE590931D1680931C1689E390E071
:1058E00090931F1680931E1687E0809310161093D6
:1058F000131684E890E0A0E0B0E080931416909333
:105900001516A0931616B09317160F94800182E017
:105910000C94DE3481309105A9F440E060E070E041
:10592000CB010E9436CD10921D1610921C1685E0F8
:105930008093101682E88093131684E390E1A0E030
:10594000B0E093CB029711F00C94E53446E060E0B0
:1059500070E0CB010E9436CD10921D1610921C16DD
:1059600085E08093101682E8809313168AE390E115
:10597000A0E0B0E07ACB843320E19207A105B10525
:1059800051F46091CC157091CD1580E090E00F94AA
:10599000061E40E010C08A339041A105B10511F008
:1059A0000C94E5346091CC157091CD1580E090E0B9
:1059B0000F94061E46E00E9436CD0C94E53480918B
:1059C000CC159091CD15009709F462CE81309105E8
:1059D00009F04CC080912518882319F083E090E0ED
:1059E00002C082E090E090931D1680931C1685E023
:1059F0008093101682E88093131685E490E1A0E06E
:105A0000B0E08093141690931516A0931616B093D9
:105A100017160F9480018AE090E090931D168093F2
:105A20001C1685E08093101682E88093131680E0A0
:105A300092E1A0E0B0E08093141690931516A09325
:105A40001616B09317160F9480010E94A3CD8111F2
:105A500003C08CED96E002C080ED96E090939E0925
:105A600080939D0982E08093131171C1823091056A
:105A700009F0A8C081E08093290288E0E5EAF8E017
:105A8000DF011D928A95E9F780E090E0A0E2B1E4A1
:105A90008093A5089093A608A093A708B093A808A0
:105AA0008093A9089093AA08A093AB08B093AC0880
:105AB00084E690E090931D1680931C1605E00093F9
:105AC000101612E81093131684E590E1A0E0B0E000
:105AD0008093141690931516A0931616B09317166C
:105AE0000F94800120E030E040E251E46091A90889
:105AF0007091AA088091AB089091AC080F94671E32
:105B00000F94632670931D1660931C160093101655
:105B10001093131688E590E1A0E0B0E0809314168E
:105B200090931516A0931616B09317160F94800134
:105B300060910E0C70910F0C8091100C9091110CD3
:105B40000F94632670931D1660931C160093101615
:105B50001093131686E390E1A0E0B0E08093141652
:105B600090931516A0931616B09317160F948001F4
:105B70008091120C9091130C90931D1680931C161B
:105B8000009310161093131684E390E1A0E0B0E0A8
:105B90008093141690931516A0931616B0931716AB
:105BA0000F94800162E070E080E090E00E94B3CE4C
:105BB00081E09AE590931D1680931C1681E490E095
:105BC0000C9421368330910509F076C01092B30809
:105BD00080E00E949FCE20E030E040E251E40F944C
:105BE000671E0F94632670931D1660931C1605E0C4
:105BF0000093101612E81093131688E490E1A0E0C9
:105C0000B0E08093141690931516A0931616B093D7
:105C100017160F94800181E00E949FCE20E030E0B3
:105C200040E251E40F94671E0F94632670931D1693
:105C300060931C1600931016109313168AE490E1DB
:105C4000A0E0B0E08093141690931516A09316165A
:105C5000B09317160F94800182E00E949FCE20E03F
:105C600030E040E251E40F94671E0F946326709376
:105C70001D1660931C1600931016109313168CE4D7
:105C800090E1A0E0B0E08093141690931516A093D5
:105C90001616B09317160F94800162E070E080E052
:105CA00090E00E94B3CE81E09AE590931D16809318
:105CB0001C1687E490E0C5C78430910509F485C6B9
:105CC0008530910549F44EE750E160E070E089EEDF
:105CD00094E00F942F0179C6069709F076C68CECF4
:105CE00096E090939E0980939D098BE090E02BC2F3
:105CF0008091CC159091CD15019711F51092290244
:105D000081E09AE590931D1680931C168FE390E036
:105D100090931F1680931E1687E08093101682E8DA
:105D20008093131684E890E0A0E0B0E0809314160E
:105D300090931516A0931616B09317160F94800122
:105D40008091CC159091CD15029709F03EC681E067
:105D50009AE590931D1680931C1680E490E077C915
:105D6000E091CC15F091CD153197EB30F10508F0AD
:105D7000E4C18827ED56FF4F8F4F0D94EE2480919C
:105D8000141480FF5CC6869580FD5CC658C62DEC59
:105D90003CEC4CEC5DE36091071470910814809129
:105DA000091490910A140F94F7246B017C0120E0F0
:105DB00030E040EA51EC0F94572787FDC2C120E044
:105DC00030E040EA51E4C701B6010F94011E1816F5
:105DD0000CF03FC6B6C12DEC3CEC4CEC5DE36091A1
:105DE0000714709108148091091490910A140F946B
:105DF000F6246B017C0120E030E040EA51EC0F9486
:105E0000572787FD9EC120E030E040EA51E4C701FA
:105E1000B6010F94011E18160CF092C692C180E0D4
:105E20000F94C2060E94A3CD811103C083E796E0C0
:105E300002C085E696E090939E0980939D0982E0DA
:105E40008093131181E09AE590931D1680931C16A0
:105E500084E590E090931F1680931E1687E0809350
:105E6000101682E88093131684E890E0A0E0B0E07A
:105E70008093141690931516A0931616B0931716C8
:105E80000F9480015EC183E08093131183E090E062
:105E900090931D1680931C1685E08093101682E85F
:105EA000809313168DE890E1A0E0B0E08093141683
:105EB00090931516A0931616B09317160F948001A1
:105EC000E12CF12C00E0DD24D394AA24A39445E036
:105ED000942E55E0852E62E8762EDD2031F0CC241C
:105EE000C39435E0B32E10E005C0CC24CA94BB2483
:105EF000BA9414E0DA24B116D1F1802F90E04897DB
:105F0000A4F50F5FF701919EE00DF11D1124EE0F36
:105F1000FF1FEE0FFF1FE559FC4E20E030E04AE77F
:105F200054E460817181828193810F94671E0F9484
:105F3000632670931D1660931C1680921016709243
:105F40001316802F90E08158974F880F991F092EC4
:105F5000000CAA0BBB0B8093141690931516A093FC
:105F60001616B09317160F9480011C0DC4CFBFEF07
:105F7000EB1AFB0AE5E0EE16F10409F0AECF81E082
:105F80009AE590931D1680931C1685E590E09093FA
:105F90001F1680931E1687E08093101682E8809368
:105FA000131684E890E0A0E0B0E08093141690937C
:105FB0001516A0931616B09317160F94800187E05C
:105FC00096E090939E0980939D09BBC042E060E0FB
:105FD00070E080E890E40E94C1CD40E060E070E0B5
:105FE0008DE693E40E94C1CD41E060E070E081E67F
:105FF00093E413C042E060E070E080E890E40E9427
:10600000C1CD40E060E070E080E292E40E94C1CD4A
:1060100041E060E070E080E292E40E94C1CD86E061
:10602000809313118EC042E060E070E080E890E45D
:106030000E94C1CD40E060E070E089ED93E4E6CFDE
:1060400042E060E070E080E890E40E94C1CD40E072
:1060500060E070E089ED93E40CC042E060E070E045
:1060600080E890E40E94C1CD40E060E070E080E212
:1060700092E40E94C1CD41E060E070E08DEC93E4D9
:10608000CCCF8091251881111CC083E090E09093C3
:106090001D1680931C1685E08093101682E880936D
:1060A000131685E490E1A0E0B0E08093141690937D
:1060B0001516A0931616B09317160F94800181E061
:1060C0001BC082E090E090931D1680931C1685E023
:1060D0008093101682E88093131685E490E1A0E087
:1060E000B0E08093141690931516A0931616B093F3
:1060F00017160F94800180E00F94C20620E030E074
:1061000048EC52E4609107147091081480910914CE
:1061100090910A140F94671E0F94632670931D16B6
:1061200060931C1685E08093101682E88093131606
:1061300086E290E1A0E0B0E09BCE8BEE95E00E947D
:10614000B5538AE090E090931D1680931C1685E06D
:106150008093101682E8809313164BC184E08093DD
:1061600013118091C4159091C515A091C615B091D9
:10617000C7156091CC157091CD158834F0E19F075B
:10618000A105B10509F453C08A3420E19207A105A5
:10619000B10509F456C08C3430E19307A105B1056F
:1061A00009F45AC086349041A105B10509F05EC0DA
:1061B00063307105B9F58AED95E090939E0980935F
:1061C0009D0981E08093B408809329021092A4086D
:1061D00081E09AE590931D1680931C168AE490E066
:1061E00090931F1680931E1687E08093101612E876
:1061F0001093131684E890E0A0E0B0E080931416AA
:1062000090931516A0931616B09317160F9480014D
:106210008AE090E090931D1680931C1685E0809391
:106220001016E5C06093B30810921311CEC380E03E
:1062300090E8ADEEB3E48CA39DA3AEA3BFA3312C35
:1062400015C080E090E0A1EEB3E48CA39DA3AEA3C3
:10625000BFA3332433940AC080E090E0ABEEB3E4F4
:106260008CA39DA3AEA3BFA382E0382E80E090E074
:106270000F94061E20E030E040E251E40F94F12537
:106280006B017C0120E030E0A9010F94011E87FF23
:1062900009C010929E0810929F081092A0081092B8
:1062A000A1081FC02CA13DA14EA15FA1C701B6014D
:1062B0000F94572718164CF0C0929E08D0929F0852
:1062C000E092A008F092A1080CC08CA19DA1AEA103
:1062D000BFA180939E0890939F08A093A008B093BD
:1062E000A10860919E0870919F088091A0089091EC
:1062F000A108432D0E94C1CD61E070E080E090E0F4
:106300000E94B3CE80E00E949FCE20E030E040E2C9
:1063100051E40F94671E0F94632670931D166093CB
:106320001C1605E00093101612E81093131688E46B
:1063300090E1A0E0B0E08093141690931516A0931E
:106340001616B09317160F94800181E00E949FCE1D
:1063500020E030E040E251E40F94671E0F94632682
:1063600070931D1660931C1600931016109313164D
:106370008AE490E1A0E0B0E08093141690931516A3
:10638000A0931616B09317160F94800182E00E9416
:106390009FCE20E030E040E251E40F94671E0F945E
:1063A000632670931D1660931C16009310161093AD
:1063B00013168CE490E1A0E0B0E080931416909363
:1063C0001516A0931616B09317160F94800161E06E
:1063D00070E080E090E00E94B3CE109213118AE04A
:1063E00090E090931D1680931C1600931016109346
:1063F000131680E092E1A0E0B0E00C943528809183
:10640000C4159091C515A091C615B091C7158635D4
:10641000E0E19E07A105B10509F041C020E030E0B0
:1064200040E253E460910E0C70910F0C8091100CBF
:106430009091110C0F94011E2091CC153091CD1527
:1064400087FF0AC42530310508F006C480EA90E0D1
:1064500090931D1680931C1685E08093101612E809
:106460001093131680E290E1A0E0B0E08093141640
:1064700090931516A0931616B09317160F948001DB
:1064800065E070E080E090E00E94B3CE81E09AE5A4
:1064900090931D1680931C1682E490E0D2C384353D
:1064A000F0E19F07A105B105B9F46091CC15709199
:1064B000CD1580E090E00F94061E20E030E040E231
:1064C00051E40F94F1256093A5087093A60880937A
:1064D000A7089093A80879C288359041A105B10515
:1064E00009F073C26091CC157091CD1580E090E0F9
:1064F0000F94061E20E030E040E251E40F94F125B5
:106500006093A9087093AA088093AB089093AC0895
:106510005CC26091CC157091CD1584EC95E00F9420
:10652000F3098091CC159091CD1582309105A1F0A1
:1065300038F4009771F00197E1F482E195E043C2ED
:106540008430910579F058F0059799F489E995E040
:106550000BC08CEF94E037C286EB95E005C08CEA67
:1065600095E002C087EA95E090939E0980939D098B
:106570002CC286E295E027C285E395E00E94B553E0
:106580008091CC159091CD158130910519F46499C5
:10659000C3C41BC2892B09F018C283E495E00E9492
:1065A000B55380919A08813039F589E595E00E94CC
:1065B000B55381E09AE590931D1680931C168EE2E8
:1065C00090E090931F1680931E1687E0809310161C
:1065D00082E88093131684E890E0A0E0B0E0809316
:1065E000141690931516A0931616B09317160F94C1
:1065F00080011092111135C0823069F48DE695E06A
:106600000E94B55381E09AE590931D1680931C1665
:1066100086E390E00EC0833031F581E895E00E947A
:10662000B55381E09AE590931D1680931C1681E482
:1066300090E090931F1680931E1687E080931016AB
:1066400082E88093131684E890E0A0E0B0E08093A5
:10665000141690931516A0931616B09317160F9450
:1066600080011092461310929A080E9435EEADC137
:106670008091CC159091CD158F3F910531F028F088
:106680008FEF90E0A0E0B0E002C0A0E0B0E0809327
:10669000060290930702A0930802B093090280912A
:1066A000060290910702A0910802B091090200979A
:1066B000A105B10509F510921D1610921C1605E0F2
:1066C0000093101612E8109313168AE890E1A0E0E8
:1066D000B0E08093141690931516A0931616B093FD
:1066E00017160F94800189E090E090931D16809317
:1066F0001C16009310163DC00196A11DB11D05E0AA
:10670000B695A795979587950A95D1F70197A10911
:10671000B109009731E0A307B10550F0B0931D1601
:10672000A0931C1690931F1680931E1687E005C039
:1067300090931D1680931C1685E08093101612E826
:10674000109313168AE890E1A0E0B0E0809314164D
:1067500090931516A0931616B09317160F948001F8
:1067600088E090E090931D1680931C1685E080933E
:106770001016109313168CE890E1A0E0B0E080931F
:10678000141690931516A0931616B09317160F941F
:1067900080018091060290910702A0910802B091B9
:1067A0000902BA2FA92F982F88270097E1E0AE079A
:1067B000B10550F0B0931D16A0931C1690931F16B0
:1067C00080931E1687E005C090931D1680931C16BB
:1067D00085E08093101682E88093131681EA90E09A
:1067E000A0E0B0E00C94352885E995E00E94B5530F
:1067F0000E942ACD4091C4155091C5156091C615CF
:106800007091C715882339F0433DF0E25F076105B9
:10681000710509F4C7C3423D50426105710509F095
:10682000D4C08091CC159091CD15019709F00CC57D
:106830000E942ACD882309F407C58091841A87FD18
:10684000C4C0A2E18A02C0011124815C934E0E945F
:10685000F05DC12C90E2D92EE12CF12C05E012E87C
:1068600010921D1610921C160093101610931316FA
:10687000C0921416D0921516E0921616F0921716C2
:106880000F948001BFEFCB1ADB0AEB0AFB0AEAE0A8
:10689000CE16E0E2DE06E104F10411F70091841A5D
:1068A000F2E10F02800111240952154EF801019006
:1068B0000020E9F7C8018E1B9F0B439697FD0196B8
:1068C0007C01F594E7941E141F040CF0C6C49E01CD
:1068D0002F5F3F4F690184E1D9011D928A95E9F745
:1068E000A70166EA75E0C9010F946A28B801C601DC
:1068F0008E0D9F1D0F94552840E050E260E070E03F
:10690000C6010F942F0162E070E080E090E00E94E9
:10691000B3CE40E060E070E08FE793E40E949CEE2D
:1069200041E060E070E08FE793E40E949CEE1092FB
:1069300005028DE090E090931D1680931C1685E073
:106940008093101612E81093131684E190E1A0E0F2
:10695000B0E08093141690931516A0931616B0937A
:1069600017160F94800162E070E080E090E00E94D2
:10697000B3CE81E09AE590931D1680931C1685E3B3
:1069800090E090931F1680931E1687E08093101658
:106990001093131684E890E0A0E0B0E08093141602
:1069A00090931516A0931616B09317160F948001A6
:1069B00081E0809329028093111183E0809312116A
:1069C00004C08EE895E00E94B55380E5E0ECF5E167
:1069D000DF011D928A95E9F78AE58093C11585EA62
:1069E0008093C2150C942E2186E194E10E94FE5BF7
:1069F000F701E05AF94E8083809160168A3581F064
:106A00001E141F0414F00C944D22D601E02F1D9289
:106A1000EA95E9F71092A3081092A2080C944D226F
:106A200062E070E080E090E00E94B3CEFFEFEF1AEA
:106A3000FF0AF092A308E092A2080C944D228CEB7E
:106A400096E002C08BEA96E090939E0980939D09A0
:106A500055CB88E290E00F9475042DEC3CEC4CECA7
:106A60005DE360910714709108148091091490916E
:106A70000A140F94F7246B017C0120E030E040EA17
:106A800051EC0F94572787FD12C020E030E040EA18
:106A900051E4C701B6010F94011E181644F0C092CC
:106AA0000714D0920814E0920914F0920A1420E01E
:106AB00030E048EC52E46091071470910814809122
:106AC000091490910A140F94671E0F946326709313
:106AD0001D1660931C1685E08093101682E8809343
:106AE000131686E290E1A0E0B0E080931416909334
:106AF0001516A0931616B09317160F948001609187
:106B00000714709108148091091490910A148E0151
:106B10000B5E1F4F23E041E00F94D9189F938F9392
:106B20008DE996E09F938F93045111091F930F9362
:106B30000F94991DC8010E948DCF88E996E076C018
:106B400088ED9FEF0F9475042DEC3CEC4CEC5DE36D
:106B500060910714709108148091091490910A149F
:106B60000F94F6246B017C0120E030E040EA51EC08
:106B70000F94572787FD12C020E030E040EA51E42F
:106B8000C701B6010F94011E181644F0C0920714F5
:106B9000D0920814E0920914F0920A1420E030E038
:106BA00048EC52E460910714709108148091091424
:106BB00090910A140F94671E0F94632670931D160C
:106BC00060931C1685E08093101682E8809313165C
:106BD00086E290E1A0E0B0E0809314169093151641
:106BE000A0931616B09317160F94800160910714A6
:106BF000709108148091091490910A148E010B5E13
:106C00001F4F23E041E00F94D9189F938F938AE898
:106C100096E09F938F93045111091F930F930F9444
:106C2000991DC8010E948DCF85E896E090939E093A
:106C300080939D090F900F900F900F900F900F90E1
:106C400080CA90931F1680931E1687E080931016BB
:106C5000109313160C9431282430310589F481E007
:106C60000F94CA172091A9083091AA084091AB0847
:106C70005091AC080F94F72441E00F94A117B2C0D3
:106C80002530310508F4F4C02630310509F431C14E
:106C900008F023C181E08093AD0840E060E070E03F
:106CA0008EE393E40E9436CD20E030E048EC52E4DD
:106CB00060910E0C70910F0C8091100C9091110C42
:106CC0000F94671E6B017C016091120C7091130C84
:106CD000072E000C880B990B0F94081E9B01AC012A
:106CE000C701B6010F94F1250F946A266436710529
:106CF00010F064E670E070931D1660931C1605E0BA
:106D00000093101612E81093131684E290E1A0E0AD
:106D1000B0E08093141690931516A0931616B093B6
:106D200017160F94800160910E0C70910F0C8091DA
:106D3000100C9091110C0F94632670931D166093A4
:106D40001C16009310161093131686E390E1A0E032
:106D5000B0E08093141690931516A0931616B09376
:106D600017160F9480018091120C9091130C909340
:106D70001D1680931C16009310161093131684E3AF
:106D800090E1A0E0B0E08093141690931516A093C4
:106D90001616B09317160F94800165E070E080E03E
:106DA00090E00E94B3CE81E09AE590931D16809307
:106DB0001C1684E490E090931F1680931E1687E0C3
:106DC000809310161093131684E890E0A0E0B0E0D2
:106DD0008093141690931516A0931616B093171659
:106DE0000F94800120E030E040E251E46091A5087A
:106DF0007091A6088091A7089091A8080F94671E2B
:106E00000F94632670931D1660931C1605E0009383
:106E1000101612E81093131684E590E1A0E0B0E09C
:106E20008093141690931516A0931616B093171608
:106E30000F94800120E030E040E251E46091A90825
:106E40007091AA088091AB089091AC080F94671ECE
:106E50000F94632670931D1660931C1600931016F2
:106E60001093131688E590E1A0E0B0E00C9435286B
:106E70002230310579F480E00F94CA172091A508DB
:106E80003091A6084091A7085091A8080F94F724C4
:106E900040E0F3CE2330310570F081E00F94CA1743
:106EA0002091A9083091AA084091AB085091AC08F4
:106EB0000F94F624E1CE2130310509F093CF80E024
:106EC0000F94CA172091A5083091A6084091A708F1
:106ED0005091A8080F94F624DBCF213F310509F02B
:106EE00081CF1092AD0861E070E080E090E00E94F8
:106EF000B3CE81E09AE590931D1680931C1681E431
:106F000090E090931F1680931E1687E080931016D2
:106F100082E88093131658CF83EF95E00E94B55313
:106F200081E00E9468948DE090E090931D1680931C
:106F30001C1685E08093101612E81093131684E156
:106F400090E1A0E0B0E08093141690931516A09302
:106F50001616B09317160F94800183E080931211D8
:106F600081E09AE590931D1680931C1685E390E0CE
:106F700090931F1680931E1687E08093101610932F
:106F8000131684E890E0A0E0B0E08093141690938C
:106F90001516A0931616B09317160F948001109231
:106FA0009A0813CD8BE096E00E94B5538091851A24
:106FB0009091861A99272091CC153091CD15821782
:106FC000930708F402CD8EE995E00E94B5538091B5
:106FD000CC1581508093841AA4ED8A2EA0E29A2EBB
:106FE000A12CB12C05E012E810921D1610921C166F
:106FF0000093101610931316809214169092151683
:10700000A0921616B09217160F9480012FEF821AD5
:10701000920AA20AB20A3EED831630E29306A10458
:10702000B10411F78091841AA2E18A02C0011124EF
:10703000FC01E952F54E7F0101900020E9F7C701FC
:107040008E1B9F0B439697FD01968C011595079516
:1070500010161106FCF49E012F5F3F4F690184E179
:10706000D9011D928A95E9F7A80166EA75E0C90180
:107070000F946A28B701C601800F911F0F945528FD
:1070800044ED50E260E070E0C6010F942F0105E08E
:1070900012E806C044ED50E260E070E0C701F5CFB1
:1070A00010921D1610921C160093101610931316B2
:1070B0008092141690921516A0921616B09217167A
:1070C0000F948001BFEF8B1A9B0AAB0ABB0AE6EE56
:1070D0008E16E0E29E06A104B10411F78E010F5F47
:1070E0001F4F84E1D8011D928A95E9F78091861A95
:1070F0008F938091851A8F938091CD158F93809176
:10710000CC158F9380EB95E09F938F931F930F93F4
:107110000F9484284EED50E260E070E0C8010F94B7
:107120002F0162E070E080E090E00E94B3CE0FB6E5
:10713000F894DEBF0FBECDBF31E2C32E32E1D32EB5
:10714000E12CF12C43E1442E40E6542E612C712CAD
:1071500088248394912CAA24AA94BA2C75E0272E13
:10716000E2E83E2E0AE010E08091851A9091861A9E
:107170008815990594F1B0921D16A0921C162092C4
:1071800010163092131640921416509215166092F3
:107190001616709217160F94800110931D16009307
:1071A0001C162092101630921316C0921416D0920C
:1071B0001516E0921616F09217160F948001FFEF45
:1071C0008F1A9F0A20E1420E511C611C711C3FEF77
:1071D000C31AD30AE30AF30AC7CF8091CC15909162
:1071E000CD1524E0880F991F2A95E1F78D5F9F49FF
:1071F000A0E0B0E020EF37E830931D1620931C1676
:1072000005E00093101612E81093131680931416DD
:1072100090931516A0931616B09317160F9480012D
:107220008091CC159091CD15805E9D4EA0E0B0E090
:1072300026E030E030931D1620931C1600931016A4
:10724000109313160C9435288091CC159091CD1580
:10725000892B11F40C94482BB8CB40E050E260E04D
:1072600070E0C8014ECBE3960FB6F894DEBF0FBEB8
:10727000CDBFDF91CF911F910F91FF90EF90DF90E5
:10728000CF90BF90AF909F908F907F906F905F90C6
:107290004F903F902F9008952F923F924F925F9280
:1072A0006F927F928F929F92AF92BF92CF92DF9216
:1072B000EF92FF920F931F93CF93DF93CDB7DEB77B
:1072C000C154D1090FB6F894DEBF0FBECDBF2296D0
:1072D0008FAF2297209145122CAF21E020934512C9
:1072E000809166128D3409F4B3C4843511F40C9482
:1072F0003B4B873411F00C94424B80916412909177
:1073000065128B31910509F420C2B4F484309105E3
:1073100034F482309105E4F597FF2EC095C4853191
:10732000910511F40C94444B8A31910509F409C27A
:10733000049709F089C4C6C18A32910509F4B5C31E
:107340004CF48D319105B1F00CF429C24E9709F43B
:1073500065C27AC48B35910509F425C38C35910536
:1073600009F425C38A35910509F06EC41092CD0841
:107370000C94444B14E03FC280912F02882311F4F7
:107380000C94444B0E9443E10E94B9BE0C94444BC0
:1073900020912F02222311F40C94444B11E0029708
:1073A00009F010E00E9443E119821A821B821C82BC
:1073B0001D821E821F82188682E50E94EA9388231E
:1073C00009F438C10E946A934B015C0120E030E06F
:1073D000A9010F94011E882309F442C180910D1860
:1073E00090910E18A0910F18B09110188CA39DA326
:1073F000AEA3BFA38091111890911218A0911318F9
:10740000B091141888A799A7AAA7BBA78091E313E6
:107410009091E413A091E513B091E6138CA79DA77A
:10742000AEA7BFA78091E7139091E813A091E9134D
:10743000B091EA1388AB99ABAAABBBAB2CA53DA529
:107440004EA55FA56CA17DA18EA19FA10F94011EE9
:1074500081110DC028A939A94AA95BA968A579A5F8
:107460008AA59BA50F94011E882309F4F9C020E08A
:1074700030E0A901C501B4010F94011E881F8827BF
:10748000881F181729F080E090E0A0E8BFEB04C047
:1074900080E090E0A0E8BFE388AF99AFAAAFBBAFB0
:1074A0002CA13DA14EA15FA16CA57DA58EA59FA598
:1074B0000F94F6246CAB7DAB8EAB9FAB28A539A5A2
:1074C0004AA55BA568A979A98AA99BA90F94F62466
:1074D0006B017C012CA93DA94EA95FA9CA01B90184
:1074E0000F94671E2B013C01A7019601C701B6014D
:1074F0000F94671E9B01AC01C301B2010F94F724E6
:107500000F94A5272B013C019B01AC0160E070E0CA
:1075100080E89FE30F94F12521966CAF7DAF8EAF8D
:107520009FAF219720E030E040E05FE3C301B2016C
:107530000F94671E2B013C01A5019401C501B40104
:107540000F94671E4B015C01A3019201C301B201BC
:107550000F94671E9B01AC01C501B4010F94F62482
:107560000F94A52728AD39AD4AAD5BAD0F94671ECA
:107570004B015C01C701B601905821962CAD3DAD81
:107580004EAD5FAD21970F94671EA50194010F9436
:10759000671E6B017C012CA53DA54EA55FA56CA1C6
:1075A0007DA18EA19FA10F94F72420E030E040E060
:1075B0005FE30F94671E9B01AC01C701B6010F94F6
:1075C000F7242CA13DA14EA15FA10F94F62469835D
:1075D0007A838B839C8328A939A94AA95BA968A5CA
:1075E00079A58AA59BA50F94F72420E030E040E020
:1075F0005FE30F94671E6B017C0121962CAD3DADBE
:107600004EAD5FAD21976CA97DA98EA99FA90F945E
:10761000671EA50194010F94671E9B01AC01C70171
:10762000B6010F94F72428A539A54AA55BA50F94A8
:10763000F62412C089E40E94EA93882331F00E9464
:107640006A9369837A838B839C838AE40E94EA939A
:10765000882331F00E946A936D837E838F8398879D
:1076600020E030E0A90169817A818B819C810F94AF
:10767000011E81110BC020E030E0A9016D817E81E7
:107680008F8198850F94011E8823A1F0412FBE01A0
:107690006F5F7F4F83EE93E10E940EB60F94060159
:1076A00060930C1470930D1480930E1490930F1428
:1076B0000C94444B0F94310A8CE797E00F944C09DB
:1076C0000C94444B80E50E94EA93882329F00E94A1
:1076D0001ACD6B017C0103C0C12CD12C760183E54E
:1076E0000E94EA93882361F00E946A9320E030E0D0
:1076F0004AE754E40F94671E0F946A266B017C01DD
:107700000E945F8C8091970B811105C060E082E937
:1077100097E00E94F6ED0F940601C60ED71EE81EF4
:10772000F91E0F940601DC01CB018C199D09AE09ED
:10773000BF09B7FD02C00C94444B80E00E94D653B1
:10774000F0CF0E942BAA0C94444B0E94B77C81116D
:107750000C94444B80E090E0A8E4B2E489839A83DF
:10776000AB83BC8380E090E0A0E2B1E48D839E8394
:10777000AF83B88789879A87AB87BC8780E50E94EB
:10778000EA93882321F00E943293862F01C080E083
:10779000BE016F5F7F4F0E942EED0C94444B809191
:1077A000960B8770873011F00C944F4B60E08FE49C
:1077B0000E94F79381110C94444B0C944F4B809191
:1077C000251881111DC00E9400828823F9F01150F4
:1077D00011F40C94394D40E050E060E078E085E031
:1077E0000E94C69461E083EF97E00E940C948BEDB9
:1077F00097E00E94F1BB0E94B77C882301F306C08A
:1078000060E08FE40E94F7938823E9F20E943094AD
:107810008EE998E00E94F1BB0C94444B2091FF1339
:1078200030910014409101145091021460910D1890
:1078300070910E1880910F18909110180F94F724E2
:10784000AB01BC0188E50E94FCCF6C8F7D8F8E8FD1
:107850009F8F20910314309104144091051450918E
:10786000061460911118709112188091131890915C
:1078700014180F94F724AB01BC0189E50E94FCCFDA
:1078800069837A838B839C83BE016F5F7F4FCE01B8
:107890004C960E941CA6882311F40C94444B80E063
:1078A0000F94C2060E949DC161E085E40E94F79397
:1078B000182F21E0482FBE016F5F7F4FCE014C96FD
:1078C0000E945BFB6B017C019B01AC010F94E927DB
:1078D00081115FC08C8C9D8CAE8CBF8C20E030E021
:1078E000A901C501B4010F94011E87FF05C027E15E
:1078F00037EB41E558EB04C027E137EB41E558E3AE
:10790000C501B4010F94F724AB01BC0180EC98E0F1
:107910000F94000A89809A80AB80BC8020E030E020
:10792000A901C501B4010F94011E87FF05C027E11D
:1079300037EB41E558EB04C027E137EB41E558E36D
:10794000C501B4010F94F724AB01BC018BEB98E0A7
:107950000F94000A20E030E0A901C701B6010F949E
:10796000011E87FF05C027E137EB41E558EB04C056
:1079700027E137EB41E558E3C701B6010F94F7243F
:10798000AB01BC0186EB98E00F94000A8AE00E94EC
:10799000AA520E9484C1113011F40E9471890E9480
:1079A0007DC40C94444B2093CD080C94444B8DED36
:1079B000282E82E0382E93E7E92E92E1F92E2DE071
:1079C00038E13DA32CA323EFC22E23E1D22E00E009
:1079D00010E0D1018D911D010E94EA93882309F4E2
:1079E0004BC00E946A932B013C01133049F0F60111
:1079F00020813181428153810F94F6242B013C0177
:107A0000ACA1BDA12D913D914D915C91C301B201FD
:107A10000F94F6244B015C012DEB37E346E855EB60
:107A20000F94572787FD0AC02DEB37E346E855E34F
:107A3000C501B4010F94011E1816F4F4133051F46B
:107A40004092191850921A1860921B1870921C18C4
:107A500001E012C0A5019401F7016081718182816A
:107A600093810F94F724D7016D937D938D939C930D
:107A70001397812F0E9402BE1F5FB4E0EB0EF11C32
:107A8000ECA1FDA13496FDA3ECA3F4E0CF0ED11C34
:107A9000143009F09ECF002321F089E198E10E9483
:107AA000708C0E947DC40C94444B80912F028823DB
:107AB00011F40C94444B89E40E94EA93082F882324
:107AC00021F00E946693E82E01C0E12C8AE40E9416
:107AD000EA93182F882321F00E946693F82E01C0A4
:107AE000F12C002319F024E02E1528F0112349F081
:107AF00034E03F1530F488EC98E00F944C090C9476
:107B0000444B0E9428930023F1F020915F133091A1
:107B100060134E2D4203B001439F700D11248091DC
:107B2000551390915613680F791F072E000C880B80
:107B3000990B0F94081E6093E3137093E4138093E2
:107B4000E5139093E6131123F1F020916113309126
:107B500062134F2D4203B001439F700D1124809199
:107B6000571390915813680F791F072E000C880B3C
:107B7000990B0F94081E6093E7137093E81380939A
:107B8000E9139093EA1360E080E50E94F79388235D
:107B9000C1F10023D1F02091FF13309100144091E6
:107BA0000114509102146091E3137091E4138091D9
:107BB000E5139091E6130F94F6246093E31370930A
:107BC000E4138093E5139093E6131123D1F02091F1
:107BD00003143091041440910514509106146091DF
:107BE000E7137091E8138091E9139091EA130F94D1
:107BF000F6246093E7137093E8138093E91390934E
:107C0000EA1340E050E0BA0186E40E94FCCF6B0129
:107C10007C0120E030E0A9010F945727181684F466
:107C200020E030E040E752E4C701B6010F94F125AF
:107C3000609363027093640280936502909366027E
:107C40000E94B9BE0C94444B0E94717C0C94444B2E
:107C500080916412909165128537910509F49AC755
:107C60000CF053C18934910509F479C40CF06CC04F
:107C70008A31910509F4FEC2B4F58431910509F405
:107C800073C294F48131910509F44DC244F4029712
:107C900010F00C94384B0E94D4B90C94444B42978A
:107CA00009F4A6C60C94384B8731910509F486C2B5
:107CB0008CF48531910509F47DC2469711F00C943E
:107CC000384B0E94D75D80919817877F80939817D3
:107CD0000C94444B8831910509F488C2499709F402
:107CE000BEC20C94384B8F31910509F4F1C37CF47A
:107CF0008C31910509F436C30CF4CAC28D3191055B
:107D000009F43AC34E9709F43EC30C94384B8A32B7
:107D1000910509F4FDC364F48032910509F492C31E
:107D2000819711F00C94384B0E946BD60C94444B05
:107D30008B32910509F40FC4C09711F00C94384BA5
:107D40000E94667D0C94444B8836910509F4B0C4BA
:107D5000D4F58135910509F433C6C4F48C3491050A
:107D600009F40CC44CF48B34910511F00C94384B8D
:107D70000E945A8A0C94444B8D34910509F402C434
:107D80008E34910509F402C40C94384B8435910566
:107D900009F42EC674F48235910509F426C683359C
:107DA000910511F00C94384B81E08093C7080C9436
:107DB000444B8535910509F447C68C35910509F486
:107DC0005CC60C94384B8E36910509F4EBC4D4F4A0
:107DD0008B36910509F4E4C554F48936910509F40C
:107DE0007DC58A36910509F4B3C50C94384B8C36A1
:107DF000910511F40C94444B8D36910509F47BC424
:107E00000C94384B8137910509F422C55CF48F3608
:107E1000910509F4D8C48037910511F40C94444BB2
:107E20000C94384B8237910509F4B1C6833791051C
:107E300011F00C94384B8AE49BE00F944C0960E0FD
:107E40008AE39BE00E9465BA60E085E29BE00E94C5
:107E500065BA61E08EE19BE00E9465BA61E083E172
:107E60009BE00E9465BA61E083E09BE00E9465BAF6
:107E700060E08AEF9AE00E9465BA61E080EF9AE0E4
:107E80000E9465BA61E086EE9AE00E9465BA61E000
:107E90008EED9AE00E9465BA61E080ED9AE00E9462
:107EA00065BA61E082EC9AE00E9465BA60E083EB1B
:107EB0009AE00E9465BA60E085EA9AE00E9465BA9D
:107EC00060E08FE89AE00E9465BA61E08EE79AE090
:107ED0000E9465BA61E08FE69AE00E9465BA61E0AF
:107EE0008AE59AE00E9465BA61E087E49AE00E9420
:107EF00065BA60E08AE39AE00E9465BA60E086E2D3
:107F00009AE00E9465BA0C94444B8E32A1E09A0725
:107F100011F40C9426490CF06FC08B3C910509F4C8
:107F2000FFC6ACF58D37910509F447C5BCF487371A
:107F3000910509F47AC60CF43EC68837910509F418
:107F400077C68937910511F00C94384B10928D0942
:107F500010928C090E94F2C50C94444B8E3B910503
:107F600009F4AAC454F48C38910509F493C48B39EC
:107F7000910509F4C7C40C94384B883C910509F469
:107F80005FC6893C910509F4A8C60C94384B8C3D1A
:107F9000910509F417C79CF48D3C910509F4E2C6DC
:107FA0000CF4DDC68E3C910509F4EAC6833D9105CB
:107FB00011F00C94384B0E94F0E30C94444B883140
:107FC000E1E09E0709F4ADC754F48D3D910509F435
:107FD00006C7823E910509F458C70C94384B82328B
:107FE00021E0920711F40C9428488D32914011F44D
:107FF0000C9433480C94384B843F41E0940711F4BF
:108000000C94864A0CF043C08239B1E09B0711F40E
:108010000C947049DCF48033F1E09F0711F40C9468
:10802000B34814F40C946A49803931E0930711F491
:108030000C946D498139914011F00C94384B81E0DA
:108040000E94B9890E947DC40C94444B843AA1E0FB
:108050009A0711F40C9483496CF48A39E1E09E0785
:1080600011F40C94444B8C39914011F40C947849E0
:108070000C94384B853A21E0920711F40C94864910
:108080008C3A914011F40C94F6490C94384B883595
:1080900042E0940711F40C94AE4A1CF5873FB1E01E
:1080A0009B0711F40C948C4A7CF4853FF1E09F0708
:1080B00011F40C94894A863F914011F00C94384B8E
:1080C0000E9485F50C94444B883F31E0930711F4EE
:1080D0000C94954A8C30924011F40C94A64A0C945E
:1080E000384B8C36A3E09A0711F40C94444B7CF483
:1080F0008B35E2E09E0711F40C94B14A833593402E
:1081000011F00C94384B0E94EAB30C94444B803A23
:1081100023E0920709F4CCC1873E934011F40C94FC
:108120002A4B0C94384B8091601284FF02C00C944F
:108130004B4D8091621287FF02C00C944B4D809191
:108140006312837011F00C944B4D60E087EE98E061
:108150000E94F6ED5F988A98809108018170809363
:10816000060112980C94444B8FEF98E00F944C0941
:108170001092910B8CE095E10E947D668BE1ECE022
:10818000F5E1DE01119601900D928A95E1F740E04C
:1081900050E0BE016F5F7F4F80E090E00E945D5F26
:1081A000CE0101960E94B36780EF98E00F944C09CE
:1081B0000C94444B0E94485E0C94444BE0911C1379
:1081C000F0911D138081882329F0803209F41082F8
:1081D0003196F8CF40E061E080911C1390911D131F
:1081E0000E943361109247130C94444B8091230BEF
:1081F0008823E9F080E090E0A0EAB1E488A399A3A5
:10820000AAA3BBA31C8E1D8E1E8E1F8E19821A82DE
:108210001B821C8220E0AE01405E5F4FBE01645EA7
:108220007F4FCE0101960E9486950C94444B0E948C
:1082300048D7882321F00E94E85D0E945A8A40E0D6
:1082400050E060E179E085E00E947F9561E082E0A6
:1082500094E30E940C940E947AEE0C94444B80911B
:10826000981782FF03C08B7F809398170E9422E3A8
:108270000C94444B8091981783FD02C00C94444B9E
:1082800083E50E94EA9381110C94674D0C94444B52
:1082900083E40E94A1938823D9F184E299E00F94AA
:1082A0004C098091B614882351F1BE016F5F7F4F56
:1082B00083EB94E10E9444658E010F5F1F4FD8014C
:1082C0008D918D01882319F00E94AA52F8CFBE012A
:1082D0006F5F7F4F80E090E00E94FB608091351AD5
:1082E000882389F080E20E94AA5205E31AE1F8018E
:1082F00081918F01882339F00E94AA52F8CF8AE138
:1083000099E00F944C098AE00E94AA520C94444BC5
:1083100083E50E94EA93882309F10E944293182F73
:1083200090E0CD970CF01CE31093BE080F9406016B
:108330006B017C01212F30E0A8EEB3E00F94AB2459
:10834000C60ED71EE81EF91EC092BA08D092BB080E
:10835000E092BC08F092BD080C94444B0E94B05DC2
:108360000C94444B40E060E080911C1390911D13ED
:108370000E9433610C94444B809198178E7F8093B8
:1083800098170C94444B8091981783FD02C00C946D
:10839000444B0E9440FD8091981783FD02C00C94CD
:1083A000444B60911C1370911D13CE014C960F9499
:1083B0008D038C01009711F40C94444B6C8D7D8DD2
:1083C00019821C8222E0AC01CE0101960E94966BBC
:1083D000811102C0F12C14C0CE0101960F94FB0252
:1083E0008823C1F361E0CE0101960E9428650097C1
:1083F00089F325EEDC012C931C820E943767F82E4E
:10840000CE0101960E94B367B801FF2089F08EE487
:1084100099E00F941E0A8AE00E94AA5210929417C3
:108420001092951710929617109297170C94444B30
:1084300086E399E00F941E0A83E399E00F944C09B8
:108440000C94444B8091981782FD0E945F8C809120
:10845000981783FD02C00C94444B60E080E50E94B5
:10846000F793182F482F61E080911C1390911D13F2
:108470000E94336183E50E94EA93882381F00E9481
:108480003293AB01BC0140939417509395176093BE
:1084900096177093971783EB94E10E943E640E94B5
:1084A000E85D11110C94444B0E945A8A0C94444B81
:1084B00020911C1330911D13909198179260909306
:1084C000981740E060E0C9010E9433610C94444B6E
:1084D0000E94A6EC6C8F7D8F8E8F9F8FBE016F5F89
:1084E0007F4FCE014C960E948FD560E0CE01019661
:1084F0000E9451EE0F94350ABE016F5F7F4F8CE5ED
:1085000099E00F941E0A8AE00E94AA520C94444BF0
:1085100083E50E94EA93882311F40C94444B0E9453
:108520004293F82E6DE070E080E50E9451A78C0127
:1085300097FF02C00C94444BE82E60E089E40E944F
:10854000F79381110C94784D802F0E941B5081115C
:10855000B9C40C94784D0E94E0E40C94444B80E53F
:108560000E94A193882311F40C94444B8091981796
:1085700082FF02C00C94444B0C94914D0E94F5EC88
:108580000C94444B0E940A8B0C94444B60E070E0C6
:1085900083E50E9451A78E34910531F40E94C58B6A
:1085A0000E947AEE0C94444B87EC99E00F944C09AE
:1085B00060917C0970917D098EEB99E00F94F3092D
:1085C00060917E0970917F0981EB99E00F94F30926
:1085D00060917C0970917D0980917E0990917F095D
:1085E000681B790B80911811815021E030E08230B6
:1085F00010F020E030E0621B730B86EA99E00F94E4
:10860000F3098AE00E94AA528EE999E00F944C097E
:108610008091800990918109A0918209B09183098C
:108620008C8F9D8FAE8FBF8FBE016F5F7F4FCE014E
:108630004C960E948FD5BE016F5F7F4F81E999E014
:108640000F941E0A8091840990918509A091860952
:10865000B09187098C8F9D8FAE8FBF8FBE016F5FEA
:108660007F4FCE014C960E948FD5BE016F5F7F4F2A
:1086700081E899E00F941E0A20E030E04AE754E4D4
:10868000609188097091890980918A0990918B097C
:108690000F94F125AB01BC0189E699E00F94000A23
:1086A0008DE60E94AA528AE00E94AA520C94444B82
:1086B0008091A31083FF02C00C94444B0E94F2E10E
:1086C00087FF02C00C94444B83E50E94EA93882301
:1086D00079F00E946A930F9463268B01CB010E946C
:1086E000B0DF0135110524F40E940A8B0E947AEE56
:1086F0000F947117C9C78091A31083FDC5C70E944D
:10870000F2E1F82E87FDC0C783E50E94EA93082FA7
:10871000811106C082E50E94EA93182F8823C1F1D7
:108720000E946A930F946326CB010E94B0DF0E94DF
:108730006A9320E030E040EA52E40F94011E1816DC
:1087400014F40C949C4D0E940A8B0E947AEE609166
:10875000120C7091130C072E000C880B990B0F94C0
:10876000081E4B015C0140900E0C50900F0C609065
:10877000100C7090110CA30192010F94572718163A
:1087800014F40C94AF4D002311F40C94A04D11E09F
:108790000F947117112309F477C7602F8F2D0E9452
:1087A000BCD972C78EE40E94EA93882309F46CC78F
:1087B0000E943293609318137093191380931A13C5
:1087C00090931B1361C783E50E94A193882331F026
:1087D00060E083E50E9460A78093A3100F94350AA0
:1087E00087EF99E00F944C098091A310882369F1D9
:1087F0000DEEE02E09E0F02E00E010E020E0809188
:10880000A31090E0A0E0B0E0002E04C0B695A795BC
:10881000979587950A94D2F780FF0EC0DD24D394F4
:10882000D20E222319F08CE20E94AA52F701859100
:1088300094910F944C092D2D0F5F1F4FB2E0EB0E5A
:10884000F11C05301105D9F65ECD89EE99E059CDC0
:1088500083E50E94EA93882371F00E944293282FB7
:1088600030E02D3331051CF4809300020DC78CE3FA
:108870008093000209C70F94350A4091000250E02E
:1088800060E070E08EEF99E00F94E2098AE00E94C8
:10889000AA52FAC68091A31083FDF6C683E50E9412
:1088A000EA93882309F4F0C60E946A930F94632622
:1088B000CB010E941A93E8C68091A31083FDE4C601
:1088C00083E50E94EA93182F81110C94B24D82E542
:1088D0000E94EA9381110C94B24DD6C60E94F2E137
:1088E000182F87FD0AC083E29AE00F944C09812F6C
:1088F0000E94CCD78AE00E94AA52ECADE0934512C8
:108900000C94384F83E50E94EA93882309F4BCC68F
:108910000E944293182F90E0CD970CF01CE3109327
:10892000C3080F9406016B017C01212F30E0A8EEF3
:10893000B3E00F94AB24C60ED71EE81EF91EC092FA
:10894000BF08D092C008E092C108F092C2089CC64D
:1089500060E080E50E9460A7F82EF1E0F81708F4C7
:1089600093C681E40E94A193882321F06091F70BC4
:10897000062F02C00FEF10E083E50E94EA938823E0
:1089800049F00E9432938B016F3F710519F010F08E
:108990000FEF10E0EF2DF0E0E950F44F008374C6C4
:1089A00060E080E50E9460A7823008F06DC6E82F85
:1089B000F0E0E950F44F108267C60E9422E364C6DB
:1089C0000E94C1DF0E940A8B0E94A08D0E945D5010
:1089D0001092DB0B1092DA0B1092D90B68EE73E059
:1089E00080E090E00F941D094FC61092C7084CC656
:1089F00083E50E94EA93882399F00E946A9320E01D
:108A000030E04AE754E40F94671E0F946A2660939F
:108A1000010270930202809303029093040234C611
:108A20008091601284FF02C00C94E74D8091621225
:108A300087FF02C00C94E74D80916312837011F0A0
:108A40000C94E74D0C94184E83E50E94A193882363
:108A500009F41AC60E946A9320E030E04AE754E421
:108A60000F94671E0F946A266093C8087093C90814
:108A70008093CA089093CB0807C60E94F2E187FD55
:108A800003C69091601294FD04C09091621297FF0A
:108A90000AC0BDEDCB2EB2E0DB2E14EAE12E10E1D0
:108AA000F12E10E009C090916312937091F7682F36
:108AB00081E00E94A5E4E8C5D6018D916D010E9478
:108AC000EA93882309F459C0133009F04FC00E947B
:108AD0006A934B015C0120E030E040EA51E40F94DE
:108AE000011E87FF3AC0A50194016091C4107091E6
:108AF000C5108091C6109091C7100F94F1252B01DD
:108B00003C019B01AC016091D4107091D510809113
:108B1000D6109091D7100F94671E6093D410709365
:108B2000D5108093D6109093D7106091EF0B709171
:108B3000F00B8091F10B9091F20B0F94061EA301A4
:108B400092010F94671E0F946A266093EF0B709347
:108B5000F00B8093F10B9093F20B8092C4109092E3
:108B6000C510A092C610B092C71007C00E946A93A9
:108B7000F701648B758B868B978B1F5FF4E0EF0E8C
:108B8000F11C143009F098CF0E943B8C7DC50E94E7
:108B90007FBA7AC580911C1390911D13009741F004
:108BA000DC012C91222321F060E00E9451EE6CC583
:108BB0000E947AEE69C500911C1310911D1394E078
:108BC000F12C40E0915021F1F8018081282F2B7F7A
:108BD000213421F421812133D9F407C08035C1F437
:108BE000818180538A3048F013C0813421F085346C
:108BF00021F441E002C0FF24F39498012E5F3F4F1F
:108C000089012F5F3F4FF80180818032C9F3DACFAD
:108C100041110F94350AFF2021F081E39CE00F946D
:108C20004C09C8010E94B5532FC50E949BC52CC595
:108C300081E080938D0980938C090E94F2C524C540
:108C40000E94F2E1182F87FD1FC584E40E94A193C2
:108C5000882309F43FC00E946A936B017C0101E004
:108C600020E030E0A9010F94011E811101C000E055
:108C70000093FD1020E030E0A901C701B6010F9478
:108C8000011E882339F10E946A9324E01202F00148
:108C90001124EE5FFE4E608371838283938320E014
:108CA00030E0A901609102117091031180910411CB
:108CB000909105110F94011E81110CC080E090E08D
:108CC000A0EEBFE38093021190930311A0930411CF
:108CD000B09305110E94CA8ED7C40E94F2E187FDAD
:108CE000D3C4ADEDEA2EA2E0FA2E04EA10E1D701DA
:108CF0008D917D010E94A193882349F00E946A937F
:108D00000F946A26F80160837183828393830C5FDA
:108D10001F4FF0E1043B1F0751F70E94F48BB4C4CE
:108D20000E94F2E187FDB0C4FDEDEF2EF2E0FF2ED0
:108D300004EA10E1D7018D917D010E94A19388235F
:108D400039F00E946A93F80164A375A386A397A3E0
:108D50000C5F1F4FF0E1043B1F0761F795C40E94B1
:108D6000A4CC92C48091601281FD65C7809161128C
:108D700081FD61C7809162128C7009F05CC784C468
:108D80007DEDC72E72E0D72EE0E9EE2EE9E0FE2E53
:108D900010E0D6018D916D010E94A193882351F0BE
:108DA0000E946A93F7016083718382839383812F8A
:108DB0000E9402BE1F5FF4E0EF0EF11C133049F772
:108DC0000C94513D83E50E94EA93882309F45CC426
:108DD0000E94669390934F0280934E0255C40E9466
:108DE000F2E1F82E87FD50C483E50E94EA930F2D2F
:108DF0000F2C000C110B882369F10E946693F80177
:108E0000EE0FFF1FE55EFD4F91838083000F111F62
:108E1000000F111F98012B5E3D4F7901BC01990F86
:108E2000880B990B0F94081E2AE037ED43E25CE3B0
:108E30000F94671EF801E250FF4E2081318142817C
:108E400053810F94671ED7016D937D938D939C93EF
:108E500013971AC40F94350A85E40E94AA5280E33E
:108E60008F0D0E94AA52000F111FF801E55EFD4F01
:108E70006081718184E59CE00F94110A85E20E9473
:108E8000AA528AE00E94AA52FFC380E50E94A193E1
:108E9000882309F4F9C360E070E080E50E9451A7DF
:108EA000F82E6FEF7FEF83E50E9451A78C010196AA
:108EB000039708F0E9C3F7FCE7C38F2D0E941B500E
:108EC000882339F00F94310A8CE59CE00F944C090B
:108ED000DBC30E945F8C60E08F2D0E94A8FF0F3FD4
:108EE000BFEF1B0731F00130110571F000E010E019
:108EF0000DC08F2D0E9450FF31E020E0892B09F03A
:108F000030E0032F122F02C001E010E08F2D0E94ED
:108F100050FF8017910709F4B7C380E00E94D65331
:108F2000F5CF80E50E94A193882309F4ADC30E9488
:108F300066938C01892B09F07FC083E50E94A19381
:108F4000882389F00E9466938F3FEFEF9E0729F4F4
:108F500084E995E10E94625097C3BC0184E995E1E0
:108F60000E94325191C30F94350A60E070E084E8AA
:108F70009CE00F94110A8091961528E532E0690172
:108F8000C81AD10887FDD394CC0CDD1CCC0CDD1C99
:108F90000D2C000CEE08FF088091951528E830E0B4
:108FA0004901881A910887FD9394880C991C880CB4
:108FB000991C092C000CAA08BB08809194158F3FBE
:108FC000C1F090E0FC01EE0FFF1F8E0F9F1FFC0110
:108FD000E95DFA4E2181328183E0220F331F8A95A9
:108FE000E1F794E0369527959A95E1F72E5F3F4F8C
:108FF00002C020E030E02F5F3F4FC901330FAA0BC2
:10900000BB0B9C01AD01281939094A095B09A4EB86
:10901000B0E00F949824A7019601281939094A094C
:109020005B090F947924B90181E89CE00F94110A3F
:109030008AE00E94AA5228C30F94310AB8018AE735
:109040009CE00F94110A8BE69CE00F944C091CC322
:109050008AE50E94EA93811147C683E50E94EA935C
:10906000811142C611C360E085E40E9460A78111AE
:1090700073C080E50E94A193882351F00E946A93F7
:109080006093150C7093160C8093170C9093180C2A
:1090900089E40E94A193882381F00E946A932CEABC
:1090A00035EC47E25EE30F94671E6093190C7093F2
:1090B0001A0C80931B0C90931C0C84E40E94A193C7
:1090C000882381F00E946A932CEA35EC47E25EE344
:1090D0000F94F12560931D0C70931E0C80931F0C50
:1090E0009093200C0F94350A4091150C5091160C5A
:1090F0006091170C7091180C87EB9CE00F94000A9C
:109100002CEA35EC47E25EE36091190C70911A0C81
:1091100080911B0C90911C0C0F94F125AB01BC01AC
:1091200083EB9CE00F94000A2CEA35EC47E25EE307
:1091300060911D0C70911E0C80911F0C9091200C61
:109140000F94671EAB01BC018FEA9CE00F94000AEC
:109150008AE00E94AA5298C20F94310A8DE99CE0DD
:109160000F944C0991C280E50E94A193882351F08D
:109170000E946A9360936C0970936D0980936E09E5
:1091800090936F0989E40E94A193882381F00E9443
:109190006A932CEA35EC47E25EE30F94671E609316
:1091A000700970937109809372099093730984E434
:1091B0000E94A193882381F00E946A932CEA35ECE7
:1091C00047E25EE30F94F12560937409709375098B
:1091D00080937609909377090F94350A40916C0932
:1091E00050916D0960916E0970916F0983EC9CE05C
:1091F0000F94000A2CEA35EC47E25EE360917009B7
:109200007091710980917209909173090F94F12501
:10921000AB01BC018FEB9CE00F94000A2CEA35EC0B
:1092200047E25EE360917409709175098091760957
:10923000909177090F94671EAB01BC018BEB9CE00A
:109240000F94000A8AE00E94AA521EC283E50E947F
:10925000A193182F882371F00E946A930F946326BC
:1092600070931A026093190221E0672B09F020E045
:109270002093090C80E50E94A193882359F0209146
:10928000190230911A02232B11F00E9456938093F9
:10929000090CFAC11111F8C10F94350A83EE9CE054
:1092A0000F944C098091090C882319F08BEC9CE0F9
:1092B00002C087EC9CE00F944C09609119027091F8
:1092C0001A0282ED9CE00F94110A8EEC9CE00F9440
:1092D0004C09DAC10E9413D0D7C10E945F8CD4C15F
:1092E00080E00E94B9890E9471890E947DC4CCC12E
:1092F00080916012887809F080C580916212867032
:1093000009F07BC556C50E946CA7BEC16FEF7FEF09
:1093100089E40E9451A7F82E6FEF7FEF8AE40E9444
:1093200051A7E82E8AE50E94A193182F811105C04C
:1093300081E50E94A193B82E01C0B12CF7FC06C0B4
:10934000E7FC04C0111109C0B11007C00F94310A25
:109350008DE49DE00F944C0997C1F4E0FF1510F0E7
:10936000FE1538F40F94310A8EE29DE00F944C09FB
:109370008BC1CF2C0F2C000CDD080E2D0E2C000CF9
:10938000110B0E946A93BB2099F025E02C9DF001FF
:109390002D9DF00D1124E00FF11FEE0FFF1FEE0FBA
:1093A000FF1FE559FC4E208131814281538103C06A
:1093B00020E030E0A9010F94F7249B01AC0185E087
:1093C0008C9DF0018D9DF00D1124E00FF11FEE0F2B
:1093D000FF1FEE0FFF1FE559FC4E208331834283B0
:1093E00053836E2D8F2D0E94CECE4EC10E94B77C2E
:1093F00081114AC10EE115E22DE038E13DA32CA315
:10940000CE0101965C0143E7842E45E2942E1C01B7
:10941000F8016591759185919491ACA1BDA1CD9014
:10942000DD90ED90FD90BDA3ACA3A70196010F9434
:10943000F6242B013C01F1016083718382839383C5
:1094400020E030E040EA51EC0F94572787FD0AC036
:1094500020E030E040EA51E4C301B2010F94011E64
:1094600018162CF4F401849118160CF4F6C4D101EA
:10947000CD90DD90ED90FD901D0120E030E040EAC0
:1094800051ECC701B6010F94572787FD0AC020E0B1
:1094900030E040EA51E4C701B6010F94011E1816EE
:1094A00064F40F94310A8BE89DE00F944C0961E05D
:1094B0008DE79DE00E94F6EDE7C00C5F1F4FBFEF08
:1094C0008B1A9B0AE5E20A321E0709F0A1CF30E9A8
:1094D000E32E39E0F32E10E0F50181919191A191F5
:1094E000B1915F01F70181939193A193B1937F01B2
:1094F000812F0E9402BE1F5F133071F70E947DC44E
:1095000060E08DE69DE00E94F6EDBEC00E94D1E7CE
:10951000BBC00E94D3F9B8C061E083E50E94F79315
:1095200091E089270E94CAF6AFC081E080935A1368
:109530000E94EFEE10925A13882309F4A5C00F94ED
:10954000350A89EA9DE00F944C099EC080919817D6
:1095500082FF9AC080628093981796C00E941BE297
:1095600093C00E94F2E1082F87FD8EC085E50E941E
:10957000A1938823B1F1E02E002E000CFF080E9479
:109580006A934B015C0120E030E0A9010F9457275A
:1095900087FF04C0B7FAB094B7F8B094C70123E0CE
:1095A000880F991F2A95E1F79C012D593C4E7901AE
:1095B000D9018D929D92AD92BC92139720E030E03C
:1095C0004AEF53E4C501B4010F94572718164CF421
:1095D00080E090E0AAEFB3E4F70180839183A28357
:1095E000B3838CE40E94A193882309F44DC0002E1C
:1095F000000C110B0E946A936B017C0120E030E0AB
:10960000A9010F94572787FF04C0F7FAF094F7F8E1
:10961000F09420E030E04AEF53E4C701B6010F9424
:109620005727980193E0220F331F9A95E1F7F9012C
:10963000ED59FC4E18162CF0C482D582E682F782D2
:1096400023C080E090E0AAEFB3E484839583A683EF
:10965000B7831AC081E080932F021092D70B60E08D
:1096600083E50E94F79381110FC00E9456D70CC06A
:109670000E94717C09C080916412882329F00E94A5
:10968000876C02C00E94717C2296FFAD2297F11177
:1096900002C00E94F3B22CAD20934512E9C30E9490
:1096A0005F8C309125183CAB80E00F94C2060E947D
:1096B0009DC181E080938D090E94F2C588E50E94DA
:1096C000A193182F89E50E94A193082F8AE50E9493
:1096D000A1931013C0C1181711F0012FBCC101E0F4
:1096E00011E091E09CA70E94289382E50E94EA93F2
:1096F000882361F00E946A936B017C0120E030E0D6
:10970000A9010F94011E882369F106C0C12CD12C38
:1097100030E8E32E30E4F32E111103C0002309F4E6
:10972000FCC0C092EB13D092EC13E092ED13F092D8
:10973000EE13A7019601609115187091161880918B
:109740001718909118180F94011E87FF0BC01982EB
:109750001A821B821C82BE016F5F7F4F8BEE93E1EA
:109760000E949FC2112309F4D3C0002309F4CDC085
:1097700010921118109212181092131810921418B7
:1097800010920D1810920E1810920F1810921018B7
:109790000E9448C3E3E7F5E2A491A8AFE7E6F5E24B
:1097A000C590D590E590F490EBE6F5E28590959024
:1097B000A590B490A5019401C701B6010F94572755
:1097C00018162CF4A7019601C501B40104C0A50127
:1097D0009401C701B6010F94F1252B013C01EEE283
:1097E000F5E285919591A591B4918CA39DA3AEA32B
:1097F000BFA3EAE2F5E285919591A591B49188A77E
:1098000099A7AAA7BBA79C01AD016CA17DA18EA1C0
:109810009FA10F945727181634F428A439A49AA5A9
:1098200098AB1BA505C02CA03DA0AEA1A8AB1FA165
:10983000A3019201C301B2010F94671E20E030E042
:1098400040E85FE30F94F7240F94A527910148A9FE
:10985000512F0F94671E68A379A38AA39BA3E4E703
:10986000F5E2149120E030E040EC5FE3C501B40183
:109870000F94671E4B015C01612F110F770B880B52
:10988000990B0F94081E9B01AC01C501B4010F9404
:10989000671E69837A838B839C8320E030E040ECF1
:1098A0005FE3C701B6010F94671E6B017C01B8AD81
:1098B0006B2FBB0F770B880B990B0F94081E9B0126
:1098C000AC01C701B6010F94671E6C8F7D8F8E8F20
:1098D0009F8FAE01405E5F4FBE016F5F7F4FCE0135
:1098E0004C960E947DC20E947AF510921118109237
:1098F0001218109213181092141810920D1810923A
:109900000E1810920F181092101880E00E944AC38F
:10991000002319F081E00E944AC3ECA5EE2309F46C
:109920008CC080E00E942199809114148370833050
:1099300051F060E08DEC97E00E94F6ED0F94350A4F
:109940008EEB97E093C00E9448C3809115189091C8
:109950001618A0911718B09118188093EB139093D4
:10996000EC13A093ED13B093EE132091FF133091FD
:109970000014409101145091021460E070E080EAFC
:1099800092E40F94F6246B017C016093E3137093CF
:10999000E4138093E5139093E61320910314309120
:1099A0000414409105145091061460E070E080EAC0
:1099B00092E40F94F6244B015C016093E7137093DB
:1099C000E8138093E9139093EA1327E137EB41ED15
:1099D00058EB0F94572787FD40C023E030E041EE5D
:1099E00053E4C501B4010F94011E1816B4F127E128
:1099F00037EB41ED58EBC701B6010F94572787FDB0
:109A00002CC023E030E84DEE53E4C701B6010F94BB
:109A1000011E181614F119821A821B821C82AE01D3
:109A20004F5F5F4F67EE73E183EE93E10E947DC26B
:109A300082E00E944AC30E9471890E9448C38091BB
:109A40008C0980938D098CA90F94C2060E9484C151
:109A50000E947DC419CE8CA746CE60E08DEA97E0C7
:109A60000E94F6ED0F94350A8BE997E00F944C09AC
:109A7000E2CF61E081E998E00E940C948CE198E0EB
:109A80000E94F1BB61E084EE93E30E940C948DE0B0
:109A900098E00F94260288E50E94A19381115F98B7
:109AA00089E50E94A19381118A988AE50E94A19379
:109AB000882329F08091080181708093060185E454
:109AC0000E94A193882309F4DFCD1298DDCD0E9476
:109AD0003293AB01BC014093941750939517609358
:109AE00096177093971783EB94E10E943E64CCCD58
:109AF00061E0802F0E94A8FF6F2D802F0E9479FFC8
:109B00006F2D70E0802F0E94E4FF47E0E41203C055
:109B1000F092F80BB9CD89E0E812B6CDF092F70BD0
:109B2000B3CD0E94429390E08536910514F084E60F
:109B300090E080934713A8CD0E945A8A0C94A743C3
:109B4000A3019201C501B4010F94572718163CF0E8
:109B50008FEC99E060E00E94F6ED0C94C7438CED29
:109B600099E0F8CF0E946A930F946326CB010E947C
:109B70001A930E946A9320E030E040EA50E40F9488
:109B80005727181614F40E945A8A60916909709137
:109B90006A09072E000C880B990B0F94081E209160
:109BA00065093091660940916709509168090F94E1
:109BB000572718161CF484E19AE002C085E09AE069
:109BC00060E00E94F6ED812F0E943ED85DCD0E949C
:109BD0005F8C88E50E94A193882331F05F9A809181
:109BE00014148E7F8093141489E50E94A193882316
:109BF00031F08A9A809114148D7F809314148AE531
:109C00000E94A193882359F080910801809581706A
:109C100080930601809114148B7F8093141485E443
:109C20000E94A193882309F42FCD0E9419502CCDB6
:109C30000E94A08D29CD82E40E94A193882351F037
:109C40000E941ACD6093B4107093B5108093B61033
:109C50009093B71083E50E94A193882351F00E944E
:109C60006A936093E4107093E5108093E6109093EC
:109C7000E71084E50E94A193882351F00E946A9323
:109C80006093E8107093E9108093EA109093EB10C2
:109C90008AE40E94A193882309F4F6CC0E946A9377
:109CA0006B017C012AE037ED43E25CE30F94572718
:109CB00087FD13C02AE939E949E95EE3C701B60126
:109CC0000F94011E18164CF0C092DF0BD092E00BDF
:109CD000E092E10BF092E20BD7CC0F94310A85E3CE
:109CE0009CE00F944C09D0CC0E946A9320E030E0B5
:109CF00040E050EC0F94011E87FD15C00E946A934E
:109D000020E030E040E050E40F94572718162CF084
:109D10000E946A936B017C010BC0C12CD12CE12CF9
:109D200010E4F12E05C0C12CD12CE12CB0ECFB2E9F
:109D30002091C0103091C1104091C2105091C310B9
:109D4000C701B6010F94671E0F946326CB010F94D1
:109D5000750480E50E94A193882329F00E94569300
:109D6000882309F491CCA7019601609107147091A2
:109D700008148091091490910A140F94F7246093A9
:109D80000714709308148093091490930A140F9485
:109D9000350A40910714509108146091091470918C
:109DA0000A148CE89CE00F94000A8AE00E94AA52F0
:109DB0006BCC0F94350A8DE19DE00F944C09809196
:109DC0002A02811117C086EF9CE00F944C098AE0AB
:109DD0000E94AA5240915B0250915C0260915D0228
:109DE00070915E028DEF9CE00F94000A8AE00E9461
:109DF000AA524ACC8AEF9CE0E8CF88E40E94A19363
:109E0000882321F00E9456938093CC0882E50E941B
:109E1000A193082F83E50E94A193182F011102C07E
:109E2000882351F010925F090E944050112321F0C5
:109E30000E94569380932A0284E40E94A19388236F
:109E400009F422CC0E946A9360935B0270935C02D7
:109E500080935D0290935E0217CCF7FAF094F7F8C6
:109E6000F094D101CD92DD92ED92FC921397FFCA4E
:109E7000CF5BDF4F0FB6F894DEBF0FBECDBFDF91D3
:109E8000CF911F910F91FF90EF90DF90CF90BF90F7
:109E9000AF909F908F907F906F905F904F903F908A
:109EA0002F900895CF92DF92EF92FF920F931F931E
:109EB000CF93DF936C018B017A01EC01CD52D74F28
:109EC000888187FF04C0FB011182108224C02CE02E
:109ED0002C9DC0012D9D900D11242881AC01420FB5
:109EE000511D27FD5A952091931530E042175307D5
:109EF00094F42881AC01420F511D27FD5A959A0117
:109F0000FA01EE0FFF1F2E0F3F1FF901E95DFA4E18
:109F1000208127FD19C088818F5F88832CE02C9DCC
:109F2000C0012D9D900D11242881AC01420F511DBF
:109F300027FD5A952091931530E042175307BCF442
:109F400028812C3044F113C02881820F911D27FDF8
:109F50009A95FC01EE0FFF1F8E0F9F1FFC01E95D1C
:109F6000FA4E808160E08F770E9479FFD4CFF801AC
:109F700080819181049680349C4918F480E49CE9A6
:109F800004C0F801808191810496F7019183808358
:109F90008FEF888345C0F801408151812881BC0141
:109FA000620F711D27FD7A959B01FB01EE0FFF1FCC
:109FB0002E0F3F1FF901E95DFA4E21813281240FF6
:109FC000351FF701318320832881AC01420F511DD9
:109FD00027FD5A959A01FA01EE0FFF1F2E0F3F1F22
:109FE000F901E95DFA4E208127FF1AC02881820F0E
:109FF000911D27FD9A95FC01EE0FFF1F8E0F9F1FED
:10A00000FC01E95DFA4E808161E08F77DF91CF91AD
:10A010001F910F91FF90EF90DF90CF900C9479FFFC
:10A02000DF91CF911F910F91FF90EF90DF90CF9034
:10A030000895129A0895FF920F931F93CF93DF9381
:10A040001F92CDB7DEB7F82E0EEC1DE041E050E0D8
:10A05000B801CE0101960F943B1D89818F1102C07A
:10A0600081E007C00F5F1F4F8DE0073E180771F7B3
:10A0700080E00F90DF91CF911F910F91FF90089595
:10A0800080915B0290915C02A0915D02B0915E02B2
:10A090008093321190933311A0933411B093351102
:10A0A00008958091D608811107C00E94D3F98823B2
:10A0B00019F081E08093D6080895E7EFFBE0108265
:10A0C00011820895DC01EC91F0E0CF01880F991F17
:10A0D000E80FF91FE95DFA4E80818F77808308953C
:10A0E0008F929F92AF92BF92CF92DF92EF92FF92A8
:10A0F0000F93CF93DF931F92CDB7DEB75C016B0157
:10A100007A014901F501808191810F94312489837D
:10A11000002311F0F6018083BE016F5F7F4FC40101
:10A120000F941701F50180819181019691838083BD
:10A13000FFEFCF1ADF0A81E0E81AF10819F780E093
:10A140000F90DF91CF910F91FF90EF90DF90CF9024
:10A15000BF90AF909F908F9008957F928F929F9223
:10A16000AF92BF92CF92DF92EF92FF920F931F9325
:10A17000CF93DF931F92CDB7DEB77C0159018B01DE
:10A180006B01C40ED51E0C151D0559F1F701808019
:10A190009180F80171908F017982C4010F9431246C
:10A1A000781691F0672DC4010F943924C4010F94DF
:10A1B00031249981891741F00F94350A84EB9DE091
:10A1C0000F944C0981E00EC0BE016F5F7F4FC50147
:10A1D0000F941701F701808191810196918380830B
:10A1E000D2CF80E00F90DF91CF911F910F91FF9020
:10A1F000EF90DF90CF90BF90AF909F908F907F9027
:10A200000895009781F41092900082E0809391006D
:10A210001092950010929400C19A80917100826012
:10A220008093710008958130910569F41092A00027
:10A2300082E08093A1001092A5001092A40089BB37
:10A24000809372000895029761F41092200182E0D9
:10A250008093210110922501109224018ABB8093E2
:10A26000730008957F928F929F92AF92BF92CF9288
:10A27000DF92EF92FF920F931F93CF93DF93FC0136
:10A280009081943208F0CEC06B017F01892F90E05D
:10A29000FC01EE0FFF1F8E0F9F1FFC01E95DFA4EC0
:10A2A000808161E08F770E94A8FFF70111821282FE
:10A2B00080816CE00F94BA24FCE08F9FB0011124E0
:10A2C00040E050E09B01240F351FF901EE0FFF1F06
:10A2D0002E0F3F1FF901E95DFA4E908197FD08C0EE
:10A2E0004F5F5F4F4C30510569F790E00E9401517C
:10A2F000F7017080C72DD0E08E01000F111FF8010B
:10A30000EC0FFD1FE95DFA4E80818068808377FC49
:10A3100089C0F0E2CF16F2E0DF060CF041C0F70191
:10A32000828128E532E0281B310987FD3395220F11
:10A33000331F220F331F032E000C440B550B81815A
:10A3400068E870E04B01881A910887FD9394880CA7
:10A35000991C880C991C092C000CAA08BB08D7FC76
:10A360000BC0B601653B710514F064EB70E0072E7D
:10A37000000C880B990B03C060E070E0CB0128193A
:10A3800039094A095B090F94472424EB30E040E087
:10A3900050E00F947924820E931EA41EB51E01C0B6
:10A3A0004601F3E2F71558F1F701218188E890E0C2
:10A3B000821B910927FD9395880F991F880F991F7C
:10A3C0008816990684F0F701228188E592E0821BC5
:10A3D000910927FD9395880F991F880F991F88165B
:10A3E00099060CF4C40102972FB7F894C00FD11F3F
:10A3F000C95DDA4E880F991F9A8389832FBF62E364
:10A4000070E080E090E0DF91CF911F910F91FF907D
:10A41000EF90DF90CF90BF90AF909F908F907F9004
:10A420000D941D09DF91CF911F910F91FF90EF9037
:10A43000DF90CF90BF90AF909F908F907F900895C6
:10A440001F920F920FB60F9211240BB60F922F93FB
:10A450003F934F935F936F937F938F939F93AF93AC
:10A46000BF93EF93FF9348E251E064E271E082E032
:10A4700090E00E94524FFF91EF91BF91AF919F9159
:10A480008F917F916F915F914F913F912F910F909D
:10A490000BBE0F900FBE0F901F9018951F920F923A
:10A4A0000FB60F9211240BB60F922F933F934F9339
:10A4B0005F936F937F938F939F93AF93BF93EF932C
:10A4C000FF9348EA50E064EA70E081E090E00E9487
:10A4D000524FFF91EF91BF91AF919F918F917F91DB
:10A4E0006F915F914F913F912F910F900BBE0F9005
:10A4F0000FBE0F901F9018951F920F920FB60F92DC
:10A5000011240BB60F922F933F934F935F936F934A
:10A510007F938F939F93AF93BF93EF93FF9348E9FC
:10A5200050E064E970E080E090E00E94524FFF91BB
:10A53000EF91BF91AF919F918F917F916F915F91BB
:10A540004F913F912F910F900BBE0F900FBE0F9028
:10A550001F9018959091C00095FFFCCF8093C60086
:10A5600008958F929F92AF92BF92EF92FF920F93B6
:10A570001F93CF93DF93CDB7DEB7A0970FB6F894B4
:10A58000DEBF0FBECDBF611571058105910591F14B
:10A5900000E0842E912CA12CB12C102FEE24E394FA
:10A5A000F12CEC0EFD1EE00EF11C07FDFA94A50146
:10A5B00094010F945724F7016083B901CA010F5F1A
:10A5C000611571058105910541F71F3F31F1E1E00A
:10A5D000F0E0EC0FFD1FE10FF11D17FDFA958081F2
:10A5E0008A3010F097E301C090E3890F0E94AA52CD
:10A5F0001150EBCF80E3A0960FB6F894DEBF0FBEEC
:10A60000CDBFDF91CF911F910F91FF90EF90BF9041
:10A61000AF909F908F900C94AA52A0960FB6F8948A
:10A62000DEBF0FBECDBFDF91CF911F910F91FF9085
:10A63000EF90BF90AF909F908F900895CF92DF9250
:10A64000EF92FF926B017C0197FF0BC08DE20E949D
:10A65000AA52F094E094D094C094C11CD11CE11C87
:10A66000F11C4AE0C701B601FF90EF90DF90CF9058
:10A670000C94B1528F929F92AF92BF92CF92DF9281
:10A68000EF92FF92CF936B017C01B42E20E030E07B
:10A69000A9010F94011E87FF07C08DE20E94AA52F4
:10A6A000F7FAF094F7F8F094C0E060E070E080E032
:10A6B0009FE3CB1541F02DEC3CEC4CEC5DE30F94AB
:10A6C000671ECF5FF6CF9B01AC01C701B6010F94A7
:10A6D000F7246B017C010F946A264B015C014AE070
:10A6E0000E94B152CC2389F1C501B4010F94061E1A
:10A6F0009B01AC01C701B6010F94F6246B017C01EC
:10A700008EE20E94AA5220E030E040E251E4C7010C
:10A71000B6010F94671E4B015C010F9463266B0119
:10A72000770FEE08FF08C701B6010E941E53C7014C
:10A73000B6010F94081E9B01AC01C501B4010F9432
:10A74000F6246B017C01C150F1F6CF91FF90EF90A0
:10A75000DF90CF90BF90AF909F908F9008958DE045
:10A760000E94AA528AE00C94AA52CF93DF93EC0184
:10A770008991882319F00E94AA52FACFDF91CF91D4
:10A780000C94AF538091941290919512981759F0B0
:10A79000E92FF0E0EC56FD4E82819F5F9F7790930A
:10A7A000951290E008958FEF9FEF08952F923F92BA
:10A7B0004F925F926F927F928F929F92AF92BF92D1
:10A7C000CF92DF92EF92FF920F931F93CF93DF937D
:10A7D000CDB7DEB728970FB6F894DEBF0FBECDBF5A
:10A7E000E82E0E94501D0F9406014B015C018091E0
:10A7F0000002882359F180914512882339F1409154
:10A80000D7085091D8086091D9087091DA0895015D
:10A810008401041B150B260B370B37FD2AC0833030
:10A8200079F03CF4813094F00F94350A86E19EE093
:10A830000BC0843059F40F94350A87EE9DE004C0B4
:10A840000F94350A8FEF9DE00F944C092091000280
:10A8500030E0A8EEB3E00F94AB24860E971EA81E3E
:10A86000B91E8092D7089092D808A092D908B092C9
:10A87000DA0880912A02882319F180915F098111F9
:10A880001FC08091981782FD08C0809118118130F7
:10A8900021F08091230B882399F0F894649919C6CC
:10A8A0006091321170913311809134119091351172
:10A8B000789420E030E0A9010F94011E87FD99C52E
:10A8C0008091200B843008F07EC20F9406014B016A
:10A8D0005C018091200B81111DC080919412909198
:10A8E0009512891B8F77B1F48091400990914109AD
:10A8F000A0914209B0914309A5019401281B390B8D
:10A900004A0B5B0BDA01C901885E9340A109B109CA
:10A91000B7FFF0C570E6F72E8091200B843008F069
:10A9200035C18091941290919512891B8F7709F40B
:10A930002DC10E94C253AC0197FDEECF209116139A
:10A94000309117138A3019F08D3009F0ECC0109255
:10A950003F092115310519F40E94679ADDCFF901ED
:10A96000E152F74F108210921713109216130FED49
:10A9700018E0F8018191803211F48F01FACF8E3402
:10A9800009F07AC00115110509F476C068E97FE085
:10A99000C8010F947F1D6C01892B41F06EE470E0BB
:10A9A000C80104960F944A28009709F4C8014AE0A8
:10A9B00050E060E070E001960F94F71A6093DB08B6
:10A9C0007093DC088093DD089093DE0840901813A4
:10A9D0005090191360901A1370901B133FEF431A95
:10A9E000530A630A730A641575058605970531F0E5
:10A9F000CD2821F460E085E69FE051C06AE270E076
:10AA0000C8010F9479289C01009709F1982F901B99
:10AA1000D12C992339F09150F801E90FF11D808173
:10AA2000D826F7CF4AE050E060E070E0C901019617
:10AA30000F94F71A4D2C512C612C712C641575054F
:10AA40008605970541F060E086E49FE028C060E05D
:10AA50008CE19FE024C08091DB089091DC08A091FC
:10AA6000DD08B091DE088093181390931913A0931A
:10AA70001A13B0931B1316C08091981780FF12C051
:10AA800064E171E1C8010F947F1D009729F0FC017A
:10AA9000838180538A3030F460E082EF9EE00E9430
:10AAA00072D774C080912F0281111CC067E470E0DE
:10AAB000C8010F944A280097A9F04AE050E060E0EE
:10AAC00070E001960F94F71A6430710581059105C5
:10AAD00048F48BE79EE00F944C0960E081E79EE02C
:10AAE0000E94F6ED8092400990924109A09242099D
:10AAF000B09243098091DF088B3309F40DCF809128
:10AB0000200B843008F008CF80919C09F89EC0018A
:10AB100011246FED78E08156964F0F94552881E00F
:10AB20000E9448B3F9CE2F3531050CF0F5CE8C35A7
:10AB3000C1F40E94C25397FDEFCE20913F0921112D
:10AB4000EBCE2091161330911713A9014F5F5F4F81
:10AB50005093171340931613F901E152F74F808376
:10AB6000DBCE8B3321F481E080933F09D5CE8091F9
:10AB70003F098111D1CEC90101969093171380939B
:10AB80001613F901E152F74F4083C6CE8091981712
:10AB900082FF19C18091200B811102C010924509DA
:10ABA000DD24D39440919417509195176091961796
:10ABB000709197178091901790919117A09192178B
:10ABC000B0919317481759076A077B0708F4D12CEF
:10ABD00000E010E0CC24C39440E6B42E54E6A52E49
:10ABE00069E6962E8091200B843008F0ECC0D110DD
:10ABF000EAC0809145098111E6C08091BB14909113
:10AC0000BC14A091BD14B091BE148093941790937E
:10AC10009517A0939617B093971741E050E0BE01A7
:10AC20006F5F7F4F83EB94E10E942368019719F4D3
:10AC3000898190E002C08FEF9FEFF82E409094172B
:10AC400050909517609096177090971740919017B5
:10AC5000509191176091921770919317DD24D394BE
:10AC6000441655066606770608F4D12C4416550698
:10AC700066067706B0F4019609F461C02AE0F21680
:10AC800009F46EC03DE0F31609F46AC043E2F4161D
:10AC900019F05AE3F5127CC080914409811178C003
:10ACA00054C00E945F8C83EB94E10E94AA6780915C
:10ACB0008F17882339F1815080938F17989EC00198
:10ACC000112441E061E0885D944F0E943361E0917E
:10ACD0008F1764E0E69FF0011124EC5DF44F408192
:10ACE00051816281738140939417509395176093BB
:10ACF00096177093971783EB94E10E943E640E942D
:10AD0000E85D16C00E94D75D0E94A08D0E940A8B4C
:10AD10000E94A6EC6D3371058105910518F483EA54
:10AD20009FE002C088EA9FE00E948FB3A092471381
:10AD30008091981782FD0DC08BEB9FE004C00F94AB
:10AD4000310A8CEA9FE00F944C0973E2F71208C0B5
:10AD500005C053E2F512DBC300E010E0C0924509E4
:10AD6000109244090115110519F40E94679A0DC04B
:10AD700080919C09B89E000D111D1124F801E15627
:10AD8000F64F108280E00E9448B300E010E02ACF26
:10AD90000F35110508F026CF8BE3F81203C0C092DF
:10ADA000440920CF8091440981111CCF80919C09D6
:10ADB000F801B89EE00DF11D1124E156F64FF08226
:10ADC0000F5F1F4F0FCF0F9406014B015C014091A5
:10ADD000C8085091C9086091CA087091CB08411504
:10ADE00051056105710529F180910C1490910D14A4
:10ADF000A0910E14B0910F14840F951FA61FB71FBA
:10AE000095018401081B190B2A0B3B0B37FD11C060
:10AE10000F94310A6091DD0B7091DE0B8FEC9FE097
:10AE20000F941E0A8AE00E94AA5280E090E00F94DC
:10AE3000260240910102509102026091030270913A
:10AE40000402411551056105710509F44EC0909148
:10AE50009A1580919B15981759F00F9406016093ED
:10AE60000C1470930D1480930E1490930F143DC026
:10AE70008091230B811137C0E11035C080910C14F3
:10AE800090910D14A0910E14B0910F14840F951F82
:10AE9000A61FB71FA5019401281B390B4A0B5B0B9A
:10AEA00057FD21C08091560981111FC081E0809318
:10AEB00056095F9A809114148E7F809314148A9A95
:10AEC000809114148D7F80931414809108018095D3
:10AED000817080930601809114148B7F80931414E9
:10AEE0000E94195002C01092560980915209909107
:10AEF0005309A0915409B0915509B501A401481B0B
:10AF0000590B6A0B7B0B77FDBCC120919A15909170
:10AF10009B158091540210915502291317C060911E
:10AF2000F70B869FB0011124660F672F661F770B02
:10AF30007195062F8091F80B189FB0011124660FB0
:10AF4000672F661F770B7195162F29C020919B15CF
:10AF500058E4259F900111242F5D334FF901EA5BDE
:10AF6000FF4F6081869FB0011124660F672F661F17
:10AF7000770B7195062F31968081819FB001112446
:10AF8000660F672F661F770B7195162F80919B15A3
:10AF900090919A15981719F08F5F8F70F9CF002351
:10AFA00031F10F940601C0904A09D0904B09E0900E
:10AFB0004C09F0904D09DC01CB01C114D104E1042E
:10AFC000F10469F48C599F4FAF4FBF4F80934A09EA
:10AFD00090934B09A0934C09B0934D0906C08C196E
:10AFE0009D09AE09BF09B7FF0AC00FEF08C0109254
:10AFF0004A0910924B0910924C0910924D09602F8A
:10B0000070E089E00E94E4FF112331F10F94060102
:10B01000C0904E09D0904F09E0905009F09051092E
:10B02000DC01CB01C114D104E104F10469F48C59B1
:10B030009F4FAF4FBF4F80934E0990934F09A093FE
:10B040005009B093510906C08C199D09AE09BF097A
:10B05000B7FF0AC01FEF08C010924E0910924F09A7
:10B060001092500910925109612F70E087E00E9400
:10B07000E4FF80913413882309F4F6C0E0902102A4
:10B08000F090220200912302109124026091120C90
:10B090007091130C6E5F7F4F072E000C880B990B7D
:10B0A0000F94081E9701A8010F94011E87FDDCC0B4
:10B0B00030909B15212C1A821B821C8280919A153C
:10B0C000831509F467C0832D90E068E4689FF00160
:10B0D000699FF00D1124EF5DF34F4589568967890B
:10B0E000708D452B462B472B89F4418D528D638DF6
:10B0F000748D452B462B472B49F4458D568D678D16
:10B1000070A1452B462B472B09F43FC078E4789F6C
:10B110009001799F300D1124C9018F5D934F6C010F
:10B12000FC0161817281838194810F94A5272B0199
:10B130003C01F60161A172A183A194A10F94061EA6
:10B140006D837E838F839887F60165A176A187A1A1
:10B1500090A50F94061E9B01AC016D817E818F81AD
:10B1600098850F94F125A30192010F94671E3B016E
:10B170006C01222D3A814B815C810F945727181660
:10B1800024F4262C7A82CB82DC8281E0830D8F70BE
:10B19000382E94CF2091250230912602409127022B
:10B1A00050912802622D7A818B819C810F94671EB9
:10B1B0009701A8010F94F7243B016C0120901D0218
:10B1C00030901E0240901F02509020029B01AC0163
:10B1D000B701C8010F94572718166CF09101A2010E
:10B1E000B301C6010F94572718161CF47101820190
:10B1F00002C0730186014090460950904709609053
:10B200004809709049099701A801C301B2010F9440
:10B2100057271816C4F420E037ED43EA5CE3B70182
:10B22000C8010F94671E6B017C0128E431EE4AE7E8
:10B230005FE3C301B2010F94671EA70196010F944B
:10B24000F7247B018C01C701D801809346099093B4
:10B250004709A0934809B0934909B701C8010F9461
:10B260006326CB010E94B0DFF4E68F0E911CA11C77
:10B27000B11C8092520990925309A0925409B09245
:10B2800055090E94679A80911811813009F06EC0AB
:10B290000F9406016B017C0180915B0990915C0920
:10B2A000A0915D09B0915E0997018601081B190BF9
:10B2B0002A0B3B0B37FD3AC08090191190901A1160
:10B2C000A0901B11B0901C110E94A6EC6093191164
:10B2D00070931A1180931B1190931C110091800997
:10B2E0001091810920918209309183090819190967
:10B2F0002A093B09DC01CB01800F911FA21FB31F5C
:10B300008093800990938109A0938209B093830967
:10B31000D701C601805F984DAF4FBF4F80935B0947
:10B3200090935C09A0935D09B0935E0980915709E1
:10B3300090915809A0915909B0915A09A701960115
:10B34000281B390B4A0B5B0B57FD10C030E8C30EAE
:10B350003EEED31EE11CF11CC0925709D092580951
:10B36000E0925909F0925A090E94E48A8091C30838
:10B37000882391F00F9406010091BF081091C00836
:10B380002091C1083091C208DC01CB01801B910BD8
:10B39000A20BB30BB7FFBEC00F9406016B017C017B
:10B3A0002091BE08222309F4D3C08091BA0890915D
:10B3B000BB08A091BC08B091BD08B701A601481B0D
:10B3C000590B6A0B7B0B77FDC3C030E0A8EEB3E0EE
:10B3D0000F94AB24C60ED71EE81EF91EC092BA0801
:10B3E000D092BB08E092BC08F092BD080E94B05D0C
:10B3F000AFC011E010935F098091230B811166C0EB
:10B400008AE196E00E94B55384E08093121182E0B5
:10B4100080939A0881E09AE590931D1680931C16FC
:10B420008EE490E090931F1680931E1687E0809321
:10B43000101682E88093131684E890E0A0E0B0E054
:10B440008093141690931516A0931616B0931716A2
:10B450000F94800110931D110E94309440E060E62B
:10B460007EE086E697E10E943C9480E30E94AA5227
:10B470008AE00E94AA520E9424948091CC0860E045
:10B48000182719F086E496E10DC08EE49EE00E9434
:10B490000C9480E30E94AA528AE00E94AA5260E0C3
:10B4A00088E29EE00E940C948CE39EE00F944C098D
:10B4B00080E30E94AA528AE00E94AA52112331F02E
:10B4C0008EE29EE090939E0980939D090E945F8C7E
:10B4D000F7C980915B0290915C02A0915D02B091EE
:10B4E0005E028093321190933311A0933411B09384
:10B4F0003511D6C98DE99FE00F944C09809240091F
:10B5000090924109A0924209B092430903CA109255
:10B5100044092BCC0F9406016B017C012091C308D8
:10B5200030E0A8EEB3E00F94AB24C60ED71EE81EA1
:10B53000F91EC092BF08D092C008E092C108F092F4
:10B54000C20880E00E94CCD78AE00E94AA5224CF91
:10B5500028960FB6F894DEBF0FBECDBFDF91CF9116
:10B560001F910F91FF90EF90DF90CF90BF90AF9021
:10B570009F908F907F906F905F904F903F902F9013
:10B5800008951F920F920FB60F9211240F900FBEC5
:10B590000F901F9018951F920F920FB60F921124C3
:10B5A0000BB60F920F931F932F933F934F935F937D
:10B5B0006F937F938F939F93AF93BF93CF93DF93BB
:10B5C000EF93FF9300919512D091941211E01D0F0B
:10B5D0001F77C091C6009091D208492F092E000C08
:10B5E000550B660B770B4131510508F064C0FA0129
:10B5F0008827E256FF4F8F4F0D94EE24CD3449F04B
:10B60000CE34B9F481E006C0CA3338F0CD3409F045
:10B6100043C082E08093D20876C0C03308F073C084
:10B62000C03209F470C0CD32B9F56DC0C13351F0EC
:10B6300018F4C03289F567C0C43331F0C83361F5FE
:10B640008BE0E8CF83E0E6CF88E0E4CFC03321F0A1
:10B65000C13311F586E0DECF84E0DCCFC833E1F4FE
:10B6600085E0D8CFC233C1F487E0D4CFC133A1F491
:10B6700089E0D0CFC03381F48AE0CCCFC73361F406
:10B680008CE0C8CFC63341F48DE0C4CFC032D9F1CD
:10B69000C33511F48EE0BECF80E1BCCF80ED8C0FBE
:10B6A0008A3088F59FE09093D2088093D1082BC010
:10B6B000CA3049F526C0CA3031F580917E168823FC
:10B6C00001F1973089F03CF49530D9F410921402CE
:10B6D0001092461316C09A3059F09F3091F4809121
:10B6E000D1080E9468940DC081E08093541109C074
:10B6F0000E94F68D0E945F8C8EEF0E94DAC20E943B
:10B7000048C31092D208011731F0ED2FF0E0EC564B
:10B71000FD4EC283D12FD0939412FF91EF91DF9110
:10B72000CF91BF91AF919F918F917F916F915F91D9
:10B730004F913F912F911F910F910F900BBE0F9042
:10B740000FBE0F901F9018958EBD0DB407FEFDCF54
:10B7500008958FEF8EBD0DB407FEFDCF8EB5089511
:10B76000909164009B7F90936400982F906A9695C7
:10B770009CBD80FD03C091E0863009F490E09DBD42
:10B780000895CF92DF92EF92FF920F931F93CF9382
:10B79000DF936C017A018B01C0E0D0E0CE15DF05AC
:10B7A00081F0D8016D918D01D601ED91FC91019050
:10B7B000F081E02DC6011995892B11F02196EECF6D
:10B7C0007E01C701DF91CF911F910F91FF90EF9004
:10B7D000DF90CF900895089580E090E00895FC01F7
:10B7E000538D448D252F30E0842F90E0821B930BE6
:10B7F000541710F0CF96089501970895FC01918D8C
:10B80000828D981761F0828DDF01A80FB11D5D96C2
:10B810008C91928D9F5F9F73928F90E008958FEF30
:10B820009FEF0895FC01918D828D981731F0828DE4
:10B83000E80FF11D858D90E008958FEF9FEF08953B
:10B84000FC01918D228D892F90E0805C9F4F821B9F
:10B8500091098F739927089586E194E10E94205CF5
:10B8600021E0892B09F420E0822F0895FC01848DCA
:10B87000DF01A80FB11DA35ABF4F2C91848D90E01A
:10B8800001968F739927848FA689B7892C93A089F5
:10B89000B1898C91837080648C93938D848D98137F
:10B8A00006C00288F389E02D80818F7D8083089512
:10B8B000EF92FF920F931F93CF93DF93EC0181E000
:10B8C000888F9B8D8C8D981305C0E889F9898081BC
:10B8D00085FD26C0F62E0B8D10E00F5F1F4F0F73F6
:10B8E0001127E02E8C8DE8120CC00FB607FCFACFA2
:10B8F000E889F989808185FFF5CFCE010E94365C09
:10B90000F1CF8B8DFE01E80FF11DE35AFF4FF0825E
:10B910009FB7F8940B8FEA89FB89808180620AC007
:10B920009FB7F894EE89FF896083E889F98980815F
:10B930008370806480839FBF81E090E0DF91CF912E
:10B940001F910F91FF90EF900895CF93DF93EC013B
:10B95000888D8823C9F0EA89FB89808185FD05C02F
:10B96000A889B9898C9186FD0FC00FB607FCF5CF69
:10B97000808185FFF2CFA889B9898C9185FFEDCFB1
:10B98000CE010E94365CE7CFDF91CF91089580E031
:10B9900090E0892B41F080E090E0892B21F00E941B
:10B9A0000000811121C080E090E0892B41F080E00F
:10B9B00090E0892B21F00E940000811118C080E0E6
:10B9C00090E0892B21F00E942C5C811113C080E053
:10B9D00090E0892BA1F080E090E0892B81F00E941B
:10B9E000000081110AC008950E940000DCCF0E946F
:10B9F0000000E5CF0E940000EACF0C9400000895FB
:10BA0000FC0120E03EE2DB014C91403241F0283065
:10BA100011F430833196DB014C91408331962F5FD6
:10BA20006F5F7F4F2B3079F7108208950F940928AC
:10BA30000F931F93CF93DF938B01EA01DB016D918D
:10BA40007C910E944465D801ED91FC911197908101
:10BA50008881992349F0893638F43196ED93FC9327
:10BA600088818F5F8883EFCF893658F48FE2808397
:10BA7000F8018081918101969183808388818F5F15
:10BA80008883DF91CF911F910F9108951F920F929C
:10BA90000FB60F9211240BB60F922F933F934F9333
:10BAA0005F936F937F938F939F93AF93BF93EF9326
:10BAB000FF9386E194E10E94365CFF91EF91BF9184
:10BAC000AF919F918F917F916F915F914F913F9136
:10BAD0002F910F900BBE0F900FBE0F901F901895D7
:10BAE0001F920F920FB60F9211240BB60F922F9345
:10BAF0008F939F93EF93FF93E0912614F091271477
:10BB00008081E0912C14F0912D1482FD12C090815F
:10BB100080912F148F5F8F7320913014821751F012
:10BB2000E0912F14F0E0EA5EFB4E958F80932F1486
:10BB300001C08081FF91EF919F918F912F910F9084
:10BB40000BBE0F900FBE0F901F9018958BE1ECE08D
:10BB5000F5E1A1EFB4E101900D928A95E1F7089526
:10BB60008091981782FF1FC084E992E10F944C09DD
:10BB700060919417709195178091961790919717EF
:10BB80004AE00E94B1528FE20E94AA52609190173F
:10BB90007091911780919217909193174AE00E94AB
:10BBA000B1520C94AF5386EA92E10D944C09109275
:10BBB000230B809198178F7D8B7F809398170E941D
:10BBC00048D7882321F083EB94E10C94AA67089569
:10BBD0008091981783FF03C084608093981708951D
:10BBE000CF92DF92EF92FF920F931F93CF93DF9349
:10BBF000CDB7DEB7EDB6FEB6DC010D900020E9F75B
:10BC00009D01281B390B2C5F3F4F4DB75EB7421B80
:10BC1000530B0FB6F8945EBF0FBE4DBF0DB71EB7E6
:10BC20000F5F1F4F9F938F9380E991E19F938F93B5
:10BC30001F930F930F94991D680154E0C50ED11CFA
:10BC40000F900F900F900F900F900F90F601808142
:10BC5000882349F0082E000C990B0F940E28F6014A
:10BC600081936F01F3CFC8010E945DB38CE891E12D
:10BC70000E948FB30FB6F894FEBE0FBEEDBEDF91EB
:10BC8000CF911F910F91FF90EF90DF90CF9008958B
:10BC90008F929F92AF92BF92CF92DF92EF92FF92DC
:10BCA000CF9380919817877F8093981780910F1575
:10BCB000882321F08CE095E10E94AA671092F0148D
:10BCC0001092ED1485E38093EC140F9406016B0140
:10BCD0007C0120EDC20E27E0D21EE11CF11CA895CC
:10BCE00061E08091EC140E9479FF61E08091EC1496
:10BCF0000E94A8FF209A289A219A2398229A81E0EC
:10BD00000E94B05B85E08093EE140E94B05BCAE0B5
:10BD10008FEF0E94A45BC150D9F7A89520E030E0D6
:10BD2000A90160E08CEE94E10E948A668093EF1492
:10BD3000813061F00F940601DC01CB018C199D0963
:10BD4000AE09BF09B7FDEACF81E062C0A8952AEA33
:10BD500031E040E050E068E08CEE94E10E948A66B9
:10BD6000853011F481E00AC0C4E00E94A95B809391
:10BD7000EF14C150D1F78A3A61F482E08093F01455
:10BD8000A8958091F014823081F0812C912C54017F
:10BD900011C00F940601DC01CB018C199D09AE097D
:10BDA000BF09B7FDD4CF82E033C0812C912CA12CE8
:10BDB00080E4B82E20E030E0A90167E38CEE94E146
:10BDC0000E948A66A501940169E28CEE94E10E94CA
:10BDD0008A668093EF14882361F00F940601DC01DA
:10BDE000CB018C199D09AE09BF09B7FDE3CF8AE0ED
:10BDF0000FC08091F014823021F520E030E0A901DD
:10BE00006AE38CEE94E10E948A66882361F088E000
:10BE10008093ED148CEE94E10E9482660F94350AB3
:10BE20008EE791E122C00E94A95B807C803C19F4DE
:10BE300083E08093F0140E94A95B0E94A95B0E949A
:10BE4000A95B8CEE94E10E9482661092EE1481E070
:10BE50000F94680C81110CC080E00F94680C811164
:10BE600007C00F94310A8AE691E10F944C091AC079
:10BE70006EEC74E18CE095E10E94D564811105C0FF
:10BE80000F94310A89E591E1F0CF8091981788608D
:10BE9000809398170F94350A8DE491E10F944C0923
:10BEA0000E945150CF91FF90EF90DF90CF90BF90C4
:10BEB000AF909F908F900C94A65D2F923F925F92CF
:10BEC0006F927F928F929F92AF92BF92CF92DF92AA
:10BED000EF92FF920F931F93CF93DF93CDB7DEB70F
:10BEE000C356D1090FB6F894DEBF0FBECDBF8C018B
:10BEF0006B014A012DB63EB6512C7E0187E5E80E56
:10BF0000F11CF6018381823008F41FC18085918580
:10BF1000A285B3858F719927AA27BB27892B8A2BE6
:10BF20008B2B09F012C11092351A45E35AE1BE017C
:10BF30006F5F7F4FC6010E943F6918160CF005C164
:10BF40008C85982F9871903129F42091910B215074
:10BF5000223078F42981222309F4F7C0253E89F2A2
:10BF60002E3279F22091351A2E3259F28A7049F622
:10BF70007CC06DB67EB6BE016F5F7F4FC7010E9469
:10BF8000005D0115110521F0F8018081811163C068
:10BF900021E081E090E0F70101900020E9F731977E
:10BFA000EE19FF09E80FF91F32968DB79EB78E1B69
:10BFB0009F0B0FB6F8949EBF0FBE8DBFEDB7FEB7B7
:10BFC00031965F01211102C0B80102C060E776E03E
:10BFD000C5010F945528B701C5010F943F2860E7AC
:10BFE00076E0C5010F943F2819A21CA221E0A70109
:10BFF000B601CE0181960E94966B81110DC0809191
:10C00000910B811109C00F94350A89E391E10F94D6
:10C010004C09C7010E94B5538BE1FE01B196DE01C8
:10C02000DC9601900D928A95E1F740E050E0BE0168
:10C03000645C7F4FC5010E945D5FCE01CC960E947B
:10C04000B367CE0181960E94B3670FB6F8947EBEA7
:10C050000FBE6DBE56CFF80101900020E9F7319771
:10C06000CF01801B910B20E096CF21E0903109F0A9
:10C0700020E08091981720FB84F9809398179031E5
:10C0800041F08985873409F03CCF8A858E3709F4E1
:10C0900038CF8091910B813021F068F08230C1F16E
:10C0A00030CF8091940B9091950B01969093950BC6
:10C0B0008093940B26CFBE016F5F7F4F87E79AE195
:10C0C0000E94005D0115110529F487E7A82E8AE179
:10C0D000B82E09C05801F50181915F018823A9F3A9
:10C0E0000E94AA52F8CFF50181915F01882319F0CF
:10C0F0000E94AA52F8CF80E20E94AA526D8D7E8DD6
:10C100008F8D98A14AE00E94B1520E94AF53F9CEA0
:10C11000BE016F5F7F4F87E79AE10E94005D811447
:10C12000910441F067E77AE1C4010F942C28892B30
:10C1300051F40BC0852D90E02091920B3091930B20
:10C140008217930711F05394DCCE0FB6F8943EBEDD
:10C150000FBE2DBECD59DF4F0FB6F894DEBF0FBE18
:10C16000CDBFDF91CF911F910F91FF90EF90DF90A6
:10C17000CF90BF90AF909F908F907F906F905F9087
:10C180003F902F900895CF93DF93CDB7DEB76B9795
:10C190000FB6F894DEBF0FBECDBF81E08093910B48
:10C1A0001092950B1092940B81EF94E10E947D66A2
:10C1B0008BE1E1EFF4E1DE01119601900D928A9599
:10C1C000E1F740E050E0BE016F5F7F4F80E090E01C
:10C1D0000E945D5FCE0101960E94B3678091940B2F
:10C1E0009091950B6B960FB6F894DEBF0FBECDBF46
:10C1F000DF91CF9108950F931F93CF93DF93CDB726
:10C20000DEB76B970FB6F894DEBF0FBECDBF8B01C4
:10C2100022E02093910B9093930B8093920B81EFEC
:10C2200094E10E947D668BE1E1EFF4E1DE0111967D
:10C2300001900D928A95E1F7A801BE016F5F7F4FD3
:10C2400080E090E00E945D5FCE0101960E94B3679E
:10C250006B960FB6F894DEBF0FBECDBFDF91CF91C6
:10C260001F910F910895DF92EF92FF920F931F930A
:10C27000CF93DF9300D01F92CDB7DEB720919817F0
:10C2800023FF3DC1F42EE62E8C010E9448D788235F
:10C2900009F481C0FF2009F48CC080918F17882396
:10C2A00051F00F94310A8FE492E10F944C0980E031
:10C2B00090E00F94260289E29BE09A8389838FE2C3
:10C2C0008093280B81E08B83F12C9BE1D92E809108
:10C2D0008E17F81678F4DF9CC0011124AE014D5F73
:10C2E0005F4FBE016F5F7F4F8058994E0E94185D6F
:10C2F000F394EDCF8B818B3578F4AE014D5F5F4FBA
:10C30000BE016F5F7F4F83EB94E10E94185D8981CE
:10C310009A8101979A838983E981FA811082E09159
:10C320008F1784E0E89FF0011124EC5DF44F8091B9
:10C33000941790919517A0919617B09197178083B5
:10C340009183A283B3830F94350AB80186E392E107
:10C350000F941E0A60918F1789E6689FB00111241F
:10C36000685D744F8BE292E10F941E0A409194171E
:10C3700050919517609196177091971785E292E109
:10C380000F94E2098AE00E94AA5280918F178F5F72
:10C3900080938F1726C0FF2039F00F94350A85E16E
:10C3A00092E10F944C091DC010928F1782E0F82E75
:10C3B00002C0FF24F3940F94350A80E192E10F94B8
:10C3C0004C0981E0F81609F497C08CEF91E10F94C5
:10C3D0004C09B80188E092E10F941E0A8AE00E949D
:10C3E000AA520E94D75DB801CE0103960F948D0327
:10C3F0008C01009709F483C06B817C81EE2009F4E5
:10C4000050C021E0AC0183EB94E10E94966B88233D
:10C4100009F43FC08091C4149091C514A091C61432
:10C42000B091C7148093901790939117A09392178F
:10C43000B093931710929417109295171092961725
:10C4400010929717B8018EEE91E10F941E0A409159
:10C45000901750919117609192177091931786EEF3
:10C4600091E10F94E2098AE00E94AA5287ED91E1DE
:10C470000F944C09B80180E090E00E94FB6080912D
:10C48000351A811102C0C80102C085E39AE160E05B
:10C4900030C0B80183EC91E10F941E0A80EC91E169
:10C4A0000FC026E5AC0183EB94E10E94966B8111ED
:10C4B0000AC0B8018CEA91E10F941E0A89EA91E161
:10C4C0000F944C091CC08091981781608093981735
:10C4D000B80180E090E00E94FB6010927E16B801E7
:10C4E00087E991E10F941E0A8AE00E94AA5260E057
:10C4F000C8010E9451EE03C082E092E168CF0F9024
:10C500000F900F900F90DF91CF911F910F91FF909F
:10C51000EF90DF900895CF92DF92EF92FF92CF934A
:10C520006B017C01C42F80912A1A90912B1AA09143
:10C530002C1AB0912D1A8C159D05AE05BF05D1F0B2
:10C540000E943767811102C080E018C02AE238E1FA
:10C55000B701A6018091331A9091341A0E94B967ED
:10C56000882391F3C0922A1AD0922B1AE0922C1AA7
:10C57000F0922D1A81E0C1118093321ACF91FF9071
:10C58000EF90DF90CF9008954F925F926F927F92DD
:10C590008F929F92AF92BF92CF92DF92EF92FF92D3
:10C5A0000F931F93CF93DF93EC0142305105610548
:10C5B000710510F480E069C089859A85AB85BC85DA
:10C5C0000196A11DB11D84179507A607B70790F323
:10C5D0008F89803149F4852E962EA72EBB248B8916
:10C5E0009C89AD89BE890FC0803221F78B889C88D9
:10C5F000AD88BE88DB01CA01E7E0B695A79597959F
:10C600008795EA95D1F7880E991EAA1EBB1E2801B0
:10C6100039016A017B0141E0C501B4010E948B62CE
:10C62000882341F29F89903161F4DD24EE24FF24B8
:10C630009601220F331FF901E65DF74E51824082C9
:10C6400011C0E894C7F8DD24EE24FF249601220FE0
:10C65000331F220F331FF901E65DF74E40825182EE
:10C66000628273829A89923080F04D815E816F81FF
:10C670007885840E951EA61EB71E80922E1A909263
:10C680002F1AA092301AB092311ADF91CF911F91D8
:10C690000F91FF90EF90DF90CF90BF90AF909F9061
:10C6A0008F907F906F905F904F900895CF92DF9220
:10C6B000EF92FF920F931F93CF93DF93FC0181853D
:10C6C0009285A385B4850196A11DB11D8417950798
:10C6D000A607B70710F480E061C08789803149F46C
:10C6E000BB27A72F962F852FC388D488E588F68887
:10C6F0000FC0803281F783899489A589B6896A0140
:10C700007B01C7E0F694E794D794C794CA95D1F714
:10C710008C0D9D1DAE1DBF1DE9016A017B018F01BE
:10C7200040912A1A50912B1A60912C1A70912D1A4F
:10C7300084179507A607B70739F040E0BC01CD0183
:10C740000E948B62882339F2F8018789803179F45D
:10C75000B701A601552766277727440F551FFA0111
:10C76000E65DF74E80819181A0E0B0E012C0B70194
:10C77000A6014F77552766277727440F551F440F8B
:10C78000551FFA01E65DF74E80819181A281B38148
:10C79000BF7088839983AA83BB8381E0DF91CF91A7
:10C7A0001F910F91FF90EF90DF90CF9008954F92DF
:10C7B0005F926F927F92AF92BF92CF92DF92EF9291
:10C7C000FF920F931F93CF93DF9300D01F92CDB7AB
:10C7D000DEB78C0149835A836B837C835901C12C5A
:10C7E000D12C7601412C82E0582E612C712C49818C
:10C7F0005A816B817C819E012F5F3F4FC8010E944F
:10C800005663882341F1D301C201F801058404C0B5
:10C81000880F991FAA1FBB1F0A94D2F7C80ED91EF2
:10C82000EA1EFB1E49815A816B817C818789803198
:10C8300039F481E0483F5F4F6105710538F4D7CF87
:10C8400081E0483F5F4F6F4F7F4088F2F501C08223
:10C85000D182E282F3820F900F900F900F90DF91C0
:10C86000CF911F910F91FF90EF90DF90CF90BF90ED
:10C87000AF907F906F905F904F9008958F929F92AE
:10C88000AF92BF92CF92DF92EF92FF920F931F93DE
:10C89000CF93DF93EC018B81811102C080E078C0DF
:10C8A00009891A892B893C89041715072607370738
:10C8B000A8F36A017B01823029F4C886D986EA860A
:10C8C000FB860DC0C114D104E104F10451F41886B3
:10C8D00019861A861B861C821D821E821F8281E099
:10C8E00057C088849984AA84BB84E98DFA8D2585F4
:10C8F00030E0275F3F4FB501A40141505109610964
:10C900007109022E04C076956795579547950A944C
:10C91000D2F7D701C6010197A109B10904C0B695A4
:10C92000A795979587952A95D2F784179507A60717
:10C93000B70720F089288A288B2871F44D895E89F1
:10C940006F89788D4C835D836E837F834C015D019D
:10C950008E010C5F1F4F16C0841B950BA60BB70BE7
:10C96000F5CF4C815D816E817F819801898D9A8D93
:10C970000E94566391E0891A9108A108B1088823A2
:10C9800009F48CCF81149104A104B10451F795CF1F
:10C99000DF91CF911F910F91FF90EF90DF90CF909B
:10C9A000BF90AF909F908F9008950F931F93CF9358
:10C9B000DF93FC012381222311F080E044C08B012E
:10C9C000EC01FB018789803139F18032B1F783E0D6
:10C9D0008B83F801428D538D648D758D4D8B5E8BED
:10C9E0006F8B788F9E012F5E3F4FC8010E94D763E7
:10C9F000882319F31A8F098F81E089831886198695
:10CA00001A861B861C821D821E821F82188A1C8623
:10CA10001D861E861F8617C082E08B831D8A1E8A94
:10CA20001F8A188EFB01808D918DA0E0B0E025E07B
:10CA3000880F991FAA1FBB1F2A95D1F7898B9A8B44
:10CA4000AB8BBC8BD7CFDF91CF911F910F91089506
:10CA5000CF93DF93EC0141E0611101C040E06C85B0
:10CA60007D858E859F850E948B62882341F0888911
:10CA700020E2829FC0011124865D974E02C080E0B3
:10CA800090E0DF91CF910895CF93DF93EB01FC010C
:10CA90002381211102C080E028C02250223020F4DE
:10CAA0008FE28883198220C060E00E942865009789
:10CAB00091F3FC0190E080E02EE23081303269F0A9
:10CAC000883029F4DE01A90FB11D2C939F5FDE0190
:10CAD000A90FB11D30813C939F5F8F5F31968B30E2
:10CAE00061F7C90FD11D188281E0DF91CF910895C0
:10CAF0003F924F925F926F927F928F929F92AF92EE
:10CB0000BF92CF92DF92EF92FF920F931F93CF933A
:10CB1000DF93CDB7DEB72C970FB6F894DEBF0FBE0C
:10CB2000CDBF5C01DC0159968D909C905A97F40121
:10CB300081859285A385B4859C01AD012F5F3F4F10
:10CB40004F4F5F4F29873A874B875C87D5011496F3
:10CB5000CD90DD90ED90FC901797C114D104E104C5
:10CB6000F10439F0BFEFCB1ADB0AEB0AFB0A312CD8
:10CB700007C0F401C080D180E280F3803324339475
:10CB8000260137011D821E821F821886F4018185CD
:10CB90009285A385B4852D813E814F8158852817C4
:10CBA00039074A075B0708F064C089859A85AB8519
:10CBB000BC858C159D05AE05BF0550F482E0C82EDE
:10CBC000D12CE12CF12C92E0492E512C612C712CAE
:10CBD0009E012F5F3F4FB701A601C4010E9456631B
:10CBE000882309F446C089819A81AB81BC81892B55
:10CBF0008A2B8B2B41F0260137019FEF491A590AE6
:10CC0000690A790A05C0C414D504E604F70491F052
:10CC10002D813E814F8158852F5F3F4F4F4F5F4F92
:10CC20002D833E834F8358873FEFC31AD30AE30A0D
:10CC3000F30AACCF0FEF1FEF2FEF3FE0B301A201DC
:10CC4000C4010E94C462F82E882399F0D50114967D
:10CC50004D915D916D917C9117974115510561053D
:10CC6000710549F093018201C4010E94C4628111DF
:10CC700002C0F12C29C0D50114964D925D926D929F
:10CC80007C921797332051F0D301C2010196A11D68
:10CC9000B11DF40180839183A283B383F50185895B
:10CCA0009689A789B08D892B8A2B8B2B69F4D501A6
:10CCB00055964D925D926D927C92589711968C91FB
:10CCC0001197806811968C938F2D2C960FB6F8943F
:10CCD000DEBF0FBECDBFDF91CF911F910F91FF90AF
:10CCE000EF90DF90CF90BF90AF909F908F907F900C
:10CCF0006F905F904F903F90089540E050E0BA01F0
:10CD00000C943E6461E0FC0180810E9479FF8FEF0A
:10CD10000C94A45BEF92FF921F93CF93DF9300D00C
:10CD20001F92CDB7DEB77C01162F29833A834B8340
:10CD30005C83FC0182810E94B05B60E0F70180812E
:10CD40000E9479FF0F94D702812F80640E94A45B18
:10CD50008C810E94A45B8B810E94A45B8A810E94CB
:10CD6000A45B89810E94A45B112311F087E801C0B4
:10CD700085E90E94A45B1C3011F40E94A95B10E0BD
:10CD80000E94A95BF701838387FF04C01F3F11F056
:10CD90001F5FF6CF0F900F900F900F90DF91CF9104
:10CDA0001F91FF90EF9008950F931F93CF93DF9300
:10CDB000EC0189018C81833039F089E0440F551FE3
:10CDC000661F771F8A95D1F79A01AB0168E1CE0102
:10CDD0000E948A66811128C08EEF8EBDF801C801BD
:10CDE0009E5F0DB407FEFDCF20812EBD0DB407FE62
:10CDF000FDCF21812EBD32968E179F0791F70DB47E
:10CE000007FEFDCF8FEF0E94A45B8FEF0E94A45B13
:10CE10000E94A95B8B838F71853041F083E1898308
:10CE2000CE010E94826619C086E016C00F94D70218
:10CE3000882379F020E030E0A9016DE0CE010E9466
:10CE40008A66811108C00E94A95B811104C011E0AB
:10CE500005C087E101C086E1898310E0CE010E9410
:10CE60008266812FDF91CF911F910F910895CF930B
:10CE70008091321A8823B9F140912A1A50912B1AC5
:10CE800060912C1A70912D1A2AE238E18091331AA0
:10CE90009091341A0E94D466C82F811102C0C0E05C
:10CEA00023C040912E1A50912F1A6091301A709120
:10CEB000311A411551056105710591F02AE238E1F9
:10CEC0008091331A9091341A0E94D466882339F3E2
:10CED00010922E1A10922F1A1092301A1092311AA4
:10CEE0001092321A01C0C1E08C2FCF910895CF93D8
:10CEF000DF93EC018B81882339F1898187FF20C082
:10CF000061E0CE010E942865FC01892BE9F0808157
:10CF1000853ED1F08B81823040F489899A89AB8932
:10CF2000BC89848F958FA68FB78F8D899E89AF8995
:10CF3000B88D938F828FB58BA48B89818F778983EE
:10CF4000DF91CF910C94376781E0888380E0DF9197
:10CF5000CF910895CF93DF93EC010E9477671B82F6
:10CF6000DF91CF910895FC01238121110C94AA67D0
:10CF70000895CF92DF92EF92FF920F931F93CF937A
:10CF8000DF93EC0189018C81833039F089E0440F13
:10CF9000551F661F771F8A95D1F79A01AB0161E192
:10CFA000CE010E948A66882339F084E08983CE010D
:10CFB0000E94826680E03EC00F9406016B017C01F6
:10CFC0002CE2C20E21E0D21EE11CF11C0E94A95BE2
:10CFD0008B838F3F61F40F940601DC01CB018C1928
:10CFE0009D09AE09BF09B7FDF1CF81E11DC08E3F9C
:10CFF000D1F48FEF8EBDF801D801A150BE4F0DB412
:10D0000007FEFDCF9EB591938EBDEA17FB07B9F7DA
:10D010000DB407FEFDCF8EB58C930E94A95B0E94D4
:10D02000A95B11E003C08FE0898310E0CE010E946C
:10D030008266812FDF91CF911F910F91FF90EF902A
:10D04000DF90CF9008952F923F924F925F926F9210
:10D050007F928F929F92AF92BF92CF92DF92EF9288
:10D06000FF920F931F93CF93DF9300D01F92CDB702
:10D07000DEB79C838B834B015A01DC0113968C91A4
:10D08000811103C08FEF9FEFE3C0EB81FC818181B1
:10D0900080FFF8CFEB81FC8181899289A389B489D3
:10D0A0004085518562857385841B950BA60BB70B54
:10D0B000A50160E070E084179507A607B70708F49C
:10D0C0005C0175018B819C8104969A838983612C14
:10D0D00042E0742EE114F10409F48BC0AB81BC81F1
:10D0E00018964D915D916D917C911B976A01B1E00D
:10D0F000DB22EB81FC812381818D928D1A012B0132
:10D1000039E056944794379427943A95D1F72230D2
:10D1100061F4FC01828D938DA48DB58DBC01CD0190
:10D12000620D731D841D951D4AC0DC0114961C916F
:10D1300011501221C114D10401F511111EC0452B4B
:10D14000462B472B59F4EB81FC8185899689A78969
:10D15000B08D84839583A683B7830FC0AB81BC81D8
:10D1600014964D915D916D917C91179729813A812B
:10D170000E945663882309F485CFEB81FC81218DC1
:10D18000328D84819581A681B7810297A109B10969
:10D19000F901058404C0880F991FAA1FBB1F0A94B8
:10D1A000D2F74685578560897189840F951FA61F20
:10D1B000B71FBC01CD01610F711D811D911D930130
:10D1C0002C193D0987012E153F0508F48901011529
:10D1D000F2E01F0779F520912A1A30912B1A40911D
:10D1E0002C1A50912D1A621773078407950719F4AA
:10D1F00021C0C5012DC09401AB01BC018091331A3F
:10D200009091341A0E94B967882309F43BCF800EAD
:10D21000911EEB81FC8180859185A285B385800F6D
:10D22000911FA11DB11D80879187A287B387E01A46
:10D23000F10A50CF40E00E948B62882309F422CF8C
:10D24000B601665D774EA801C4010F942328DFCF95
:10D250000F900F900F900F90DF91CF911F910F9132
:10D26000FF90EF90DF90CF90BF90AF909F908F9006
:10D270007F906F905F904F903F902F900895DF9236
:10D28000EF92FF920F931F93CF93DF938C01EB01EB
:10D290007A018DE0D82E40E250E0BE01C8010E9424
:10D2A00023688032910539F021E0892B09F420E0D0
:10D2B000822F819544C028812223C9F1253E11F097
:10D2C0002E3231F4E114F10431F3F7011082E3CF8F
:10D2D000E114F10441F13B853F733F3021F54A8D64
:10D2E0005B8D452B01F52F713FEF320F3530D8F4B0
:10D2F00030E021503109D29EC001D39E900D1124FF
:10D30000D701A80FB91FFE0120E0AD01253088F438
:10D3100031813D932F5F32962D30C1F7288126FF52
:10D3200002C0FA0115862B8523FDB5CF08C080E029
:10D3300006C02B3010F43481ECCF3681EACFDF9178
:10D34000CF911F910F91FF90EF90DF9008954F9232
:10D350005F926F927F929F92AF92BF92CF92DF9235
:10D36000EF92FF920F931F93CF93DF931F92CDB74E
:10D37000DEB78C017B015A01C22EDB0159968D91DB
:10D380009C915A97F801928F818FCB010E947D6604
:10D39000912CF70180859185A285B38541895289B9
:10D3A0006389748984179507A607B70708F060C0DA
:10D3B00025E0B695A795979587952A95D1F7F82FEB
:10D3C000FF70DF2ED70113968C91823008F460C075
:10D3D00041E050E0BE016F5F7F4FC7010E942368AC
:10D3E000019719F4898190E002C08FEF9FEF0196B9
:10D3F00009F44EC0F70180859185A285B3854F96CB
:10D40000A11DB11D80879187A287B387F0E2DF9EBF
:10D41000B0011124665D774E61157105C9F1DB011C
:10D420008C91882319F0853EC1F46CC191100EC017
:10D4300080912A1A90912B1AA0912C1AB0912D1A32
:10D44000F80184879587A687B787D08ADB018C91FE
:10D45000882361F0992493949CCF4BE050E0C50160
:10D460000F941628892B09F094CF14C09924939413
:10D470008C2D8274823461F4992009F48BC0F801F8
:10D48000D08861E0C8010E942865009709F00DC1AD
:10D4900080E03BC1C7FCFCCFF0E2DF9EA00111247D
:10D4A0009A01265D374ED9011B968C91817121F02E
:10D4B0008C2D827109F06AC080912A1A90912B1AE2
:10D4C000A0912C1AB0912D1AF80184879587A68710
:10D4D000B787D08ACA01865D974E7C01DC015496DD
:10D4E0004D915C91559760E070E0DA0199278827AB
:10D4F000858B968BA78BB08FF701428D538D60E0A3
:10D5000070E0482B592B6A2B7B2BD80155964D93F5
:10D510005D936D937C935897F9018385887161F4CD
:10D52000F701848D958DA68DB78DF801818B928B37
:10D53000A38BB48B81E010C0803141F598012F5E40
:10D540003F4FD80159968D919C915A970E94D7636D
:10D550008823E1F084E0F80183838C2D8F70D8015B
:10D5600011968C931197F8011482158216821782F6
:10D5700018961D921D921D921C921B97C4FEB5C059
:10D58000C8010F94FB028111B0C082CFD80113965D
:10D590001C927ECFD70113968C911397823009F499
:10D5A00077CF51968D919D910D90BC91A02D803E8D
:10D5B0009F4FAF41B10508F06BCFC7010E9478655E
:10D5C000882309F465CF0E943767882309F460CF68
:10D5D000D70159962D913C915A9714968D919D9112
:10D5E0000D90BC91A02D0297A109B109F901058404
:10D5F00004C0880F991FAA1FBB1F0A94D2F7468444
:10D60000578460887188480E591E6A1E7B1E81E00F
:10D610008093321A40922A1A50922B1A60922C1A36
:10D6200070922D1A80E092E0EAE2F8E1DF019C01BD
:10D630001D9221503040E1F7DD24D394D701599653
:10D64000ED91FC915A978481D81698F42AE238E13A
:10D65000B301A2014D0D511D611D711D8091331A41
:10D660009091341A0E94D466882309F411CFD39480
:10D67000E5CF80E092E0A0E0B0E0058404C0880F30
:10D68000991FAA1FBB1F0A94D2F7F701418952893B
:10D6900063897489840F951FA61FB71F818B928B96
:10D6A000A38BB48B8AE298E1D12C20E2DC011D929D
:10D6B0002A95E9F72BE0F501DC0101900D922A95FE
:10D6C000E1F721E238E2FC01318B208B40E058E0A9
:10D6D00057874687338B228B318F208F578B468B12
:10D6E0000E9437678111D8CED3CEC5FE09C0F8019C
:10D6F0004189528963897489C8010E943E6405C0CA
:10D7000081E003C09110A6CE93CE0F90DF91CF9110
:10D710001F910F91FF90EF90DF90CF90BF90AF904F
:10D720009F907F906F905F904F9008952F923F92BF
:10D730004F925F926F927F928F929F92AF92BF9221
:10D74000CF92DF92EF92FF920F931F93CF93DF93CD
:10D75000CDB7DEB7C254D1090FB6F894DEBF0FBE05
:10D76000CDBF4C015B016A01322E19821C821C8ED6
:10D770001F8E6115710511F410E0A6C0FC018381B4
:10D780008111FACFFA0180818F3209F09BC0F50137
:10D7900083818250823010F485010CC0F501618DC7
:10D7A000728DCE014C960E94D564882329F38E0198
:10D7B000045E1F4FC6016C010196F60120812F32D5
:10D7C000D1F3CE0101967C013C012E019CE1490E72
:10D7D000511C2396EFAE23972F2C9BE09150E7E34B
:10D7E000F0E0EC0FFD1FE90FF11D80E28083911145
:10D7F000F5CF960147E0D9018D91882369F18F32E9
:10D8000059F18E3239F44A3009F4B6CF98E04AE043
:10D810009D01F1CFE9ECF2E12491222321F0319630
:10D820008213FACFA9CF491708F4A6CF813208F4A2
:10D83000A3CF8F3709F4A0CF21E0290FE7E3F0E071
:10D84000EC0FFD1FE90FF11D9FE9980F9A3108F4C5
:10D8500080528083922FDCCF8FA9803209F48CCF45
:10D860006901F90180812F5F3F4F8F32C9F388230F
:10D87000F9F021E0AE01495C5F4FB801C7010E9499
:10D88000A769882309F478CF0A151B0519F0C80188
:10D890000E94AA676E147F0441F023969FAD2397E0
:10D8A000822D8701E92EF82E98CF942D852DF9CF62
:10D8B000232DAE01495C5F4FB801C4010E94A769E6
:10D8C000182F02C08B017DCFCE014C960E94B3670A
:10D8D000CE0101960E94B367812FCE5BDF4F0FB65A
:10D8E000F894DEBF0FBECDBFDF91CF911F910F9196
:10D8F000FF90EF90DF90CF90BF90AF909F908F9070
:10D900007F906F905F904F903F902F900895CF93AE
:10D91000C82F0F94350A84E50E94AA526C2F70E03C
:10D9200080E090E00E941E5380E20E94AA5287EBA2
:10D9300092E1CF910D944C092F923F924F925F92BA
:10D940006F927F928F929F92AF92BF92CF92DF920F
:10D95000EF92FF920F931F93CF93DF93CDB7DEB774
:10D96000CD58D1090FB6F894DEBF0FBECDBF5B0115
:10D970006A011901E996FFAEEEAEE9972091B81061
:10D980003091B9104091BA105091BB10DC016D91EB
:10D990007D918D919C910F94671E0F9464272B01AC
:10D9A0003C0125966CAF7DAF8EAF9FAF2597209140
:10D9B000BC103091BD104091BE105091BF10F501C8
:10D9C00060817181828193810F94671E0F94642717
:10D9D0004B015C0129966CAF7DAF8EAF9FAF29974D
:10D9E0002091C0103091C1104091C2105091C310CD
:10D9F000D6016D917D918D919C910F94671E0F942E
:10DA000064276B017C012D966CAF7DAF8EAF9FAF0D
:10DA10002D972091C4103091C5104091C61050919F
:10DA2000C710F10160817181828193810F94671E1B
:10DA30000F94642767966CAF7DAF8EAF9FAF6797EB
:10DA400061966CAF7DAF8EAF9FAF61978091A31051
:10DA500083FF0EC067962CAD3DAD4EAD5FAD6797B1
:10DA60002093BC153093BD154093BE155093BF1540
:10DA70008091A1109091A210892B11F00C948C7AB6
:10DA8000D801BC91A896BFAFA897F801F181AC96D8
:10DA9000FFAFAC97D8011296BC91E096BFAFE0976C
:10DAA000F801038180919A1590919B15891B8F70C5
:10DAB0008F3021F480E00E94D653F4CFF0919A1574
:10DAC000C557DF4FF883CB58D04080919A15282E48
:10DAD000312C8091B0159091B115A091B215B091F3
:10DAE000B315481A590A6A0A7B0A8091B4159091B5
:10DAF000B515A091B615B091B715A5019401281BD5
:10DB0000390B4A0B5B0B6B962CAF3DAF4EAF5FAF43
:10DB10006B978091B8159091B915A091BA15B091F5
:10DB2000BB15A7019601281B390B4A0B5B0B6F969F
:10DB30002CAF3DAF4EAF5FAF6F978091BC1590910A
:10DB4000BD15A091BE15B091BF156796CCACDDACEC
:10DB5000EEACFFAC6797C81AD90AEA0AFB0A09F4C7
:10DB600072C08091090C811128C060910E0C7091D7
:10DB70000F0C8091100C9091110C0F946326209142
:10DB8000190230911A0262177307BCF467968CADC4
:10DB90009DADAEADBFAD67978093BC159093BD159D
:10DBA000A093BE15B093BF150F94350A8EE293E192
:10DBB0000F944C09C12CD12C7601C701B6010F94EA
:10DBC000081E2091150230911602409117025091C3
:10DBD00018020F94671E4B015C0120E030E0A901A0
:10DBE0000F94572787FF04C0B7FAB094B7F8B094E2
:10DBF00020E030E04AEF53E46091C4107091C5100A
:10DC00008091C6109091C7100F94671EA5019401D2
:10DC10000F94011E87FF17C067962CAD3DAD4EAD2A
:10DC20005FAD67972093BC153093BD154093BE152B
:10DC30005093BF150F94350A8FE093E10F944C0970
:10DC4000C12CD12C7601D301C2018827B7FD839561
:10DC50009927AA27BB27182F6B962CAD3DAD4EAD4B
:10DC60005FAD6B9757FD12606F968CAD9DADAEADFD
:10DC7000BFAD6F97B7FD1460F7FC1860C701B60120
:10DC80000F94081E20911502309116024091170240
:10DC9000509118020F94671E6B017C0120E030E068
:10DCA000A9010F94572787FF04C0C701B6019058F8
:10DCB00002C0C701B60120E030E040E05FE30F940E
:10DCC000F7240F946A26E7966CAF7DAF8EAF9FAFB7
:10DCD000E79788E4829DF001839DF00D1124EF5DAC
:10DCE000F34F108215AB5301420177FE07C0882421
:10DCF0009924540184189508A608B70888E4829DE1
:10DD0000F001839DF00D1124EF5DF34F858A968A13
:10DD1000A78AB08E6B962CAD3DAD4EAD5FAD6B97C7
:10DD200067962CAF3DAF4EAF5FAF679757FF0DC003
:10DD300050954095309521953F4F4F4F5F4F6796D7
:10DD40002CAF3DAF4EAF5FAF679788E4829DF00187
:10DD5000839DF00D1124EF5DF34F67968CAD9DAD63
:10DD6000AEADBFAD6797818F928FA38FB48F6F9643
:10DD70002CAD3DAD4EAD5FAD6F97A3962CAF3DAFD3
:10DD80004EAF5FAFA39757FF0DC0509540953095AC
:10DD900021953F4F4F4F5F4FA3962CAF3DAF4EAFF6
:10DDA0005FAFA39788E4829DF001839DF00D11245D
:10DDB000EF5DF34FA3968CAD9DADAEADBFADA39718
:10DDC000858F968FA78FB0A3C301B2010F94081E51
:10DDD0002091F90B3091FA0B4091FB0B5091FC0B09
:10DDE0000F94671EA7966CAF7DAF8EAF9FAFA797BE
:10DDF00069AB7AAB8BAB9CAB6B966CAD7DAD8EADEE
:10DE00009FAD6B970F94081E2091FD0B3091FE0B78
:10DE10004091FF0B5091000C0F94671E2B013C01A9
:10DE20006DAB7EAB8FAB98AF6F966CAD7DAD8EADAD
:10DE30009FAD6F970F94081E2091010C3091020C3A
:10DE40004091030C5091040C0F94671E6B966CAFBD
:10DE50007DAF8EAF9FAF6B9769AF7AAF8BAF9CAF43
:10DE60002091050C3091060C4091070C5091080C44
:10DE7000C701B6010F94671E6B017C0121966CAF40
:10DE80007DAF8EAF9FAF219796E089169104A104D4
:10DE9000B1041CF567962CAD3DAD4EAD5FAD6797F7
:10DEA0002630310541055105C4F4A3968CAD9DADD6
:10DEB000AEADBFADA3970697A105B10574F420E000
:10DEC00030E0A901C701B6010F94572787FF16C09C
:10DED000F7FAF094F7F8F09411C0E996AEADBFAD43
:10DEE000E997CD90DD90ED90FC9020E030E0A90125
:10DEF000C701B6010F94011E882369F088E4829D52
:10DF0000F001839DF00D1124EF5DF34FC586D68699
:10DF1000E786F08A38C0A7962CAD3DAD4EAD5FAD1B
:10DF2000A797CA01B9010F94671E6B017C01A30179
:10DF30009201C301B2010F94671E9B01AC01C7019E
:10DF4000B6010F94F7246B017C016B962CAD3DADAF
:10DF50004EAD5FAD6B97CA01B9010F94671E9B016F
:10DF6000AC01C701B6010F94F7240F94A52728E44C
:10DF7000229DF001239DF00D1124EF5DF34F658785
:10DF800076878787908B88E4829DF001839DF00DD2
:10DF90001124EF5DF34FE7962CAD3DAD4EAD5FAD77
:10DFA000E79721A332A343A354A3582D492D3A2D1B
:10DFB0002B2D67968CAD9DADAEADBFAD6797881626
:10DFC0009906AA06BB0660F464965FAD64976596F1
:10DFD0004FAD659766963FAD669767962FAD67978D
:10DFE000852F942FA32FB22FA3962CAD3DAD4EAD10
:10DFF0005FADA39782179307A407B50710F4DA0162
:10E00000C901E7962CAD3DAD4EAD5FADE7978217E8
:10E010009307A407B50710F4DA01C90128E4229D8B
:10E02000F001239DF00D1124EF5DF34F85A396A31E
:10E03000A7A3B0A70697A105B10510F40C941A7B0D
:10E04000DF01AA5BBF4F8091F70B8C93E95BFF4F19
:10E050008091F80B808389288A288B2809F05F98A3
:10E0600088E4829DF001839DF00D1124EF5DF34F54
:10E07000818D928DA38DB48D892B8A2B8B2B09F0EA
:10E080008A9888E4829DF001839DF00D1124EF5D54
:10E09000F34F858D968DA78DB0A1892B8A2B8B2B65
:10E0A00029F080910801817080930601E7968CAD7C
:10E0B0009DADAEADBFADE797892B8A2B8B2B11F4AD
:10E0C0000C948E7A8091FC10882319F081508093F3
:10E0D000FC10129880E28093FC10D090E410E09045
:10E0E000E510F090E6101091E7102D2D3E2D4F2DEC
:10E0F000512FA8966FADA897AC967FADAC97E096E0
:10E100008FADE097902F0F94011E87FF0AC0A8964D
:10E11000DFAEA897AC96EFAEAC97E096FFAEE09777
:10E12000012F88E4829DF001839DF00D1124EF5DA5
:10E13000F34F2585368547855089EB962CAF3DAF4B
:10E140004EAF5FAFEB9760E070E080E89FE30F9425
:10E15000F125A7966CAF7DAF8EAF9FAFA797A8961E
:10E160002FADA897AC963FADAC97E0964FADE0973A
:10E17000502F0F94671E4B015C0180919A1590916E
:10E180009815891B8F70EC968FAFEC97A5019401C1
:10E1900060E074E284E799E40F94F1250F9464271A
:10E1A0006B017C01EC968FADEC9782508630C0F508
:10E1B0008091B4109091B510A091B610B091B710A5
:10E1C000C816D906EA06FB0658F58C199D09AE0952
:10E1D000BF09BC01CD01660F771F881F991FEC9600
:10E1E0004FADEC97042F10E020E030E0A90198013A
:10E1F0000F945724CA01B9010F94061E0F94642787
:10E200006C0D7D1D8E1D9F1D0F94061E9B01AC0184
:10E2100060E074E284E799E40F94F1254B015C011E
:10E22000A5019401EB966CAD7DAD8EAD9FADEB97E6
:10E230000F94671E9B01AC010F94671EC158DF4FFE
:10E24000688379838A839B83CF57D04088E4829DFB
:10E250008001839D100D11240F5D134FC158DF4FB6
:10E2600088819981AA81BB81CF57D040F8018183F1
:10E270009283A383B48325A136A147A150A5AB9671
:10E280002CAF3DAF4EAF5FAFAB97CA01B9010F9452
:10E29000061EAF966CAF7DAF8EAF9FAFAF979B0161
:10E2A000AC01C501B4010F94671E0F94D5250F94DE
:10E2B0006A26CD57DF4F688379838A839B83C3584F
:10E2C000D040F80166AB77AB80AF91AF8E010F5CA9
:10E2D0001F4F9E012F5D3F4FE1963FAF2EAFE1975D
:10E2E00048EC50E1C757DF4F59834883C958D040A5
:10E2F000C8014096C457DF4F99838883CC58D040DB
:10E30000C957DF4F39832883C758D04064961FAE62
:10E31000649768961FAE689790E86C969FAF6C976D
:10E32000AFE3A096AFAFA097F80121913191419151
:10E3300051918F01C501B4010F94671E6B017C01DF
:10E34000C957DF4FA881B981C758D0406D937D93DD
:10E350008D939D93C957DF4FB983A883C758D04089
:10E3600020E030E0A9010F94572787FF04C0F7FA97
:10E37000F094F7F8F094C757DF4FE881F981C95856
:10E38000D0404190519061907190C757DF4FF98311
:10E39000E883C958D040A7019601C301B2010F9488
:10E3A000011E87FF24C0A7019601C301B2010F948B
:10E3B000F1257B016C0164962FAD649768963FADA3
:10E3C00068976C964FAD6C97A0965FADA0970F9431
:10E3D000011E87FF0CC06496EFAE64976896FFAE8F
:10E3E00068976C96CFAE6C97A096DFAEA097C45797
:10E3F000DF4F28813981CC58D0402017310709F0F0
:10E4000093CF20E030E040E85FE364966FAD64971F
:10E4100068967FAD68976C968FAD6C97A0969FAD10
:10E42000A0970F94011E87FF7AC08E010F5C1F4FCB
:10E4300064962FAD649768963FAD68976C964FAD24
:10E440006C97A0965FADA097E196AEADBFADE1979A
:10E450006D917D918D919C910F94671EE196EEAD2B
:10E46000FFADE1976193719381939193E196FFAF33
:10E47000EEAFE1970E171F07D9F688E4829D800161
:10E48000839D100D11240F5D134FCD57DF4F688111
:10E4900079818A819B81C358D0400F94061E64966F
:10E4A0002FAD649768963FAD68976C964FAD6C97AB
:10E4B000A0965FADA0970F94671E0F946A26D801AF
:10E4C000D6966D937D938D939C93D99764962FAD3B
:10E4D000649768963FAD68976C964FAD6C97A09621
:10E4E0005FADA09764966FAD649768967FAD6897AF
:10E4F0006C968FAD6C97A0969FADA0970F94671EFA
:10E50000C158DF4F288139814A815B81CF57D04084
:10E510000F94671EF8016183728383839483AF969F
:10E520002CAD3DAD4EAD5FADAF97A7966CAD7DAD5B
:10E530008EAD9FADA7970F94671E67966CAF7DAFAA
:10E540008EAF9FAF679788E4829DF001839DF00DA9
:10E550001124EF5DF34F85889688A788B08C8114CD
:10E560009104A104B10419F5818D928DA38DB48D10
:10E57000892B8A2B8B2BD9F4858D968DA78DB0A1F5
:10E58000892B8A2B8B2B99F42091DC103091DD1094
:10E590004091DE105091DF1067966CAD7DAD8EAD71
:10E5A0009FAD67970F94671E0F94D5252BC2E796F2
:10E5B0002CAD3DAD4EAD5FADE797232B242B252B26
:10E5C00049F02091D8103091D9104091DA10509133
:10E5D000DB1008C02091E0103091E1104091E21072
:10E5E0005091E31067966CAD7DAD8EAD9FAD679792
:10E5F0000F94671E0F94D5250F946A266B017C013A
:10E600008091F30B9091F40BA091F50BB091F60B68
:10E61000AB962CAD3DAD4EAD5FADAB97821793077A
:10E62000A407B50708F4D6C081149104A104B1046D
:10E6300011F16091E30B7091E40B8091E50B9091E7
:10E64000E60B6C157D058E059F05A8F40F944724F5
:10E650002B013C01A5019401C701B6010F94472489
:10E66000461657066806790630F4C301B2010F94C6
:10E67000572469017A0188E4829DF001839DF00DA1
:10E680001124EF5DF34F818C928CA38CB48C811498
:10E690009104A104B10441F16091E70B7091E80B82
:10E6A0008091E90B9091EA0B6C157D058E059F0515
:10E6B000D8F4AB962CAD3DAD4EAD5FADAB970F949E
:10E6C00047242B013C01A5019401C701B6010F9419
:10E6D0004724461657066806790630F4C301B2018E
:10E6E0000F94572469017A0188E4829DF001839D8B
:10E6F000F00D1124EF5DF34F858C968CA78CB0A0A4
:10E7000081149104A104B10441F16091EB0B70916B
:10E71000EC0B8091ED0B9091EE0B6C157D058E0549
:10E720009F05D8F4AB962CAD3DAD4EAD5FADAB972C
:10E730000F9447242B013C01A5019401C701B601A8
:10E740000F944724461657066806790630F4C3012D
:10E75000B2010F94572469017A0188E4829DF00187
:10E76000839DF00D1124EF5DF34F81A092A0A3A033
:10E77000B4A081149104A104B10409F447C16091CB
:10E78000EF0B7091F00B8091F10B9091F20B6C15E7
:10E790007D058E059F0508F039C1AB962CAD3DADCA
:10E7A0004EAD5FADAB970F9447242B013C01A50103
:10E7B0009401C701B6010F94472446165706680610
:10E7C000790608F023C1C301B2010F9457246901EF
:10E7D0007A011CC181149104A104B104C9F16091B2
:10E7E000E30B7091E40B8091E50B9091E60B6C15B7
:10E7F0007D058E059F0560F50F94061EAF962CAD26
:10E800003DAD4EAD5FADAF970F94671E2B013C0140
:10E81000C501B4010F94061E4B015C01C701B6018E
:10E820000F94061EA50194010F94671E9B01AC0175
:10E83000C301B2010F94011E87FF0AC0A501940114
:10E84000C301B2010F94F1250F946A266B017C017C
:10E8500088E4829DF001839DF00D1124EF5DF34F5C
:10E86000418C528C638C748C41145104610471048A
:10E87000C9F16091E70B7091E80B8091E90B9091E1
:10E88000EA0B6C157D058E059F0560F50F94061E3D
:10E89000AF962CAD3DAD4EAD5FADAF970F94671EFB
:10E8A0004B015C01C301B2010F94061E2B013C0118
:10E8B000C701B6010F94061EA30192010F94671EB3
:10E8C0009B01AC01C501B4010F94011E87FF0AC072
:10E8D000A3019201C501B4010F94F1250F946A269A
:10E8E0006B017C0188E4829DF001839DF00D112471
:10E8F000EF5DF34F458C568C678C70A0411451042A
:10E9000061047104C9F16091EB0B7091EC0B809183
:10E91000ED0B9091EE0B6C157D058E059F0560F556
:10E920000F94061EAF962CAD3DAD4EAD5FADAF97CB
:10E930000F94671E4B015C01C301B2010F94061EC8
:10E940002B013C01C701B6010F94061EA3019201E1
:10E950000F94671E9B01AC01C501B4010F94011E09
:10E9600087FF0AC0A3019201C501B4010F94F125EC
:10E970000F946A266B017C0188E4829DF001839DDF
:10E98000F00D1124EF5DF34F81A092A0A3A0B4A0DD
:10E9900081149104A104B104C9F16091EF0B70914D
:10E9A000F00B8091F10B9091F20B6C157D058E05AB
:10E9B0009F0560F50F94061EAF962CAD3DAD4EAD94
:10E9C0005FADAF970F94671E2B013C01C501B401E9
:10E9D0000F94061E4B015C01C701B6010F94061E81
:10E9E000A50194010F94671E9B01AC01C301B20104
:10E9F0000F94011E87FF0AC0A5019401C301B20153
:10EA00000F94F1250F946A266B017C0188E4829DA6
:10EA10008001839D100D11240F5D134FF801EE5BF3
:10EA2000FF4FC082D182E282F382C701B6010F9408
:10EA3000061E6B017C0167962CAD3DAD4EAD5FAD02
:10EA400067970F94F125AB966CAF7DAF8EAF9FAFFC
:10EA5000AB97D80151966D937D938D939C9354976A
:10EA60002DEB37E346E051E4C701B6010F94671E72
:10EA70000F946A26F80161AB72AB83AB94AB29A902
:10EA80003AA94BA95CA9A7966CAD7DAD8EAD9FADA3
:10EA9000A7970F94671EAF966CAF7DAF8EAF9FAFF9
:10EAA000AF97698B7A8B8B8B9C8B2DA93EA94FA935
:10EAB00058ADA7966CAD7DAD8EAD9FADA7970F9469
:10EAC000671E4B015C016D8B7E8B8F8B988F29AD00
:10EAD0003AAD4BAD5CADA7966CAD7DAD8EAD9FAD47
:10EAE000A7970F94671E6B017C01698F7A8F8B8FBC
:10EAF0009C8F21962CAD3DAD4EAD5FAD2197A79675
:10EB00006CAD7DAD8EAD9FADA7970F94671EA79698
:10EB10006CAF7DAF8EAF9FAFA7976D8F7E8F8F8FBE
:10EB200098A3EC96FFADEC97FF2309F4BBC22091AC
:10EB30009C1564962FAF649730919D1568963FAFF2
:10EB4000689740919E156C964FAF6C9750919F15AA
:10EB5000A0965FAFA0972DEB37E346E855E36496A8
:10EB60006FAD649768967FAD68976C968FAD6C9724
:10EB7000A0969FADA0970F94011E87FD93C2809130
:10EB8000EC109091ED10A091EE10B091EF10E7967F
:10EB90008CAF9DAFAEAFBFAFE7972091F010309133
:10EBA000F1104091F2105091F310E3962CAF3DAF6D
:10EBB0004EAF5FAFE3978091F4109091F510A09164
:10EBC000F610B091F710EF968CAF9DAFAEAFBFAF20
:10EBD000EF972091F8103091F9104091FA10509170
:10EBE000FB10C158DF4F288339834A835B83CF579B
:10EBF000D040E7966CAD7DAD8EAD9FADE797905858
:10EC0000AF962CAD3DAD4EAD5FADAF970F94671E87
:10EC10002B013C01E3962CAD3DAD4EAD5FADE397CE
:10EC2000C501B4010F94671E9B01AC01C301B20181
:10EC30000F94F6242B013C01EF962CAD3DAD4EAD6B
:10EC40005FADEF97C701B6010F94671E9B01AC0142
:10EC5000C301B2010F94F6242B013C01C158DF4FD0
:10EC6000288139814A815B81CF57D040A7966CAD0E
:10EC70007DAD8EAD9FADA7970F94671E9B01AC0134
:10EC8000C301B2010F94F6242B013C012FEE3FEF9C
:10EC90004FE75FE30F94572718160CF4B2C12FEE1D
:10ECA0003FEF4FE75FEBC301B2010F94011E87FFF7
:10ECB00008C0EFEE4E2E55245A94EFE76E2EEFEB80
:10ECC0007E2EE7962CAD3DAD4EAD5FADE797AF968E
:10ECD0006CAD7DAD8EAD9FADAF970F94F62469837B
:10ECE0007A838B839C83E3962CAD3DAD4EAD5FADB7
:10ECF000E397C501B4010F94F6246D837E838F835F
:10ED00009887EF962CAD3DAD4EAD5FADEF97C70147
:10ED1000B6010F94F62469877A878B879C87C15840
:10ED2000DF4F288139814A815B81CF57D040A79638
:10ED30006CAD7DAD8EAD9FADA7970F94F6246D871A
:10ED40007E878F87988BAE014F5F5F4FA5965FAF31
:10ED50004EAFA597CE01419663969FAF8EAF639756
:10ED60008A01C12CD12C7601D8018D909D90AD9057
:10ED7000BD908D0120E030E0A901C501B4010F94E0
:10ED8000011E882371F0A5019401C501B4010F94FF
:10ED9000671E9B01AC01C701B6010F94F7246B01FC
:10EDA0007C016396EEADFFAD6397E017F107E1F6E6
:10EDB000C701B6010F94A5279B01AC0160E070E08C
:10EDC00080E89FE30F94F1256B017C01A5960EADC1
:10EDD0001FADA597A7019601D8016D917D918D91E9
:10EDE0009C910F94671EF8016193719381939193A5
:10EDF0008F0163962EAD3FAD63972E173F0751F7F6
:10EE000074EAA72E70E1B72EA8963FADA897AC96EE
:10EE10003FAFAC97A9964FADA997E4964FAFE49753
:10EE2000AA960FADAA97AB961FADAB97A596AEADC0
:10EE3000BFADA597CD90DD90ED90FD90A596BFAFAD
:10EE4000AEAFA59720E030E0A901C701B6010F944D
:10EE5000011E882361F1F5016081718182819381B6
:10EE60000F94061EA70196010F94F1256B017C01FA
:10EE700020E030E0A9010F94572787FF04C0F7FA7C
:10EE8000F094F7F8F094AC962FADAC97E4963FADC4
:10EE9000E497A801C701B6010F94011E87FF07C0C0
:10EEA000AC96CFAEAC97E496DFAEE4978701F4E082
:10EEB000AF0EB11C63962EAD3FAD6397A5964EADD8
:10EEC0005FADA5972417350709F0B0CFA3019201D4
:10EED00060E070E080E89FE30F94F62420E030E0EB
:10EEE00040E05FE30F94671E0F94A5276B017C0140
:10EEF0002091DF0B3091E00B4091E10B5091E20B40
:10EF0000AC966FADAC97E4967FADE497C8010F94D3
:10EF1000671EA70196010F94671E4B015C01A701B4
:10EF2000960160E070E080E89FE30F94F6249B0177
:10EF3000AC01C501B4010F94F1256B017C0120E007
:10EF400030E040E85FE3EB966CAD7DAD8EAD9FADFC
:10EF5000EB970F94011E87FF5CC0A3019201C301D0
:10EF6000B2010F94671E23EC38EB42E35FEB0F9482
:10EF7000671E23EF36E64FE55FE30F94F624A30107
:10EF800092010F94671E2BED3FE049EC5FE30F9475
:10EF9000F7242CEE31E548E35EE30F94F6244B01B1
:10EFA0005C0124EE3BEC46E150E40F945727181621
:10EFB00084F5A50194016BED7FE089E490E40F9462
:10EFC000F6249B01AC01EB966CAD7DAD8EAD9FAD93
:10EFD000EB970F94F125AC962FADAC97E4963FAD2F
:10EFE000E497A8010F94671E5B018C019B01AC01A3
:10EFF000B601C7010F94572718165CF46501780114
:10F0000008C03BE0C32E47EDD42E53E2E52E6BE360
:10F01000F62E88E4829DF001839DF00D1124EF5DB2
:10F02000F34FA180B280038114819501A8016496F9
:10F030006FAD649768967FAD68976C968FAD6C974F
:10F04000A0969FADA0970F945727181664F4649666
:10F05000AFAE64976896BFAE68976C960FAF6C972B
:10F06000A0961FAFA0979601A70164966FAD649715
:10F0700068967FAD68976C968FAD6C97A0969FADA4
:10F08000A0970F9457271816CCF46496CFAE6497C8
:10F090006896DFAE68976C96EFAE6C97A096FFAE61
:10F0A000A0970CC064961FAE649768961FAE6897D1
:10F0B0006C961FAE6C97A0961FAEA09780E1FE01E4
:10F0C0007196ACEEB0E101900D928A95E1F788E47B
:10F0D000829D8001839D100D11240F5D134F649656
:10F0E0008FAD649768969FAD68976C96AFAD6C973F
:10F0F000A096BFADA097F80181879287A387B487B8
:10F10000AB966CAD7DAD8EAD9FADAB9790589B012E
:10F11000AC010F94F724D8011D962D913D914D918E
:10F120005C9150970F94671E9B01AC016BE077EDEB
:10F1300083E29BE30F94F6242BE0C22E27EDD22E20
:10F1400023E2E22E2BE3F22EF801C582D682E7827B
:10F15000F086B080C180D280E380F480A701960160
:10F160000F94572787FD02C083E001C081E08B29FF
:10F1700098E4929DF001939DF00D1124EF5DF34F03
:10F18000808380E1FE01B196A0EAB5E101900D9285
:10F190008A95E1F7C0929C15D0929D15E0929E153C
:10F1A000F0929F1580E1FE01EF5BFF4FA0EBB5E110
:10F1B00001900D928A95E1F790919A1580919B1597
:10F1C000981303C084E680939715C557DF4F888155
:10F1D000CB58D0408F5F8F7080939A1580919A158D
:10F1E0009091991581508F70891709F4ABC0F090F8
:10F1F0009A158FEF8F0D8F7064968FAF6497E090A4
:10F20000991580919A15E81609F46BC0C12CD12C80
:10F210006496FFAD6497FE1509F463C08F2E912CA0
:10F2200028E4289D8001299D100D11240F5D134FA6
:10F23000D8018C9183FD32C0A4960FAFA497A896F5
:10F240001FAFA8971996BC916896BFAF6897F80151
:10F25000F2856C96FFAF6C97D8011B96BC91A09677
:10F26000BFAFA097F801F484258036804780508492
:10F27000A201910168966FAD68976C967FAD6C970F
:10F280008B2F9F2D0F94011E811152C1C114D104E7
:10F2900059F0D6018C9180FD4BC106C0A496CFAE2B
:10F2A000A497A896DFAEA89764968FAD6497815017
:10F2B0008F7064968FAF6497809199158E1107C0F7
:10F2C000A496CFACA497A896DFACA897A1CF6496DC
:10F2D000FFAD6497FE1529F081E08E0D8F70E82E4A
:10F2E000EBCF2091991564962FAF6497C12CD12C48
:10F2F00080919A1564963FAD6497831719F1832E18
:10F30000912C48E4489D8001499D100D11240F5D0A
:10F31000134FD8018C9183FD0AC05801C114D10448
:10F3200039F0C6010E94B39E811102C08AC1560104
:10F3300064968FAD64978F5F8F7064968FAF64977C
:10F340006501D6CFD0909B1580909A1528E4D814EB
:10F3500069F08FEF880D8F70289FF0011124EF5D09
:10F36000F34F908193FF02C0882EF1CF212C312CD6
:10F37000412C512C64961FAE649768961FAE689717
:10F38000712C612C00E010E0E12CF12C8D1409F4BB
:10F3900081C048E44D9D800111240F5D134FD801B9
:10F3A0008C9183FD19C015966D917D918D919C91E5
:10F3B00018970F94A527C62EB72EA82E992EE114C4
:10F3C000F10409F455C0F701808180FD0EC0D80119
:10F3D0008C9180FD0AC04CC06496CFAC649768964F
:10F3E000BFAC6897A72C962C48C0F701808181603C
:10F3F0008083C7010E94B39E811136C0F7016181ED
:10F400007281838194810F94A5279B01AC0160E0F8
:10F4100070E080E89FE30F94F1251B012C019B0114
:10F42000AC016C2D7B2D8A2D992D0F94671E69835D
:10F430007A838B839C8364962FAD649768963FADE7
:10F440006897472D562DC201B1010F94671E698B35
:10F450007A8B8B8B9C8BAE014F5F5F4FBE016F5ED3
:10F460007F4FC7010E942F8FD7018C918E7F8C9385
:10F470002C2C3B2C4A2C592C780181E08D0D8F705F
:10F48000D82E6496CFAE64976896BFAE68977A2CF4
:10F49000692C7CCF0115110509F4CCC0F8018081DD
:10F4A00081608083C7010E94B39E811130C0D80162
:10F4B00011966D917D918D919C9114970F94A52734
:10F4C0009B01AC0160E070E080E89FE30F94F125C0
:10F4D0006B017C012DEC3CEC4CE45DE30F94671E6A
:10F4E00069837A838B839C839101A201C701B60152
:10F4F0000F94671E698B7A8B8B8B9C8BAE014F5F51
:10F500005F4FBE016F5E7F4FC8010E942F8FF801D1
:10F5100080818E7F80838EC080E015C1D090E810FE
:10F52000E090E910F090EA101091EB100C947570D7
:10F5300028E4289DF001299DF00D1124EF5DF34F83
:10F54000808181FD45C0C114D10431F0F601A58050
:10F55000B680C780D08408C08BE0A82E87EDB82E77
:10F5600083E2C82E8BE3D82E28E4289DF001299D44
:10F57000F00D1124EF5DF34F81899289A389B4893D
:10F58000BC01CD0190589B01AC010F94F724D80128
:10F590001D962D913D914D915C9150970F94671E52
:10F5A0009B01AC01C601B5010F94F6243B015C013F
:10F5B0009B01AC0168966FAD68976C967FAD6C97B8
:10F5C000A0968FADA0979F2D0F94011E87FF0AC0B4
:10F5D00068966FAC68976C967FAC6C97A096AFAC52
:10F5E000A097BF2C9301A501C201B1010F94011E88
:10F5F000882309F459CEB8E4B89DC001B99D900D97
:10F600001124FC01EF5DF34F6F01808181608083E5
:10F61000C8010E94B39E882329F0D6018C918E7F69
:10F620008C9342CEC301D501F60185839683A783CF
:10F63000B0873ACE80916F00826080936F0081E046
:10F6400082C0D6018C9181FD58C0D60115962D91AE
:10F650003D914D915C9118976B962CAF3DAF4EAF9D
:10F660005FAF6B971501B5E02B0E311CF80145809B
:10F67000568067807084A30192016B966CAD7DAD5E
:10F680008EAD9FAD6B970F94011E87FF36C0F601BC
:10F6900081899289A389B489BC01CD0190589B01CD
:10F6A000AC010F94F724D6011D962D913D914D91FB
:10F6B0005C9150970F94671E9B01AC016B966CADEB
:10F6C0007DAD8EAD9FAD6B970F94F6246B017C01E1
:10F6D0009B01AC01C301B2010F94572718166CF4BB
:10F6E000D8018C9181608C93C5010E94B39E8823C0
:10F6F000F1F0F80180818E7F808328E4289DF0015D
:10F70000299DF00D1124EF5DF34F2185328543854E
:10F71000548565817681878190850F94011E8111C2
:10F7200007CE64963FAD64973093991501CED10111
:10F73000CD92DD92ED92FC9213976496BFAD6497E3
:10F74000B0939915DACFC357DF4F0FB6F894DEBFE9
:10F750000FBECDBFDF91CF911F910F91FF90EF9022
:10F76000DF90CF90BF90AF909F908F907F906F90E1
:10F770005F904F903F902F900895CF92DF92EF923D
:10F78000FF920F931F93CF93DF93CDB7DEB76497AC
:10F790000FB6F894DEBF0FBECDBFC98ADA8AEB8AF6
:10F7A000FC8AFC0180819181A281B38189839A8343
:10F7B000AB83BC83FB0180819181A281B3818D8366
:10F7C0009E83AF83B887FA0180819181A281B38142
:10F7D00089879A87AB87BC87F90180819181A28153
:10F7E000B3818D879E87AF87B88BAE01475F5F4F30
:10F7F000BE016B5F7F4FCE0101960E94548E8091B7
:10F80000A1109091A210892B81F4CE0141967C0128
:10F810009E01235F3F4FAE01475F5F4FBE016B5FAD
:10F820007F4F40970E949C6C01C080E064960FB6A9
:10F83000F894DEBF0FBECDBFDF91CF911F910F9126
:10F84000FF90EF90DF90CF900895CF93DF93CDB7E7
:10F85000DEB760970FB6F894DEBF0FBECDBFEDE008
:10F86000F8E180819181A281B38189839A83AB83FE
:10F87000BC8384819581A681B7818D839E83AF836C
:10F88000B88780859185A285B38589879A87AB875C
:10F89000BC8784859585A685B7858D879E87AF872C
:10F8A000B88BAE01475F5F4FBE016B5F7F4FCE01EC
:10F8B00001960E94548E9E01235F3F4FAE01475F29
:10F8C0005F4FBE016B5F7F4FCE0101960E94B58CEA
:10F8D00060960FB6F894DEBF0FBECDBFDF91CF911B
:10F8E00008950F94350A6091DD0B7091DE0B8CEF5B
:10F8F00092E10F941E0A89EF92E10D944C099091C8
:10F90000DB0B9817C9F08093DB0B811109C0809144
:10F91000D90B8093F70B8091DA0B8093F80B089545
:10F920008091F70B8093D90B1092F70B8091F80B15
:10F930008093DA0B1092F80B0895CF93DF93CDB735
:10F94000DEB78091D70B81110FC09E01275F3F4F1B
:10F950004F8158856FE370E087E99BE00F94C81DE5
:10F9600087E99BE00E948DCFDF91CF9108951F938F
:10F97000CF93DF938091960BC82FC270D82FD4708D
:10F98000182F117080FF04C0CC2311F0D11145C095
:10F990000F94350A83EF92E10F944C09111103C0C3
:10F9A00088E50E94AA52C11103C089E50E94AA52AB
:10F9B000D11103C08AE50E94AA528BEE92E10F9406
:10F9C0004C09DD2319F04FEA55E002C046E458E047
:10F9D000CC2319F02FEA35E002C022E736E01123EC
:10F9E00019F08FEA95E002C084E796E05F934F93A9
:10F9F0003F932F939F938F9389ED92E19F938F93E2
:10FA00001F920E949D7C8DB79EB709960FB6F89401
:10FA10009EBF0FBE8DBF81E001C080E0DF91CF911E
:10FA20001F910895AF92BF92CF92DF92EF92FF9213
:10FA30000F931F93CF93DF93CDB7DEB72C970FB6FD
:10FA4000F894DEBF0FBECDBF2DEDC22E22E0D22E28
:10FA50005C0170E0CB0183529D4F7C01CE14DF042A
:10FA600009F180E20E94AA52F60181916F010E9481
:10FA7000AA528AE30E94AA52F50161917191819183
:10FA800091915F018E010F5F1F4F23E041E00F94C2
:10FA9000D9188C01F80181918F018823F9F20E9415
:10FAA000AA52F8CF8AE00E94AA522C960FB6F89478
:10FAB000DEBF0FBECDBFDF91CF911F910F91FF90A1
:10FAC000EF90DF90CF90BF90AF9008952F923F922C
:10FAD0004F925F926F927F928F929F92AF92BF925E
:10FAE000CF92DF92EF92FF920F931F93CF93DF930A
:10FAF000CDB7DEB7C154D1090FB6F894DEBF0FBE43
:10FB0000CDBF2DB73EB73FA72EA70E94B77C81116E
:10FB10004FC461E086E50E9460A78D8B853018F0A8
:10FB200080EF94E179C03D89332321F080ED94E1A9
:10FB30000F944C096AE080E50E9460A7182F8CEFB3
:10FB4000810F8F3218F08CEA94E166C060E085E4A2
:10FB50000E94F793811103C082E08FA302C091E05D
:10FB60009FA360910D1870910E1880910F189091BD
:10FB700010186D837E838F839887C0901118D09062
:10FB80001218E0901318F0901418C986DA86EB86E4
:10FB9000FC862091FF133091001440910114509184
:10FBA00002140F94F724AB01BC0188E50E94FCCF3E
:10FBB0006D877E878F87988B29853A854B855C85F5
:10FBC00060910314709104148091051490910614AF
:10FBD0000F94F724AB01BC0189E50E94FCCF698B2F
:10FBE0007A8B8B8B9C8BBE016F5E7F4FCE010D9607
:10FBF0000E941CA6811103C084E994E10DC08CE42D
:10FC00000E94A193082F882381F00E9442938E8B3B
:10FC1000803128F081E694E10F944C09C9C3AE8984
:10FC2000A13021F4B2E0BE8B01C01E8A60E083E502
:10FC30000E94F7938CAB882321F0011102C0E7E00A
:10FC4000EE8BFD89F33020F087E494E10F944C09AA
:10FC5000209125182BAF80E00F94C2060E949DC111
:10FC6000812F90E09EAB8DABADB7BEB7E4E01E9F99
:10FC7000A019B10911240FB6F894BEBF0FBEADBFD5
:10FC80002DB73EB72F5F3F4F3DA72CA72D894FA122
:10FC9000BE016F5E7F4FCE010D960E945BFB9B0104
:10FCA000AC010F94E9278111ECC20F940601611594
:10FCB00071058105910511F00F94921933EF3F8B77
:10FCC0008FE4888F93EC998F37EC232EA3EFAA8FC4
:10FCD000BFE4BB8FE3ECEC8FF7E4FD8F1EA233246F
:10FCE0003394412C512C32014AA25BA26CA27DA21A
:10FCF0002E89822F90E0DC0111972296BFAFAEAF24
:10FD00002297FEA1EF2FF0E0FF8FEE8F2DA93EA9E5
:10FD1000E217F3070CF0CDC23E89332309F46EC11C
:10FD20000F9444192AE030E040E050E00F94792429
:10FD30000F94081E20E030E040EA50E40F9457276B
:10FD400018161CF001E010E002C00FEF1FEF0F9437
:10FD5000441928E631E040E050E00F9479240F94F4
:10FD6000081E4B015C010F94441923E330E040E08E
:10FD700050E00F9479246B5F7F4F8F4F9F4F0F940C
:10FD8000081E68A779A78AA79BA78D898430E1F40C
:10FD900048A559A56AA57BA589E394E10F94000ABB
:10FDA000B501A40181E394E10F94000A8BE294E190
:10FDB0000F944C090130110519F483E40E94AA52F2
:10FDC00087E294E10F944C09312CC801110FAA0B62
:10FDD000BB0B8FAB98AFA9AFBAAF832D90E0229643
:10FDE000AEADBFAD22978A179B070CF007C1BCA927
:10FDF000BB2379F06FA978AD89AD9AAD0F94081E39
:10FE00009B01AC010F94F72420E030E040E952E47C
:10FE10001AC00F94441924E130E040E050E00F9400
:10FE20007924675E7F4F8F4F9F4F0F94081E6B01A1
:10FE30007C016FA978AD89AD9AAD0F94081E9B0126
:10FE4000AC01C701B6010F94671E9B01AC01C5014F
:10FE5000B4010F94F7244B015C0120E030E044EB47
:10FE600053E40F94572718164CF420E030E044EB8D
:10FE700053E4C501B4010F94F624EDCF20E030E047
:10FE8000A901C501B4010F94011E87FF0BC020E03A
:10FE900030E044EB53E4C501B4010F94F7244B0167
:10FEA0005C01ECCF2BED3FE049E450E4C501B40127
:10FEB0000F94671E20E030E044E353E40F94F125F3
:10FEC0006B017C010F94EC2568AB79AB8AAB9BABE3
:10FED0002091FF13309100144091011450910214AD
:10FEE0006D857E858F8598890F94F6246CAF7DAFE4
:10FEF0008EAF9FAF28A939A94AA95BA968A579A5A2
:10FF00008AA59BA50F94671E9B01AC016CAD7DADCE
:10FF10008EAD9FAD0F94F7246D837E838F8398877A
:10FF2000C701B6010F94972768AB79AB8AAB9BAB3F
:10FF3000209103143091041440910514509106143B
:10FF400069897A898B899C890F94F6246B017C01DD
:10FF500028A939A94AA95BA968A579A58AA59BA55D
:10FF60000F94671E9B01AC01C701B6010F94F724E3
:10FF700069877A878B879C874BED51E060E070E062
:10FF8000CE0105960E94EA9942EC51E060E070E0F3
:10FF9000CE0109960E94EA99ED89E430F9F44D8189
:10FFA0005E816F8178858BE194E10F94000A498529
:10FFB0005A856B857C8588E194E10F94000A409115
:10FFC000151850911618609117187091181885E13E
:10FFD00094E10F94000A8AE00E94AA5219821A82C0
:10FFE0001B821C82AE014F5F5F4FBE01675F7F4F78
:10FFF000CE0105960E947DC23394EFCE20E04FA142
:020000021000EC
:10000000BE016F5E7F4FCE010D960E945BFBD62E28
:10001000E72EF82E192FEE8DFF8DEE0FFF1FEE0F3E
:10002000FF1F2CA53DA5E20FF31F862F9E2DAF2DA0
:10003000B12F80839183A283B383312C2D2D3E2D4C
:100040004F2D512F6D2D7E2D8F2D912F0F94E92740
:10005000811102C0332433942D2D3E2D4F2D512F6D
:100060006D2D7E2D8F2D912F0F94E927811121C1A8
:1000700000E0412C512C3201ECA5FDA534E0039F9A
:10008000E00DF11D11242081318142815381C30192
:10009000B2010F94F7242B013C010F5F8EA1801752
:1000A00058F78E8C9F8C9FEF891A990A092C000CA7
:1000B000AA08BB08C501B4010F94081E6E8F7F8F7C
:1000C00088A399A39B01AC01C301B2010F94F12550
:1000D0006AA37BA38CA39DA32A8D3B8D4C8D5D8D44
:1000E0006D2D7E2D8F2D912F0F94011E87FF04C043
:1000F000DA8EEB8EFC8E1D8F2F89388D498D522D17
:100100006D2D7E2D8F2D912F0F945727181624F4C7
:10011000DF8AE88EF98E212EC12C412C512C320120
:10012000ECA5FDA5A4E0CA9EE00DF11D11242AA1B5
:100130003BA14CA15DA160817181828193810F946B
:10014000F6249B01AC010F94671E9B01AC01C30117
:10015000B2010F94F7242B013C01C394BEA1BC153E
:10016000F8F62E8D3F8D48A159A10F94F1250F94DB
:10017000A5272B013C018D8982508E3708F07DC068
:10018000C501B4010E941E536DA97EA980E194E1CE
:100190000F94110A96E7A92E96E0B92EF5018191E8
:1001A0005F01882319F00E94AA52F8CF43E06D2D19
:1001B0007E2D8F2D912F0E943A53FD89F23009F444
:1001C00059C00CE716E0D8018D918D01882319F0F4
:1001D0000E94AA52F8CF44E06AA17BA18CA19DA104
:1001E0000E943A5304E816E0F80181918F018823B8
:1001F00019F00E94AA52F8CF46E0C301B2010E9452
:100200003A530DE816E0D8018D918D01882319F03D
:100210000E94AA52F8CF43E06A8D7B8D8C8D9D8D14
:100220000E943A5304E916E0F80181918F01882376
:1002300019F00E94AA52F8CF43E06F89788D898D1A
:10024000922D0E943A530BE916E0D8018D918D0151
:10025000882319F00E94AA52F8CF2A8D3B8D4C8D2D
:100260005D8D6F89788D898D922D0F94F62443E0F2
:100270000E943A538AE00E94AA52BEA1BF5FBEA369
:1002800040CDE3EFEF8BFFE4F88F23EC298F87EC71
:10029000282E33EF3A8F8FE48B8F93EC9C8FA7E45B
:1002A000AD8F312C412C512C32014AA25BA26CA2A1
:1002B0007DA280E00E94B989332009F46AC085E0FC
:1002C00094E10F944C09BD89BB2309F44DC004EAA5
:1002D00016E0F80181918F01882319F00E94AA523B
:1002E000F8CF46E06AA17BA18CA19DA10E943A5360
:1002F0000BEA16E0D8018D918D01882319F00E9438
:10030000AA52F8CF43E06A8D7B8D8C8D9D8D0E9423
:100310003A5302EB16E0F80181918F01882319F01E
:100320000E94AA52F8CF43E06F89788D898D922D73
:100330000E943A5309EB16E0D8018D918D01882374
:1003400019F00E94AA52F8CF2A8D3B8D4C8D5D8DFD
:100350006F89788D898D922D0F94F62443E00E9449
:100360003A538AE00E94AA5202EC16E0F801819109
:100370008F01882319F00E94AA52F8CF46E0C301EA
:10038000B2010E943A538AE00E94AA528AE00E9477
:10039000AA520E9484C18BAD0F94C2060E947DC4F4
:1003A0002EA53FA50FB6F8943EBF0FBE2DBF07C0C8
:1003B0008EA59FA50FB6F8949EBF0FBE8DBFAEA5AC
:1003C000BFA50FB6F894BEBF0FBEADBFCF5BDF4F6A
:1003D0000FB6F894DEBF0FBECDBFDF91CF911F9156
:1003E0000F91FF90EF90DF90CF90BF90AF909F90D4
:1003F0008F907F906F905F904F903F902F900895D7
:100400002F923F924F925F926F927F928F929F9224
:10041000AF92BF92CF92DF92EF92FF920F931F9312
:10042000CF93DF93CDB7DEB7E5970FB6F894DEBF75
:100430000FBECDBF3090251887E50E94A193882379
:1004400009F4F9C080915F1390916013892B29F40E
:100450000F94310A83EF93E134C08AE50E94EA9356
:10046000882379F00E946A932091FB133091FC134A
:100470004091FD135091FE130F94F6246B017C0103
:1004800008C0C0901518D0901618E0901718F0907A
:10049000181820E030E040E251ECC701B6010F949B
:1004A000572787FD0AC020E030E040E251E4C70151
:1004B000B6010F94011E18163CF40F94310A86EE13
:1004C00093E10F944C09BFC040E050E060EC7FE73F
:1004D00088E50E94FCCF2091F3133091F4134091F2
:1004E000F5135091F6130F94F6242B013C0140E0D4
:1004F00050E060EC7FE789E50E94FCCF2091F71384
:100500003091F8134091F9135091FA130F94F62497
:100510004B015C016FEF89E40E9460A7182F6FEF19
:100520008AE40E9460A7082FA3019201C301B201CF
:100530000F94E927811158C0A5019401C501B401A8
:100540000F94E927811150C0609155137091561393
:10055000072E000C880B990B0F94081E9B01AC0111
:10056000C301B2010F94F62420E030E0A9010F94FA
:10057000F72420E030E0A9010F94F1250F946326C1
:10058000162F6091571370915813072E000C880B8B
:10059000990B0F94081E9B01AC01C501B4010F9487
:1005A000F62420E030E0A9010F94F72420E030E0A9
:1005B000A9010F94F1250F946326062F812F012E98
:1005C000000C990B97FD04C005971CF014E001C0C6
:1005D00010E0802F002E000C990B97FD04C00597AA
:1005E0001CF004E001C000E0153068F5063058F555
:1005F00080E00F94C20625E01202F0011124E00F02
:10060000F11D07FDFA95EE0FFF1FEE0FFF1FE559D5
:10061000FC4EC082D182E282F382A7019601602F54
:10062000812F0E94CECE832D0F94C206332059F025
:100630000E947DC408C08AE40E94A193182F8823D9
:1006400021F00E949D9910E0D6C460E070E086E53C
:100650000E9451A79A8F898F059718F08EEB93E12E
:10066000A1C260E084E40E94F793282E40E050E0AD
:10067000BA018AE50E94FCCF6DA77EA78FA798AB31
:1006800040E050E86BEB75E483E50E94FCCF20E08E
:1006900030E040E752E40F94F12560935F027093DD
:1006A0006002809361029093620288E40E94A193A9
:1006B000882309F40BC10E946A930F946326698B07
:1006C0007A8B8B8B9C8B69887A888090FF139090B3
:1006D0000014A0900114B090021420E030E0A901B1
:1006E000C501B4010F94F724D62EE72EF82E092F5A
:1006F00020E030E040E450E40F94011E87FF05C085
:10070000D12CE12CF0E4FF2E00E469897A8977FE90
:1007100002C06F5F7F4F7595679588279927861B65
:10072000970B9E8B8D8BBC0163517F4F072E000C66
:10073000880B990B0F94081E562E672E782EC92E03
:100740002D2D3E2D4F2D502F0F94572718161CF48A
:10075000D52C73010C2D6D2D7E2D8F2D902F0F9488
:1007600063266B017C012B0120E030E84DEE53E461
:10077000C501B4010F94F724962EA72EB82E092F89
:1007800020E030E84BEE53E40F945727181634F46A
:10079000912C60E8A62E7BEEB72E03E469897A8956
:1007A0006C0D7D1D072E000C880B990B0F94081EF5
:1007B0006B017C01292D3A2D4B2D502F0F94011EDA
:1007C00087FF04C09C2CAD2CBE2C0F2D692D7A2DDB
:1007D0008B2D902F0F946326788F6F8B809003144E
:1007E00090900414A0900514B090061420E030E01E
:1007F000A901C501B4010F94F724D62EE72EF82ED7
:10080000092F20E030E040E450E40F94011E87FF00
:1008100005C0D12CE12C50E4F52E00E46D897E89D1
:100820006F517F4F072E000C880B990B0F94081EF9
:100830006D8B672E782EC92E2D2D3E2D4F2D502FCE
:100840000F94572718161CF4DD8873010C2D6D2D9D
:100850007E2D8F2D902F0F9463266B017C013B0121
:1008600020E030E041EE53E4C501B4010F94F724D9
:10087000962EA72EB82E092F20E030E84FED53E436
:100880000F945727181634F4912C30E8A32E4FED0F
:10089000B42E03E469897A896C0D7D1D072E000C46
:1008A000880B990B0F94081E6B017C01292D3A2DA2
:1008B0004B2D502F0F94011E87FF04C09C2CAD2C94
:1008C000BE2C0F2D692D7A2D8B2D1FC18CE40E941B
:1008D000EA93882369F00E946A932091F313309180
:1008E000F4134091F5135091F6130F94F6242BC096
:1008F00020E030E0A9016091FF1370910014809115
:100900000114909102140F94F7246B017C0120E0F4
:1009100030E040E450E40F94011E87FD0DC020E05C
:1009200030E0A901C701B6010F94011E87FF09C07D
:10093000C12CD12C760105C0C12CD12C20E4E22E93
:10094000FE2CC701B6010F9463262B0182E50E949D
:10095000EA93882369F00E946A932091F3133091FF
:10096000F4134091F5135091F6130F94F6243CC004
:1009700020E030E84DEE53E46091FF1370910014D5
:1009800080910114909102140F94F724D62EE72E33
:10099000F82E092F20E030E84BEE53E40F94572750
:1009A000181634F4D12C80E8E82E9BEEF92E03E4DF
:1009B000B20165527E4F072E000C880B990B0F94E5
:1009C000081E962EA72EB82EC92E2D2D3E2D4F2D4A
:1009D000502F0F94011E87FF03C0D92C75010C2DD9
:1009E0006D2D7E2D8F2D902F0F946326788F6F8B1A
:1009F00086E40E94EA93882369F00E946A9320911A
:100A0000F7133091F8134091F9135091FA130F94A2
:100A1000F6242BC020E030E0A9016091031470910E
:100A2000041480910514909106140F94F7246B011F
:100A30007C0120E030E040E450E40F94011E87FD8B
:100A40000DC020E030E0A901C701B6010F94011EDE
:100A500087FF09C0C12CD12C760105C0C12CD12C37
:100A600000E4E02EFE2CC701B6010F9463263B0183
:100A700082E40E94EA93882369F00E946A9320919D
:100A8000F7133091F8134091F9135091FA130F9422
:100A9000F6243CC020E030E041EE53E460910314C2
:100AA0007091041480910514909106140F94F7240A
:100AB000D62EE72EF82E092F20E030E84FED53E434
:100AC0000F945727181634F4D12CA0E8EA2EBFED66
:100AD000FB2E03E4B3016E537E4F072E000C880BF0
:100AE000990B0F94081E962EA72EB82EC92E2D2DC9
:100AF0003E2D4F2D502F0F94011E87FF03C0D92C80
:100B000075010C2D6D2D7E2D8F2D902F0F9463264A
:100B10007B01B301072C000C880B990B0F94081E66
:100B20006C8F7D8F8E8F9F8F69837A838B839C835D
:100B3000B201052C000C880B990B0F94081E68A3BA
:100B400079A38AA39BA36D837E838F839887BE013D
:100B50006F5F7F4FCE0105960E941CA6882301F18E
:100B6000B7010F2C000C880B990B0F94081E698796
:100B70007A878B879C87AF89B88DBD01BB0F880BA7
:100B8000990B0F94081E6D877E878F87988BBE0107
:100B9000675F7F4FCE010D960E941CA6813029F021
:100BA00082EA93E10F944C0926C2298D3A8D232BBA
:100BB00069F08CE893E10F944C09222021F082E83F
:100BC00093E10F944C098AE00E94AA520E945F8C24
:100BD00080E00F94C20681E00E94B989882321F049
:100BE000832D0F94C2062FCD0F89188D0419150976
:100BF00017FF02C00D5F1F4F1595079515950795B7
:100C0000B801012E000C880B990B0F94081E6CA3E1
:100C10007DA38EA39FA3E618F708F7FE03C033E079
:100C2000E30EF11C5701B594A794B594A794B501B0
:100C30000B2C000C880B990B0F94081E68A779A742
:100C40008AA79BA70E949DC160915F13709160135A
:100C5000072E000C880B990B0F94081E9B01AC010A
:100C60006CA17DA18EA19FA10F94011E811122C0B4
:100C70006091611370916213072E000C880B990B21
:100C80000F94081E9B01AC0168A579A58AA59BA5B8
:100C90000F94011E81110EC080915513909156132F
:100CA0004816590639F480915713909158136816D5
:100CB000790699F00E949D991093601300935F1339
:100CC000B0926213A0926113509256134092551342
:100CD0007092581360925713312C60E085E40E94A3
:100CE000F793882319F061E06CA702C082E08CA71B
:100CF00091E09B8FE12CF12C812C912C5401A1E0EF
:100D0000A98BB1E0BD8B25E02F8B10E075E5C72ED8
:100D100073E1D72EE9AAA989B1E0AB27A98B0B8D86
:100D2000C7010F2C000CAA0BBB0B8AAB9BABACAB67
:100D3000BDAB9F89911709F4BEC0612F012E000C35
:100D4000770B880B990B0F94081E2CA13DA14EA187
:100D50005FA10F94671E28A139A14AA15BA10F943E
:100D6000F7242B013C016AA97BA98CA99DA90F94AA
:100D7000081E28A539A54AA55BA50F94671E2C8DD2
:100D80003D8D4E8D5F8D0F94F7244B015C0120E06B
:100D900030E0A901C301B2010F94011E87FF04C016
:100DA00020E030E0A90104C020E030E040E05FE353
:100DB000C301B2010F94F7240F94992669837A83B3
:100DC0008B839C8320E030E0A901C501B4010F941E
:100DD000011E87FF04C020E030E0A90104C020E02C
:100DE00030E040E05FE3C501B4010F94F7240F94B5
:100DF00099266D837E838F839887A98DBA8DAB2BBF
:100E000081F0602F70E08EE693E10F94110A69E1A2
:100E100070E08CE693E10F94110A89E693E10F9458
:100E20004C091F92B9E1BF931F920F93DF92CF92AB
:100E30001F920E949D7C298D4CA5BE016B5F7F4F48
:100E4000CE0101960E945BFB4B015C010FB6F8944A
:100E5000DEBF0FBECDBF9B01AC010F94E9278823F5
:100E600021F0832D0F94C20633C0A50194016DA516
:100E70007EA58FA598A90F94F7249B01AC0165E08E
:100E80001603F0011124EE0DFF1DEE0FFF1FEE0FF4
:100E9000FF1FE559FC4E208331834283538369A9A8
:100EA000812F0E94CECE80E00E94D6530F5F8D89A5
:100EB000180F312C3ECF94E0E916F10449F0A5015A
:100EC0009401C501B4010F94E927882309F47EC079
:100ED0000E947AEE80E00E94B989882351F0832D28
:100EE0000F94C206812C912C90ECA92E9FE7B92E6D
:100EF00052C0A5019401C501B4010F94E9278111E5
:100F00004AC0222001F10F945B090F9408072110B9
:100F10003FC08DE098E10F94A9049B01AC01609162
:100F200015187091161880911718909118180F9431
:100F3000F6246093151870931618809317189093E1
:100F4000181881E026C012E084E0F82E02E0EF2CB1
:100F5000E11ADF2CD01A21E041E0602F812F0F949D
:100F6000750721E04FEF602F8E2D0F9475072FEF3F
:100F700041E06D2D812F0F9475072FEF4FEF6D2DF1
:100F80008E2D0F947507015020F71150F8F6BBCF46
:100F9000832D809325180E9484C18091251881118A
:100FA0000E9448C30E9471890E945F8C89E493E18A
:100FB0000E94F1BB0E947DC411E0A5019401C5010E
:100FC000B4010F94E927811116C03DCBA989AA234A
:100FD00061F031E03D8B65E06F8B10E08FEFE81A38
:100FE000F80A9B8D9B5F9B8F95CEBFEFBD8B2FEF3C
:100FF0002F8B14E0F3CF812FE5960FB6F894DEBF68
:101000000FBECDBFDF91CF911F910F91FF90EF9059
:10101000DF90CF90BF90AF909F908F907F906F9018
:101020005F904F903F902F90089580919A159091E6
:101030009B15891B8F708F3021F480E00E94D6535E
:10104000F4CF80919A158F5F8F70E0919A1598E494
:101050009E9FF0011124EF5DF34FDF011D929A95E1
:10106000E9F798E090834091B0155091B1156091E7
:10107000B2157091B315458B568B678B708F40916D
:10108000B4155091B5156091B6157091B715418F93
:10109000528F638F748F4091B8155091B91560913C
:1010A000BA157091BB15458F568F678F70A340910D
:1010B000BC155091BD156091BE157091BF1541A32F
:1010C00052A363A374A320919A1590919B152913A1
:1010D00003C094E69093971580939A1580916F00C2
:1010E000826080936F0008950F930FB70F93009164
:1010F0006E000F930B7F00936E0000916F000D7FC9
:1011000000936F000F930BB70F930CB70F921F92C2
:101110002F933F934F935F936F937F938F939F93FF
:10112000AF93BF93EF93FF9311240E94C79EFF914B
:10113000EF91BF91AF919F918F917F916F915F914F
:101140004F913F912F911F900F900CBF0F910BBFAC
:101150000F910260F89400936F000F9100936E005E
:101160000F910FBF0F91189580918E0980FF03C0DA
:1011700089988FEF02C0899A81E080932E11809127
:101180008E09869580FF03C08F9A8FEF02C08F98DB
:1011900081E080932F1180918E098695869580FF3E
:1011A00008C080910B0180958270809309018FEFB8
:1011B00006C080910B0182708093090181E08093C9
:1011C000301180918E0986958695869580FF03C0A3
:1011D00016988FEF02C0169A81E0809331110000BB
:1011E00000000000089580919A1590919B15891B2D
:1011F0008F7019F480E090E00895909197159923ED
:1012000051F0833030F48FEF890F19F080939715E8
:10121000F1CF10929715E0919B1588E4E89FF001BB
:101220001124EF5DF34F808180FDE4CF80919B1509
:101230008F5F8F708093981590919B158091991571
:10124000981304C08091981580939915CF01089543
:101250001F93CF93DF93CDB7DEB728970FB6F894DF
:10126000DEBF0FBECDBF69837A838B839C832D83C2
:101270003E834F8358870E94B698882311F081E0FF
:1012800026C081E00E947F7C69E170E080E090E010
:101290000F941D09BE016B5F7F4FCE0101960E9426
:1012A0009FC21091210B147080E00E947F7C11235B
:1012B00021F00E9467988111E2CF1092210B82E009
:1012C0000E94DAC20E9448C381E0111180E0289692
:1012D0000FB6F894DEBF0FBECDBFDF91CF911F9147
:1012E0000895CF92DF92EF92FF92CF93DF93CDB725
:1012F000DEB728970FB6F894DEBF0FBECDBF20E053
:1013000030E040EA50E46091151870911618809111
:101310001718909118180F94011E8823E9F01D8268
:101320001E821F821886C12CD12C80EAE82E80E410
:10133000F82EC982DA82EB82FC82BE016B5F7F4F9E
:10134000CE0101960E949FC2C0921518D092161825
:10135000E0921718F092181828960FB6F894DEBF8E
:101360000FBECDBFDF91CF91FF90EF90DF90CF9078
:101370000895BF92CF92DF92EF92FF920F931F9347
:10138000CF93DF93CDB7DEB728970FB6F894DEBFC3
:101390000FBECDBF90918F09981709F47AC0B82E6F
:1013A00080E090E0A0E2B1E48D839E83AF83B887B4
:1013B000C0900714D0900814E0900914F0900A141B
:1013C00020E030E0A901C701B6010F94011E87FF9C
:1013D0000CC0A701960160E070E080E291E40F94F8
:1013E000F6246D837E838F83988720E030E04BEE78
:1013F00053E46D817E818F8198850F94572718164D
:1014000044F480E090E0ABEEB3E48D839E83AF8341
:10141000B8872D813E814F81588560911518709154
:10142000161880911718909118180F94011E87FFB5
:101430000BC019821A821B821C82BE016F5F7F4F14
:10144000CE0105960E949FC260910D1870910E18F2
:1014500080910F1890911018209111183091121846
:10146000409113185091141819821A821B821C8201
:10147000E0901518F0901618009117181091181890
:10148000FE0131966F010E94BCC1B0928F090E948B
:10149000F2C580E028960FB6F894DEBF0FBECDBF30
:1014A000DF91CF911F910F91FF90EF90DF90CF9040
:1014B000BF900895CF93DF93C091181187ED96E008
:1014C0000E94B55380911311873009F445C083E021
:1014D0008093121181E08093290280E190E0909343
:1014E0001D1680931C1685E080931016D2E8D093C9
:1014F000131684E190E1A0E0B0E08093141690937D
:101500001516A0931616B09317160F94800161E07C
:1015100070E080E090E00E94B3CE81E09AE5909385
:101520001D1680931C1685E390E090931F16809300
:101530001E1687E080931016D093131684E890E06F
:10154000A0E0B0E08093141690931516A0931616A1
:10155000B09317160F948001C13081F1C23059F455
:101560000E94A6EC60930A1170930B1180930C11EA
:1015700090930D1102C00E94DAEC81E08093181163
:101580000F94060160930611709307118093081160
:1015900090930911C230A1F080917C0990917D094E
:1015A000019690937D0980937C09109219111092F5
:1015B0001A1110921B1110921C1102C080E001C080
:1015C00081E0DF91CF910895CF93DF9300D01F92F8
:1015D000CDB7DEB780917B098823A9F083E390E043
:1015E0009C838B831A8219829E012F5F3F4F40E1BB
:1015F00050E06CE779E0CE0103960E94AD508FEE8B
:1016000096E00E94B5530F900F900F900F90DF91CE
:10161000CF910895CF92DF92EF92FF920F931F9395
:10162000809118118150823010F080E0A7C08BE2C9
:1016300097E00E94B55380911311833009F441C0A3
:101640008FE097E00E94B5538BE197E00E94B5537D
:1016500040E060E070E0CB010E949CEE41E060E081
:1016600070E0CB010E949CEE81E080930502109215
:10167000111121E030E03093101120930F1180936D
:10168000290281E09AE590931D1680931C168DE245
:1016900090E090931F1680931E1687E0809310169B
:1016A00082E88093131684E890E0A0E0B0E0809395
:1016B000141690931516A0931616B09317160F9440
:1016C0008001109218110F94060160931411709309
:1016D0001511809316119093171180917E099091A6
:1016E0007F09019690937F0980937E09C09019111C
:1016F000D0901A11E0901B11F0901C110E94A6ECE2
:101700006093191170931A1180931B1190931C11FF
:1017100000918009109181092091820930918309FB
:101720000C191D092E093F09DC01CB01800F911F07
:10173000A21FB31F8093800990938109A09382090F
:10174000B09383090E94A6EC009184091091850949
:10175000209186093091870906171707280739074E
:1017600050F40E94A6EC60938409709385098093DD
:101770008609909387090E94E48A81E01F910F9166
:10178000FF90EF90DF90CF900895CF93DF9300D03C
:101790001F921F92CDB7DEB781E080937B09ECE703
:1017A000F9E080E1DF011D928A95E9F70E94E48A61
:1017B00086E18D8382E390E09C838B831A82198279
:1017C0009E012F5F3F4F41E050E0BE016B5F7F4FB6
:1017D000CE0103960E94AD500F900F900F900F9086
:1017E0000F90DF91CF910895CF92DF92EF92FF9209
:1017F0000F931F93CF93DF93C4EAD0E103EE1BE076
:10180000C12CD12C7601C3946991799189919991D8
:101810000F94061E288939894A895B890F94671EAF
:101820000F946A26F80161937193819391938F01CC
:10183000C616D706E806F90610F46B017C01F0E144
:10184000C43BDF0709F76FEF7FEFCB01A7019601DC
:101850000F9457242093F30B3093F40B4093F50B24
:101860005093F60BDF91CF911F910F91FF90EF9066
:10187000DF90CF9008950F931F93CF93DF9308EBE2
:1018800010E1C9EFDBE0F8012191319141915191D3
:101890008F0160E070E080E89FE30F94F125699389
:1018A000799389939993FCE0C930DF0761F70E942F
:1018B000257CDF91CF911F910F910C94F48B909127
:1018C0009A1580919B15981306C08091A110909154
:1018D000A210892B21F080E00E94D653F0CF08950A
:1018E0002091C4103091C5104091C6105091C7107E
:1018F000FC0160817181828193810F94671E0F9436
:1019000064276093BC157093BD158093BE159093AA
:10191000BF1590919A1580919B1598130C9415887A
:101920000E945F8C80916F00982F927081FF05C09C
:1019300080916F008D7F80936F004091BC15509116
:10194000BD156091BE157091BF1540935011509315
:1019500051116093521170935311992329F0809182
:101960006F00826080936F000895EF92FF920F9353
:101970001F93CF93DF937B018A01E9012091B81077
:101980003091B9104091BA105091BB10FC016081A8
:101990007181828193810F94671E0F9464276093F5
:1019A000B0157093B1158093B2159093B315209133
:1019B000BC103091BD104091BE105091BF10F70186
:1019C00060817181828193810F94671E0F946427D7
:1019D0006093B4157093B5158093B6159093B715B1
:1019E0002091C0103091C1104091C2105091C3108D
:1019F000F80160817181828193810F94671E0F9439
:101A000064276093B8157093B9158093BA159093B5
:101A1000BB152091C4103091C5104091C610509153
:101A2000C710688179818A819B810F94671E0F940A
:101A300064276093BC157093BD158093BE15909379
:101A4000BF1590919A1580919B15981741F0DF91E1
:101A5000CF911F910F91FF90EF900C9415880E94E9
:101A60005F8C80916F00982F927081FF05C08091EC
:101A70006F008D7F80936F004091B0155091B1152C
:101A80006091B2157091B315409344115093451174
:101A900060934611709347114091B4155091B5155C
:101AA0006091B6157091B715409348115093491144
:101AB00060934A1170934B114091B8155091B9152C
:101AC0006091BA157091BB1540934C1150934D1114
:101AD00060934E1170934F114091BC155091BD15FC
:101AE0006091BE157091BF154093501150935111E4
:101AF0006093521170935311992329F080916F00D4
:101B0000826080936F00DF91CF911F910F91FF90C2
:101B1000EF900895CF93DF93C82F0E94969E24E004
:101B2000C29FE0011124C750D44F0F94081E288192
:101B300039814A815B810F94671EDF91CF910895AF
:101B400090919A1580919B15981306C08091A110D1
:101B50009091A210892B21F080E00E94D653F0CF03
:101B60005F9A809114148E7F809314148A9A8091C6
:101B700014148D7F809314148091080180958170D6
:101B800080930601809114148B7F809314140C941D
:101B90001950CF93DF9390916F00292F227091FFFE
:101BA00005C090916F009D7F90936F0094E0899F96
:101BB000A0011124FA01E85CFE4E608171818281EE
:101BC0009381222329F020916F00226020936F00DF
:101BD000EA01C750D44F0F94081E288139814A81E9
:101BE0005B810F94671EDF91CF91089580916F0004
:101BF000982F927081FF05C080916F008D7F809338
:101C00006F0080919B1580939A158093991580930E
